:020000040800F2
:1000000000060020E10100086D0E0008ED0D00085B
:10001000450E0008ED0D0008190E0008E301000868
:10002000E3010008E3010008E301000841210008A2
:10003000E3010008E3010008E3010008E301000810
:10004000E3010008E3010008E3010008E301000800
:10005000E3010008E3010008093200083532000816
:10006000613200088D320008B9320008E30100084F
:10007000E3010008E3010008E3010008E3010008D0
:10008000E3010008E3010008E3010008E3010008C0
:10009000E3010008E3010008E3010008E53200087D
:1000A000E3010008E3010008E3010008E3010008A0
:1000B0007D300008E3010008E3010008E3010008C7
:1000C000E3010008E3010008E3010008E301000880
:1000D000E3010008E3010008E3010008E301000870
:1000E0004D330008E3010008E3010008E3010008C4
:1000F000E3010008E3010008E3010008E301000850
:10010000E3010008E3010008E3010008E30100083F
:10011000E3010008E3010008E3010008E30100082F
:10012000E3010008E3010008E3010008E30100081F
:10013000E3010008E3010008E3010008E30100080F
:10014000E3010008E3010008E30100087928000842
:10015000E3010008E3010008E3010008E3010008EF
:10016000E3010008E3010008E3010008E3010008DF
:10017000E3010008E3010008E3010008E3010008CF
:10018000E3010008E3010008E3010008E3010008BF
:10019000E3010008E3010008E3010008E3010008AF
:1001A000E3010008E3010008E3010008E30100089F
:1001B000E3010008E3010008E3010008E30100088F
:1001C000E3010008E3010008E3010008E30100087F
:1001D000E3010008E3010008E3010008E30100086F
:1001E00002E000F000F8FEE772B63A4880F30888B3
:1001F000394880F3098839484EF60851CEF200019B
:10020000086040F20000CCF200004EF63471CEF2ED
:1002100000010860BFF34F8FBFF36F8F40F2000003
:10022000C0F2F0004EF68851CEF200010860BFF334
:100230004F8FBFF36F8F4FF00000E1EE100A4EF6C4
:100240003C71CEF200010860062080F31488BFF3F1
:100250006F8F01F0F5FF01F0D1FF02F073FE4FF058
:1002600055301F491B4A91423CBF41F8040BFAE745
:100270001C49194A91423CBF41F8040BFAE71A495C
:100280001A4A1B4B9A423EBF51F8040B42F8040B2A
:10029000F8E700201749184A91423CBF41F8040B87
:1002A000FAE701F0AFFF02F0A1FE144C144DAC428E
:1002B00003DA54F8041B8847F9E700F041F8114CC1
:1002C000114DAC4203DA54F8041B8847F9E701F0FA
:1002D00097BF000000060020002200200000000858
:1002E00000000020000600207837000800220020CF
:1002F0004022002040220020A82D0020E00100081C
:10030000E0010008E0010008E00100082DE9F04FDD
:100310002DED108AC1F80CD0C3689D46BDEC108A43
:10032000BDE8F08F002383F311882846A047002002
:1003300001F012FBFEE701F08DFA00DFFEE700009E
:1003400038B501F0CDFE054601F0F0FE0446D8B9FF
:100350000F4B9D421AD001339D4218BF044641F213
:10036000883504BF01240025002001F0C3FE0CB134
:1003700000F076F800F010FD00F09EFB284600F03B
:10038000BFF800F06DF8F9E70025EDE70546EBE76B
:10039000010007B008B500F061FBA0F1200358424E
:1003A000584108BD07B541F21203022101A8ADF87A
:1003B000043000F071FB03B05DF804FB38B5202376
:1003C00083F311881748C3680BB101F04BFB164A41
:1003D000144800234FF47A7101F008FB002383F3E3
:1003E0001188124C236813B12368013B23606368B2
:1003F00013B16368013B63600D4D2B7833B96368BB
:100400007BB9022000F042FC322363602B78032B7F
:1004100007D163682BB9022000F038FC4FF47A73DF
:10042000636038BD40220020BD0300085C2300202B
:1004300054220020084B187003280CD8DFE800F085
:1004400008050208022000F017BC022000F00ABCD8
:10045000024B00225A607047542200205C23002087
:10046000234B244A10B51C46196801313FD0043390
:100470009342F9D16268A24239D31F4B9B6803F1C2
:10048000006303F540439A4231D2002000F02EFB76
:100490000220FFF7CFFF194B1A6C00221A64196E65
:1004A0001A66196E596C5A64596E5A665A6E5A69B0
:1004B00042F080025A615A6922F080025A615A69F8
:1004C0001A6942F000521A611A6922F000521A6148
:1004D0001B6972B64FF0E0232021C3F8084DD4E920
:1004E000003281F311889D4683F30888104710BDC0
:1004F00000C0000820C00008002200200038024090
:100500002DE9F04F93B0A94B00902022FF210AA8BB
:100510009D6800F0EBFBA64A1378A3B9A54801211A
:10052000C3601170202383F31188C3680BB101F0FD
:1005300099FAA14A9F4800234FF47A7101F056FAC4
:10054000002383F31188009B13B19C4B009A1A601F
:100550009B4A009C1378032B1EBF00231370974AFD
:100560004FF0000A18BF5360D3465646D1460120CB
:1005700000F082FB24B1914B1B68002B00F00F822E
:10058000002000F06BFA0390039B002BF2DB0120AC
:1005900000F068FB039B213B162BE8D801A252F820
:1005A00023F000BF0106000829060008BD06000868
:1005B0006F0500086F0500086F0500084507000873
:1005C000130900082D0800088F080008B708000864
:1005D000DD0800086F050008EF0800086F05000837
:1005E00061090008A10600086F050008A5090008B8
:1005F0000D060008A10600086F0500088F08000816
:100600000220FFF7C7FE002840F0F381009B022183
:10061000BAF1000F08BF1C4605A841F21233ADF82D
:10062000143000F039FAA2E74FF47A7000F016FAAD
:10063000071EEBDB0220FFF7ADFE0028E6D0013FEE
:10064000052F00F2D881DFE807F0030A0D101336FA
:1006500005230593042105A800F01EFA17E053486E
:100660000421F9E757480421F6E757480421F3E746
:100670004FF01C08404600F03BFA08F104080590D2
:10068000042105A800F008FAB8F12C0FF2D10120DE
:1006900000FA07F747EA0B0B5FFA8BFB4FF00009F4
:1006A00000F070FB26B10BF00B030B2B08BF0024EE
:1006B000FFF778FE5BE745480421CDE7002EA5D083
:1006C0000BF00B030B2BA1D10220FFF763FE0746B3
:1006D00000289BD0012000F009FA0220FFF7AAFEB3
:1006E00000265FFA86F8404600F010FA044688B10A
:1006F000404600F01BFA01360028F2D1BA46044603
:1007000041F21213022105A8ADF814303E4600F064
:10071000C3F92CE70120FFF78DFE2546234B9B688C
:10072000AB4207D9284600F0E3F9013040F066817A
:100730000435F3E7224B00251D70204BBA465D605F
:100740003E46ADE7002E3FF461AF0BF00B030B2BE1
:100750007FF45CAF0220FFF76DFE322000F07EF9DF
:10076000B0F10008FFF652AF18F003077FF44EAF68
:100770000E4A926808EB050393423FF647AFB8F57F
:10078000807F3FF743AF124B0193B84522DD4FF412
:100790007A7000F063F90390039A002AFFF636AFEF
:1007A000019B039A03F8012B0137EDE7002200209B
:1007B0005823002040220020BD0300085C230020B5
:1007C0005422002004220020082200200C220020B5
:1007D00058220020C820FFF7DDFD074600283FF41F
:1007E00015AF1F2D11D8C5F1200242450AAB25F0E7
:1007F000030028BF424683490192184400F050FA92
:10080000019A8048FF2100F071FA4FEAA8037D4960
:100810000193C8F38702284600F070FA06460028C4
:100820003FF46EAF019B05EB830539E70220FFF72C
:10083000B1FD00283FF4EAAE00F0A2F900283FF431
:10084000E5AE0027B846704B9B68BB4218D91F2FF6
:1008500011D80A9B01330ED027F0030312AA1344C8
:1008600053F8203C05934046042205A900F000FB04
:1008700004378046E7E7384600F03AF90590F2E79A
:10088000CDF81480042105A800F006F908E700233C
:10089000642104A8049300F0F5F800287FF4B6AEB4
:1008A0000220FFF777FD00283FF4B0AE049800F077
:1008B0004FF90590E6E70023642104A8049300F0B3
:1008C000E1F800287FF4A2AE0220FFF763FD0028C4
:1008D0003FF49CAE049800F04BF9EAE70220FFF7E2
:1008E00059FD00283FF492AE00F05AF9E1E70220EA
:1008F000FFF750FD00283FF489AE05A9142000F051
:1009000055F904210746049004A800F0C5F83946BB
:10091000B9E7322000F0A2F8071EFFF677AEBB075A
:100920007FF474AE384A926807EB090393423FF6AE
:100930006DAE0220FFF72EFD00283FF467AE27F0D2
:1009400003074F44B9453FF4ABAE484600F0D0F83A
:100950000421059005A800F09FF809F10409F1E7CA
:100960004FF47A70FFF716FD00283FF44FAE00F009
:1009700007F9002844D00A9B01330BD008220AA9AA
:10098000002000F0BBF900283AD02022FF210AA85D
:1009900000F0ACF9FFF706FD1C4800F0E3FF13B0D0
:1009A000BDE8F08F002E3FF431AE0BF00B030B2BA4
:1009B0007FF42CAE0023642105A8059300F062F8B3
:1009C000074600287FF422AE0220FFF7E3FC8046B2
:1009D00000283FF41BAEFFF7E5FC41F2883000F041
:1009E000C1FF059800F000FA464600F0CBF93C46FE
:1009F000BDE5064654E64FF0000907E6BA467FE635
:100A000037467DE65822002000220020A086010003
:100A100070B50F4B1B780133DBB2012B0C4611D89C
:100A20000C4D29684FF47A730E6AA2FB033201461B
:100A300022462846B047844204D1074B00221A7050
:100A4000012070BD4FF4FA7000F08CFF0020F8E731
:100A500010220020502500209023002007B50023FD
:100A6000024601210DF107008DF80730FFF7D0FF96
:100A700020B19DF8070003B05DF804FB4FF0FF3094
:100A8000F9E700000A4608B50421FFF7C1FF80F02E
:100A90000100C0B2404208BD30B4054C2368DD6996
:100AA000044B0A46AC460146204630BC604700BFB6
:100AB00050250020A086010070B501F003FA094E10
:100AC000094D3080002428683388834208D901F01A
:100AD000F3F92B6804440133B4F5404F2B60F2D393
:100AE00070BD00BF922300206423002001F0ACBA47
:100AF00000F1006000F540400068704700F10060C0
:100B0000920000F5404001F02BBA0000054B1A6836
:100B1000054B1B889B1A834202D9104401F0CCB9C3
:100B200000207047642300209223002038B5074D31
:100B300004462868204401F0C7F928B928682044F1
:100B4000BDE8384001F0D8B938BD00BF64230020AB
:100B500010F003030AD1B0F5047F05D200F1005074
:100B6000A0F51040D0F80038184670470023FBE786
:100B700000F10050A0F51040D0F8100A70470000B6
:100B8000064991F8243033B10023086A81F82430F3
:100B90000822FFF7B3BF0120704700BF6823002081
:100BA000014B1868704700BF002004E070B52A4B65
:100BB0001B68C3F30B0204461B0C62B140F21340E6
:100BC000824230D040F2194082422ED040F2214081
:100BD00082422CD10322214D0C2000FB0252556889
:100BE00042F20102934224D0B3F5805F23D041F258
:100BF0000102934221D041F2030293421FD041F2FD
:100C00000702934214BF3F233123013C0C44013DB2
:100C10000A46A24215D215F9016F501C9EB100F888
:100C2000016C0246F5E70122D5E70222D3E70C4D1D
:100C3000D6E73323E9E74123E7E75A23E5E75923DA
:100C4000E3E7104605E02C258442157001D9901C7D
:100C50005370401A70BD00BF002004E078340008D3
:100C60004C340008022802BF024B4FF080729A6198
:100C7000704700BF00080240022802BF024B4FF439
:100C800080729A61704700BF00080240022801BFCD
:100C9000024A536983F4807353617047000802402D
:100CA00010B50023934203D0CC5CC4540133F9E760
:100CB00010BD000010B5013810F9013F3BB191F9AA
:100CC00000409C4203D11AB10131013AF4E71AB154
:100CD00091F90020981A10BD1046FCE70346024621
:100CE000D01A12F9011B0029FAD1704702440346B9
:100CF000934202D003F8011BFAE770472DE9F8434D
:100D00001F4D144695F824200746884652BBDFF84D
:100D100070909CB395F824302BB92022FF214846CF
:100D20002F62FFF7E3FF95F82400C0F10802A2420A
:100D300028BF2246D6B24146920005EB8000FFF75D
:100D4000AFFF95F82430A41B1E44F6B2082E1744BA
:100D50009044E4B285F82460DBD1FFF711FF00284E
:100D6000D7D108E02B6A03EB82038342CFD0FFF791
:100D700007FF0028CBD10020BDE8F8830120FBE766
:100D800068230020024B1A78024B1A70704700BF8C
:100D9000902300201022002010B50F4C0F4800F0C7
:100DA000F7F821460D4800F01FF924680C48626DE1
:100DB000D2F8043843F00203C2F8043800F0D2FD40
:100DC0000849204600F016FA626DD2F8043823F084
:100DD0000203C2F8043810BD6C350008502500200D
:100DE00040420F00743500087047000000B59BB00A
:100DF000EFF3098168226846FFF752FFEFF305839E
:100E0000044B9A6BDA6A9A6A9A6A9A6A9A6A9A6A36
:100E10009B6AFEE700ED00E000B59BB0EFF30981AF
:100E200068226846FFF73CFFEFF30583044B9A6B9B
:100E30009A6A9A6A9A6A9A6A9A6A9B6AFEE700BFF5
:100E400000ED00E000B59BB0EFF309816822684631
:100E5000FFF726FFEFF30583034B5A6B9A6A9A6AF2
:100E60009A6A9A6A9B6AFEE700ED00E0FEE70000DE
:100E700030B5094D0A4491420DD011F8013B58405C
:100E8000082340F30004013B2C4013F0FF0384EAE5
:100E90005000F6D1EFE730BD2083B8ED026843681B
:100EA0001143016003B118477047000013B5446B4C
:100EB000D4F894341A681178042915D1217C0229B8
:100EC00012D11979128901238B4013420CD101A947
:100ED00004F14C0001F03CFFD4F89444019B2179CB
:100EE0000246206800F0CEF902B010BD143001F0C7
:100EF000BFBE00004FF0FF33143001F0B9BE000058
:100F00004C3001F091BF00004FF0FF334C3001F046
:100F10008BBF0000143001F08DBE00004FF0FF3198
:100F2000143001F087BE00004C3001F05DBF0000BE
:100F30004FF0FF324C3001F057BF000000207047E7
:100F400010B5D0F894341A6811780429044617D1E2
:100F5000017C022914D15979528901238B40134213
:100F60000ED1143001F020FE024648B1D4F894446A
:100F70004FF4807361792068BDE8104000F070B9CB
:100F800010BD0000406BFFF7DBBF000070470000A2
:100F90007FB5124B036000234360C0E90233012593
:100FA00002260F4B057404460290019300F184025F
:100FB000294600964FF48073143001F0D1FD094B9F
:100FC0000294CDE9006304F523724FF4807329463F
:100FD00004F14C0001F098FE04B070BDA834000884
:100FE000850F0008AD0E00080B68202282F31188DF
:100FF0000A7903EB820290614A79093243F82200B0
:101000008A7912B103EB8203986102230374C0F85A
:101010009414002383F311887047000038B5037FD0
:10102000044613B190F85430ABB9201D01250221BC
:10103000FFF734FF04F1140025776FF0010100F091
:10104000B9FC84F8545004F14C006FF00101BDE884
:10105000384000F0AFBC38BD10B501210446043063
:10106000FFF71CFF0023237784F8543010BD0000E5
:1010700038B504460025143001F08AFD04F14C0017
:10108000257701F059FE201D84F854500121FFF707
:1010900005FF2046BDE83840FFF752BF90F84430C6
:1010A00003F06003202B07D190F84520212A4FF050
:1010B000000303D81F2A06D800207047222AFBD13C
:1010C000C0E90E3303E0034A82630722C26303646C
:1010D000012070471122002037B5D0F894341A68E7
:1010E0001178042904461AD1017C022917D11979F3
:1010F000128901238B40134211D100F14C0528467F
:1011000001F0DAFE58B101A9284601F021FED4F819
:101110009444019B21790246206800F0B3F803B0A3
:1011200030BD0000F0B500EB810385B09E69044638
:101130000D46FEB1202383F3118804EB8507301D93
:101140000821FFF7ABFEFB685B691B6806F14C00EA
:101150001BB1019001F00AFE019803A901F0F8FD0E
:10116000024648B1039B2946204600F08BF8002335
:1011700083F3118805B0F0BDFB685A691268002A34
:10118000F5D01B8A013B1340F1D104F14402EAE798
:10119000093138B550F82140DCB1202383F31188A0
:1011A000D4F894241368527903EB8203DB689B69BB
:1011B0005D6845B104216018FFF770FE294604F10F
:1011C000140001F0FBFC2046FFF7BAFE002383F376
:1011D000118838BD7047000001F0A8B801230370E2
:1011E0000023C0E90133C36183620362C3624362C7
:1011F0000363704738B50446202383F31188002524
:10120000C0E90355C0E90555416001F09FF802238C
:10121000237085F3118838BD70B500EB8103054656
:101220005069DA600E46144618B110220021FFF70B
:101230005DFDA06918B110220021FFF757FD31466E
:101240002846BDE8704001F04BB90000826802F00A
:10125000011282600022C0E90422826101F0CCB94F
:10126000F0B400EB81044789E4680125A4698D404E
:101270003D43458123600023A2606360F0BC01F020
:10128000E7B90000F0B400EB81040789E4680125A8
:1012900064698D403D43058123600023A260636043
:1012A000F0BC01F061BA000070B5022300250446CD
:1012B0000370C0E90255C0E90455C564856180F832
:1012C000345001F0A9F863681B6823B12946204611
:1012D000BDE87040184770BD037880F85030052392
:1012E000037043681B6810B504460BB1042198478E
:1012F0000023A36010BD000090F8502043680270E6
:101300001B680BB1052118477047000070B590F8B5
:101310003430044613B1002380F8343004F1440221
:10132000204601F08BF963689B68B3B994F84430A8
:1013300013F0600535D00021204601F0DDFB0021CF
:10134000204601F0CFFB63681B6813B106212046DD
:101350009847062384F8343070BD2046984700280B
:10136000E4D0B4F84A30E26B9A4288BFE36394F960
:101370004430E56B002B4FF0200380F20381002DF9
:1013800000F0F280092284F8342083F311880021D0
:10139000D4E90E232046FFF775FF002383F311885D
:1013A000DAE794F8452003F07F0343EA022340F292
:1013B0000232934200F0C58021D8B3F5807F48D037
:1013C0000DD8012B3FD0022B00F09380002BB2D11F
:1013D00004F14C02A2630222E2632364C1E7B3F585
:1013E000817F00F09B80B3F5407FA4D194F8463014
:1013F000012BA0D1B4F84C3043F0020332E0B3F536
:10140000006F4DD017D8B3F5A06F31D0A3F5C063EE
:10141000012B90D8636894F846205E6894F84710D2
:10142000B4F848302046B047002884D04368A3630E
:101430000368E3631AE0B3F5106F36D040F602425A
:1014400093427FF478AF5C4BA3630223E3630023F2
:10145000C3E794F84630012B7FF46DAFB4F84C30FD
:1014600023F00203C4E90E55A4F84C30256478E754
:10147000B4F84430B3F5A06F0ED194F8463084F838
:101480004E30204601F020F863681B6813B101213B
:1014900020469847032323700023C4E90E339CE7BA
:1014A00004F14F03A3630123C3E72378042B10D176
:1014B000202383F311882046FFF7C8FE85F31188A7
:1014C0000321636884F84F5021701B680BB12046DC
:1014D000984794F84630002BDED084F84F30042330
:1014E000237063681B68002BD6D0022120469847E2
:1014F000D2E794F848301D0603F00F0120460AD5C4
:1015000001F08EF8012804D002287FF414AF2B4B91
:101510009AE72B4B98E701F075F8F3E794F846301B
:10152000002B7FF408AF94F8483013F00F01B3D0CC
:101530001A06204602D501F0F3FAADE701F0E6FA0B
:10154000AAE794F84630002B7FF4F5AE94F84830C3
:1015500013F00F01A0D01B06204602D501F0CCFAF3
:101560009AE701F0BFFA97E7142284F8342083F356
:1015700011882B462A4629462046FFF771FE85F33F
:101580001188E9E65DB1152284F8342083F31188CF
:101590000021D4E90E232046FFF762FEFDE60B2270
:1015A00084F8342083F311882B462A4629462046A6
:1015B000FFF768FEE3E700BFD8340008D034000826
:1015C000D434000838B590F834300446002B3ED0AF
:1015D000063BDAB20F2A34D80F2B32D8DFE803F0FB
:1015E0003731310822323131313131313131373710
:1015F000C56BB0F84A309D4214D2C3681B8AB5FB54
:10160000F3F203FB12556DB9202383F311882B46A7
:101610002A462946FFF736FE85F311880A2384F807
:1016200034300EE0142384F83430202383F31188FF
:1016300000231A4619462046FFF712FE002383F3C3
:10164000118838BD036C03B198470023E7E70021F8
:10165000204601F051FA0021204601F043FA636868
:101660001B6813B10621204698470623D7E70000E0
:1016700010B590F83430142B044629D017D8062B17
:1016800005D001D81BB110BD093B022BFBD80021AE
:10169000204601F031FA0021204601F023FA636868
:1016A0001B6813B1062120469847062319E0152B25
:1016B000E9D10B2380F83430202383F311880023F1
:1016C0001A461946FFF7DEFD002383F31188DAE797
:1016D000C3689B695B68002BD5D1036C03B1984745
:1016E000002384F83430CEE7024B0022C3E90033F4
:1016F0009A60704794230020002303748268054B8E
:101700001B6899689142FBD25A680360426010607E
:10171000586070479423002008B5202383F3118874
:10172000037C032B05D0042B0DD02BB983F3118838
:1017300008BD436900221A604FF0FF334361FFF791
:10174000DBFF0023F2E7D0E9003213605A60F3E7D1
:10175000002303748268054B1B6899689142FBD88B
:101760005A680360426010605860704794230020FC
:10177000054B19690874186802681A60536018618B
:1017800001230374FEF7C2BD9423002030B54B1C27
:101790000B4D87B0044610D02B690A4A01A800F00F
:1017A00025F92046FFF7E4FF049B13B101A800F0E0
:1017B00059F92B69586907B030BDFFF7D9FFF8E731
:1017C000942300201917000838B50C4D41612B698E
:1017D00081689A689142044603D8BDE83840FFF713
:1017E0008BBF1846FFF7B4FF01232C610146237419
:1017F0002046BDE83840FEF789BD00BF9423002095
:10180000044B1A681B6990689B68984294BF00203B
:10181000012070479423002010B5084C23682069EC
:101820001A6822605460012223611A74FFF790FF46
:1018300001462069BDE81040FEF768BD94230020F2
:1018400008B5FFF7DDFF18B1BDE80840FFF7E4BFBA
:1018500008BD0000FFF7E0BFFEE7000010B50C4C2C
:10186000FFF742FF00F0B4F80A498022204600F05A
:101870003BF8012344F8180C037400F071FC0023BA
:1018800083F3118862B60448BDE8104000F04CB8FC
:10189000BC230020DC340008EC34000800F01CB944
:1018A000EFF3118020B9EFF30583202282F3118832
:1018B0007047000010B530B9EFF30584C4F3080495
:1018C00014B180F3118810BDFFF7BAFF84F31188BB
:1018D000F9E70000034A516853685B1A9842FBD845
:1018E000704700BF001000E0826002220282704751
:1018F0008368A3F17C0243F80C2C026943F83C2C6A
:10190000426943F8382C074A43F81C2CC26843F854
:10191000102C022203F8082C002203F8072CA3F154
:10192000180070472503000810B5202383F31188A1
:10193000FFF7DEFF00210446FFF746FF002383F395
:101940001188204610BD0000024B1B6958610F2012
:10195000FFF70EBF94230020202383F31188FFF7A5
:10196000F3BF000008B50146202383F31188082047
:10197000FFF70CFF002383F3118808BD49B1064B24
:1019800042681B6918605A60136043600420FFF7C7
:10199000FDBE4FF0FF30704794230020036898424B
:1019A00006D01A680260506059611846FFF7A4BE5D
:1019B0007047000038B504460D462068844200D1C7
:1019C00038BD036823605C604561FFF795FEF4E76E
:1019D000054B03F11402C3E905224FF0FF31002249
:1019E000C3E90712704700BF9423002070B51C4E56
:1019F000C0E9032305460C4601F090FA334653F83C
:101A0000142F9A420DD13062C5E901242A600A2CB4
:101A10002CBF00190A30C6E90555BDE8704001F039
:101A20006BBA316A431AE31838BF1C469368A34265
:101A300002D9081901F06EFA73699A6894420CD8B9
:101A40005A68AC602B606A6015609A685D60121B12
:101A50009A604FF0FF33F36170BD1B68A41AECE786
:101A60009423002038B51B4C636998420DD0D0E90F
:101A7000003213605A6000228168C2609A680A448A
:101A80009A604FF0FF33E36138BD2246036842F8A5
:101A9000143F002193425A60C16003D1BDE8384031
:101AA00001F032BA9A688168256A0A449A6001F0A6
:101AB00035FA63699A68411B8A42E5D9AB181D1A49
:101AC000092D206A98BF01F10A02BDE83840104490
:101AD00001F020BA942300202DE9F041184C002792
:101AE00004F11406656901F019FA236AAA68C11A9B
:101AF0008A4215D813442362D5E9003213605A6034
:101B00006369D5F80C80EF60B34201D101F0FCF9B4
:101B100087F311882869C047202383F31188E1E700
:101B20006169B14209D013441B1ABDE8F0410A2B88
:101B30002CBFC0180A3001F0EDB9BDE8F08100BF3C
:101B40009423002000207047FEE70000704700004B
:101B50004FF0FF307047000002290CD0032904D059
:101B60000129074818BF00207047032A05D80548F7
:101B700000EBC2007047044870470020704700BF68
:101B8000D0350008202200208435000870B59AB0B6
:101B90000546084601A9144600F0C2F801A8FFF75F
:101BA0009DF8431C5B00C5E9003400222370032329
:101BB0006370C6B201AB02341046D1B28E4204F15A
:101BC000020401D81AB070BD13F8011B04F8021CFE
:101BD00004F8010C0132F0E708B5202383F31188E3
:101BE0000348FFF779FA002383F3118808BD00BF8B
:101BF0005025002090F8443003F01F02012A07D13D
:101C000090F845200B2A03D10023C0E90E3315E0DC
:101C100003F06003202B08D1B0F848302BB990F8BE
:101C20004520212A03D81F2A04D8FFF737BA222AD1
:101C3000EBD0FAE7034A82630722C2630364012000
:101C4000704700BF1822002007B5052917D8DFE824
:101C500001F0191603191920202383F31188104A63
:101C600001900121FFF7D8FA01980E4A0221FFF7EF
:101C7000D3FA0D48FFF7FCF9002383F3118803B072
:101C80005DF804FB202383F311880748FFF7C6F9AA
:101C9000F2E7202383F311880348FFF7DDF9EBE730
:101CA00024350008483500085025002038B50C4D73
:101CB0000C4C0D492A4604F10800FFF767FF05F1B7
:101CC000CA0204F110000949FFF760FF05F5CA7266
:101CD00004F118000649BDE83840FFF757BF00BFC0
:101CE000182A002020220020043500080E350008A4
:101CF0001935000870B5044608460D46FEF7EEFF9C
:101D0000C6B22046013403780BB9184670BD32467E
:101D10002946FEF7CFFF0028F3D10120F6E70000A7
:101D20002DE9F04705460C46FEF7D8FF2B49C6B211
:101D30002846FFF7DFFF08B10636F6B228492846E5
:101D4000FFF7D8FF08B11036F6B2632E0BD8DFF8D4
:101D50008C80DFF88C90234FDFF894A02E7846B962
:101D60002670BDE8F08729462046BDE8F04701F01F
:101D700065BB252E2ED1072241462846FEF79AFF45
:101D800070B9194B224603F10C0153F8040B42F8C9
:101D9000040B8B42F9D11B78137007350D34DDE746
:101DA000082249462846FEF785FF98B90F4BA21C2A
:101DB000197809090232C95D02F8041C13F8011BE5
:101DC00001F00F015345C95D02F8031CF0D118342E
:101DD0000835C3E704F8016B0135BFE7F0350008AB
:101DE0001935000806360008F8350008107AFF1F7C
:101DF0001C7AFF1FBFF34F8F024AD368DB03FCD46A
:101E0000704700BF003C024008B5094B1B7873B90E
:101E1000FFF7F0FF074B1A69002ABFBF064A5A6056
:101E200002F188325A601A6822F480621A6008BD92
:101E3000762C0020003C02402301674508B50B4B7F
:101E40001B7893B9FFF7D6FF094B1A6942F000429D
:101E50001A611A6842F480521A601A6822F4805299
:101E60001A601A6842F480621A6008BD762C00205D
:101E7000003C02400B28F0B516D80C4C0C492378D6
:101E80007BB90C4D0E460C234FF0006255F8047BD5
:101E900046F8042B013B13F0FF033A44F6D101232B
:101EA000237051F82000F0BD0020FCE7A82C002092
:101EB000782C002018360008014B53F8200070479A
:101EC000183600080C2070470B2810B5044601D9BD
:101ED000002010BDFFF7CEFF064B53F82430184406
:101EE000C21A0BB90120F4E712680132F0D1043BA9
:101EF000F6E700BF183600080B2838B5044628D886
:101F0000FFF7CEFCFFF776FFFFF77EFF124AF323C1
:101F1000D360E300DBB243F4007343F002031361C8
:101F2000136943F48033136105462046FFF762FFCF
:101F3000FFF7A0FF094B53F8241000F0E9F82846FA
:101F4000FFF77CFFFFF7B6FC2046BDE83840FFF7FF
:101F5000BBBF002038BD00BF003C0240183600085F
:101F600012F001032DE9F04105460E4614464BD10F
:101F70008218B2F1016F61D8314B1B6813F0010375
:101F80005CD0304FFFF78CFCFFF73EFFF323FB6084
:101F9000FFF730FF314640F20128032C18D824F017
:101FA0000104284E0C446D1A40F20118A142336915
:101FB00005EB01072AD123F001033361FFF73EFF50
:101FC000FFF778FC0120BDE8F081043C0435E4E72C
:101FD000AB07E4D13B6923F440733B613B6943EABF
:101FE00008033B6151F8046B2E60BFF34F8FFFF77E
:101FF00001FF2B689E42E8D03B6923F001033B615F
:10200000FFF71CFFFFF756FC0020DCE723F44073CA
:102010003361336943EA080333610B883B80BFF3C4
:102020004F8FFFF7E7FE3F8831F8023BBFB2BB425C
:10203000BCD0336923F001033361E1E71846C2E7FE
:1020400000380240003C0240084908B50B7828B12E
:102050001BB9FFF7D9FE01230B7008BD002BFCD084
:10206000BDE808400870FFF7E9BE00BF762C0020ED
:1020700010B50244064BD2B2904200D110BD441CB0
:1020800000B253F8200041F8040BE0B2F4E700BFBF
:10209000502800400F4B30B51C6F240407D41C6F30
:1020A00044F400741C671C6F44F400441C670A4C21
:1020B000236843F4807323600244084BD2B29042F9
:1020C00000D130BD441C00B251F8045B43F82050ED
:1020D000E0B2F4E7003802400070004050280040B1
:1020E00007B5012201A90020FFF7C2FF019803B044
:1020F0005DF804FB13B50446FFF7F2FFA04205D0DC
:10210000012201A900200194FFF7C4FF02B010BD15
:1021100070470000034B1A681AB9034AD2F87428B2
:102120001A607047AC2C00200030024008B5FFF761
:10213000F1FF024B1868C0F3407008BDAC2C0020C2
:10214000EFF3098305494A6B22F001024A636833C1
:1021500083F30988002383F31188704700EF00E0C0
:10216000202080F3118862B60C4B0D4AD96821F407
:10217000E0610904090C0A43DA60D3F8FC2009493C
:1021800042F08072C3F8FC200A6842F001020A6043
:102190001022DA7783F82200704700BF00ED00E0DC
:1021A0000003FA05001000E010B5202383F3118826
:1021B0000E4B5B6813F4006314D0F1EE103AEFF3AA
:1021C0000984683C4FF08073E361094BDB6B236645
:1021D00084F30988FFF714FB10B1064BA36110BD0F
:1021E000054BFBE783F31188F9E700BF00ED00E042
:1021F00000EF00E0370300083A03000870470000D2
:10220000FEE700000A4B0B480B4A90420BD30B4BE6
:10221000DA1C121AC11E22F003028B4238BF0022C0
:102220000021FEF763BD53F8041B40F8041BECE7E4
:10223000B8370008A82D0020A82D0020A82D0020C8
:102240007047000070B5D0E915439E6800224FF03A
:10225000FF3504EB42135101D3F800090028BEBF3B
:10226000D3F8000940F08040C3F80009D3F8000B10
:102270000028BEBFD3F8000B40F08040C3F8000B2D
:10228000013263189642C3F80859C3F8085BE0D2DC
:102290004FF00113C4F81C3870BD00001D4B03EB58
:1022A00080022DE9F043D2F80CC05D6DDCF81420FB
:1022B000461CD2F800E005EB063605EB40185168E5
:1022C00071450AD3D5F83438012202FA00F023EA26
:1022D0000000C5F83408BDE8F083BCF81040AEEB50
:1022E0000103A34228BF2346D8F81849A4B2B3EB90
:1022F000840FF0D89468A4F1040959F8047F37607A
:10230000A4EB09071F44042FF7D81C440B44946026
:102310005360D4E7B02C0020890141F02001016115
:1023200003699B06FCD41220FFF7D4BA10B5054C04
:102330002046FEF753FF4FF0A0436365024BA365B1
:1023400010BD00BFB02C00206C36000870B50378BB
:10235000012B054650D12A4B446D98421BD1294B85
:102360005A6B42F080025A635A6D42F080025A65FD
:102370005A6D5A6942F080025A615A6922F080020D
:102380005A610E2143205B6900F0D4FB1E4BE360D1
:102390001E4BC4F800380023C4F8003EC02323605D
:1023A0006E6D4FF40413A3633369002BFCDA012331
:1023B00033610C20FFF78EFA3369DB07FCD412205F
:1023C000FFF788FA3369002BFCDA0026A66028465E
:1023D000FFF738FF6B68C4F81068DB68C4F814684E
:1023E000C4F81C684BB90A4BA3614FF0FF3363611B
:1023F000A36843F00103A36070BD064BF4E700BF80
:10240000B02C00200038024040140040030020029D
:10241000003C30C0083C30C0F8B5446D0546002192
:102420002046FFF779FFA96D00234FF001128F6856
:10243000C4F834384FF00066C4F81C284FF0FF3061
:1024400004EB431201339F42C2F80069C2F8006BEB
:10245000C2F80809C2F8080BF2D20B686A6DEB6586
:10246000636210231361166916F01006FBD1122067
:10247000FFF730FAD4F8003823F4FE63C4F80038CC
:10248000A36943F4402343F01003A3610923C4F874
:102490001038C4F814380A4BEB604FF0C043C4F84E
:1024A000103B084BC4F8003BC4F81069C4F800396D
:1024B000EB6D03F1100243F48013EA65A362F8BDEB
:1024C0004836000840800010426D90F84E10D2F857
:1024D000003823F4FE6343EA0113C2F80038704762
:1024E0002DE9F84300EB8103456DDA68166806F0C4
:1024F0000306731E022B05EB41130C4680460FFAB0
:1025000081F94FEA41104FF00001C3F8101B4FF062
:10251000010104F1100398BFB60401FA03F39169B5
:102520008EBF334E06F1805606F5004600293AD09C
:10253000578A04F15801490137436F50D5F81C18E8
:102540000B43C5F81C382B180021C3F81019536928
:102550000127611EA7409BB3138A928B9B08012A17
:1025600088BF5343D8F85C20981842EA034301F12E
:10257000400205EB8202C8F85C0021465360284601
:10258000FFF7CAFE08EB8900C3681B8A43EA84533D
:10259000483464011E432E51D5F81C381F43C5F83A
:1025A0001C78BDE8F88305EB4917D7F8001B21F428
:1025B0000041C7F8001BD5F81C1821EA0303C0E747
:1025C00004F13F0305EB83030A4A5A60284621467B
:1025D000FFF7A2FE05EB4910D0F8003923F40043C1
:1025E000C0F80039D5F81C3823EA0707D7E700BF41
:1025F0000080001000040002826D1268C265FFF7BF
:1026000021BE00005831436D49015B5813F400406E
:1026100004D013F4001F0CBF0220012070470000FB
:102620004831436D49015B5813F4004004D013F462
:10263000001F0CBF022001207047000000EB810149
:10264000CB68196A0B6813604B68536070470000D1
:1026500000EB810330B5DD68AA691368D36019B94E
:10266000402B84BF402313606B8A1468426D1C4466
:10267000013CB4FBF3F46343033323F0030302EBA5
:10268000411043EAC44343F0C043C0F8103B2B68F9
:1026900003F00303012B09B20ED1D2F8083802EB84
:1026A000411013F4807FD0F8003B14BF43F08053F7
:1026B00043F00053C0F8003B02EB4112D2F8003B5C
:1026C00043F00443C2F8003B30BD00002DE9F04167
:1026D000244D6E6D06EB40130446D3F8087BC3F817
:1026E000087B38070AD5D6F81438190706D505EB44
:1026F00084032146DB6828465B689847FA071FD5A4
:10270000D6F81438DB071BD505EB8403D968CCB9A0
:102710008B69488A5A68B2FBF0F600FB16228AB928
:102720001868DA6890420DD2121AC3E900242023F7
:1027300083F311880B482146FFF78AFF84F3118841
:10274000BDE8F081012303FA04F26B8923EA020356
:102750006B81CB68002BF3D021460248BDE8F041E5
:10276000184700BFB02C002000EB810370B5DD6876
:10277000436D6C692668E6604A0156BB1A444FF403
:102780000020C2F810092A6802F00302012A0AB2E6
:102790000ED1D3F8080803EB421410F4807FD4F86C
:1027A000000914BF40F0805040F00050C4F8000908
:1027B00003EB4212D2F8000940F00440C2F80009CD
:1027C000D3F83408012202FA01F10143C3F83418A6
:1027D00070BD19B9402E84BF4020206020682E8A29
:1027E0008419013CB4FBF6F440EAC44040F00050C8
:1027F0001A44C6E7F8B504461E48456D05EB441378
:10280000D3F80869C3F80869F10717D5D5F8103867
:10281000DA0713D500EB8403D9684B691F68DA68BF
:10282000974218D2D21B00271A605F60202383F3DF
:1028300011882146FFF798FF87F31188330617D5D3
:10284000D5F834280123A340134211D02046BDE817
:10285000F840FFF723BD012303FA04F2038923EABA
:10286000020303818B68002BE8D021469847E5E7F7
:10287000F8BD00BFB02C00202DE9F74F984C666DD5
:102880007569B3691D4015F48058756107D02046FD
:10289000FEF70AFD03B0BDE8F04FFFF785BC002D41
:1028A00012DAD6F8003E8E489F071EBFD6F8003ECB
:1028B00023F00303C6F8003ED6F8043823F00103E2
:1028C000C6F80438FEF718FD280505D58448FFF73B
:1028D000B9FC8348FEF700FDA9040CD5D6F80838EA
:1028E00013F0060FF36823F470530CBF43F4105336
:1028F00043F4A053F3602A0704D56368DB680BB187
:1029000077489847EB0274D4AF0227D5D4F8549097
:10291000DFF8CCB100274FF0010A09EB4712D2F8DB
:10292000003B03F44023B3F5802F11D1D2F8003BD4
:10293000002B0DDA62890AFA07F322EA03036381A6
:1029400004EB8703DB68DB6813B1394658469847C8
:10295000A36D01379B68FFB29F42DED9E80617D509
:10296000676D3A6AC2F30A1002F00F0302F4F01224
:10297000B2F5802F00F08880B2F5402F08D104EB2B
:1029800083030022DB681B6A07F5805790426DD1F4
:102990002903D6F8184813D5E20302D50020FFF723
:1029A00095FEA30302D50120FFF790FE670302D531
:1029B0000220FFF78BFE260302D50320FFF786FED9
:1029C0006D037FF567AFE00702D50020FFF712FF28
:1029D000A10702D50120FFF70DFF620702D50220F3
:1029E000FFF708FF23077FF555AF0320FFF702FF2E
:1029F00050E7636DDFF8E8B0019300274FF0010A5C
:102A0000A36D9B685FFA87F999453FF67DAF019BFF
:102A100003EB4913D3F8002902F44022B2F5802FCA
:102A200022D1D3F80029002A1EDAD3F8002942F077
:102A30009042C3F80029D3F80029002AFBDB606D1F
:102A40004946FFF769FC22890AFA09F322EA0303DF
:102A5000238104EB8903DB689B6813B14946584620
:102A600098474846FFF71AFC0137C9E7910708BFA6
:102A7000D7F80080072A98BF03F8018B02F1010202
:102A800098BF4FEA182881E7023304EB830207F569
:102A900080575268D2F818C0DCF80820DCE9001C26
:102AA000A1EB0C0C002188420AD104EB830463687B
:102AB0009B699A6802449A605A6802445A6067E7C0
:102AC00011F0030F08BFD7F800808C4588BF02F8CB
:102AD000018B01F1010188BF4FEA1828E3E700BF2D
:102AE000B02C0020436D03EB4111D1F8003B43F4BF
:102AF0000013C1F8003B7047436D03EB4111D1F85F
:102B0000003943F40013C1F800397047436D03EBFB
:102B10004111D1F8003B23F40013C1F8003B70478A
:102B2000436D03EB4111D1F8003923F40013C1F8D0
:102B30000039704700F1604303F561430901C9B2F0
:102B400083F80013012200F01F039A4043099B0001
:102B500003F1604303F56143C3F880211A607047B5
:102B600030B5039C0172043304FB0325C0E906530E
:102B7000049B03630021059BC160C0E90000C0E91C
:102B80000422C0E90842C0E90A11436330BD0000D5
:102B9000416A0022C0E90411C0E90A22C2606FF054
:102BA0000101FEF707BF0000D0E90432934201D1D2
:102BB000C2680AB9181D7047002070470369196080
:102BC000C2680132C260C2691344826903619342E0
:102BD00024BF436A03610021FEF7E0BE38B5044616
:102BE0000D46E3683BB16269131D1268A36213448A
:102BF000E362002007E0237A33B929462046FEF736
:102C0000BDFE0028EDDA38BD6FF00100FBE70000E3
:102C1000C368C269013BC36043691344826943616D
:102C2000934224BF436A436100238362036B03B171
:102C30001847704770B52023044683F31188866ACD
:102C40003EB9FFF7CBFF054618B186F31188284639
:102C500070BDA36AE26A13F8015BA362934202D3D8
:102C60002046FFF7D5FF002383F31188EFE700002C
:102C70002DE9F84F04460E46174698464FF02009B6
:102C800089F311880025AA46D4F828B0BBF1000FBB
:102C900009D141462046FFF7A1FF20B18BF31188EF
:102CA0002846BDE8F88FD4E90A12A7EB050B521AA3
:102CB000934528BF9346BBF1400F1BD9334601F122
:102CC000400251F8040B43F8040B9142F9D1A36A76
:102CD00040334036A3624035D4E90A239A4202D3F6
:102CE0002046FFF795FF8AF31188BD42D8D289F3B9
:102CF0001188C9E730465A46FDF7D2FFA36A5B4404
:102D00005E44A3625D44E7E710B5029C01720433A0
:102D100004FB0321C0E906130023C0E90A33039B27
:102D20000363049BC460C0E90000C0E90422C0E959
:102D30000842436310BD0000026AC260426AC0E9F3
:102D400004220022C0E90A226FF00101FEF732BE20
:102D5000D0E904239A4201D1C26822B9184650F83A
:102D6000043B0B607047002070470000C368C269D5
:102D70000133C3604369134482694361934224BFB2
:102D8000436A43610021FEF709BE000038B50446DE
:102D90000D46E3683BB123691A1DA262E269134440
:102DA000E362002007E0237A33B929462046FEF784
:102DB000E5FD0028EDDA38BD6FF00100FBE700000B
:102DC00003691960C268013AC260C269134482692A
:102DD0000361934224BF436A036100238362036B50
:102DE00003B118477047000070B520230D46044614
:102DF000114683F31188866A2EB9FFF7C7FF10B119
:102E000086F3118870BDA36A1D70A36AE26A01335C
:102E10009342A36204D3E16920460439FFF7D0FF4F
:102E2000002080F31188EDE72DE9F84F04460D46A8
:102E3000904699464FF0200A8AF311880026B3463F
:102E4000A76A4FB949462046FFF7A0FF20B187F394
:102E500011883046BDE8F88FD4E90A073A1AA8EB82
:102E60000607974228BF1746402F1BD905F140039C
:102E700055F8042B40F8042B9D42F9D1A36A403346
:102E8000A3624036D4E90A239A4204D3E16920467A
:102E90000439FFF795FF8BF311884645D9D28AF3A1
:102EA0001188CDE729463A46FDF7FAFEA36A3B446E
:102EB0003D44A3623E44E5E7D0E904239A4217D19A
:102EC000C3689BB1836A8BB1043B9B1A0ED013601D
:102ED000C368013BC360C3691A44836902619A42B3
:102EE00024BF436A036100238362012318467047AD
:102EF0000023FBE700F088B84FF0804300225863BE
:102F00001A610222DA6070474FF080430022DA60D3
:102F1000704700004FF08043586370474FF0804384
:102F2000586A70474B6843608B688360CB68C360A6
:102F30000B6943614B6903628B6943620B680360F1
:102F40007047000008B5264B26481A6940F2FF1169
:102F50000A431A611A6922F4FF7222F001021A610F
:102F60001A691A6B0A431A631A6D0A431A651E4AD4
:102F70001B6D1146FFF7D6FF02F11C0100F58060C2
:102F8000FFF7D0FF02F1380100F58060FFF7CAFFBC
:102F900002F1540100F58060FFF7C4FF02F17001F7
:102FA00000F58060FFF7BEFF02F18C0100F5806044
:102FB000FFF7B8FF02F1A80100F58060FFF7B2FF4C
:102FC00002F1C40100F58060FFF7ACFF02F1E001FF
:102FD00000F58060FFF7A6FFBDE8084000F09AB852
:102FE00000380240000002407836000808B500F0C2
:102FF00007FAFEF733FCFFF78DF8BDE80840FEF74F
:1030000055BE000070470000104B1A6C42F00102E0
:103010001A641A6E42F001021A660D4A1B6E93681A
:1030200043F0010393604FF0804353229A624FF0C4
:10303000FF32DA6200229A615A63DA605A60012232
:103040005A6108211A601C20FFF774BD0038024045
:10305000002004E04FF0804208B51169D3680B40AE
:10306000D9B2C9439B07116107D5202383F3118887
:10307000FEF714FC002383F3118808BD08B5FFF7A1
:10308000E9FFBDE80840FFF78FB800001F4B1A6941
:103090006FEAC2526FEAD2521A611A69C2F3080289
:1030A0001A614FF0FF301A695A69586100215A6954
:1030B00059615A691A6A62F080521A621A6A02F0F9
:1030C00080521A621A6A5A6A58625A6A59625A6A6D
:1030D0001A6C42F080521A641A6E42F080521A66DC
:1030E0001A6E0B4A106840F480701060186F00F47C
:1030F0004070B0F5007F1EBF4FF48030186719672D
:10310000536823F40073536000F05AB9003802404A
:1031100000700040334B4FF080521A64324A4FF433
:10312000404111601A6842F001021A601A68910762
:10313000FCD59A6822F003029A602A4B9A6812F032
:103140000C02FBD1196801F0F90119609A601A6844
:1031500042F480321A601A689203FCD55A6F42F02A
:1031600001025A671F4B5A6F9007FCD51F4A5A60DD
:103170001A6842F080721A601B4A53685904FCD5E1
:10318000184B1A689201FCD5194A9A60194B1A68B3
:10319000194B9A42194B21D1194A1168194A914287
:1031A0001CD140F205121A60144A136803F00F0391
:1031B000052BFAD10B4B9A6842F002029A609A688A
:1031C00002F00C02082AFAD15A6C42F480425A6486
:1031D0005A6E42F480425A665B6E704740F2057246
:1031E000E1E700BF0038024000700040085440078B
:1031F00000948838002004E011640020003C024064
:1032000000ED00E041C20F41084A08B5516913685A
:103210000B4003F00103536123B1054A13680BB15E
:1032200050689847BDE80840FEF7BEBF003C01402B
:10323000282D0020084A08B5516913680B4003F097
:103240000203536123B1054A93680BB1D0689847D4
:10325000BDE80840FEF7A8BF003C0140282D002033
:10326000084A08B5516913680B4003F00403536121
:1032700023B1054A13690BB150699847BDE808406E
:10328000FEF792BF003C0140282D0020084A08B5F7
:10329000516913680B4003F00803536123B1054AD9
:1032A00093690BB1D0699847BDE80840FEF77CBF31
:1032B000003C0140282D0020084A08B551691368D8
:1032C0000B4003F01003536123B1054A136A0BB19D
:1032D000506A9847BDE80840FEF766BF003C0140D1
:1032E000282D0020174B10B55A691C68144004F4AF
:1032F00078725A61A30604D5134A936A0BB1D06A57
:103300009847600604D5104A136B0BB1506B984771
:10331000210604D50C4A936B0BB1D06B9847E2059C
:1033200004D5094A136C0BB1506C9847A30504D51A
:10333000054A936C0BB1D06C9847BDE81040FEF77E
:1033400033BF00BF003C0140282D00201A4B10B5B0
:103350005A691C68144004F47C425A61620504D521
:10336000164A136D0BB1506D9847230504D5134AC7
:10337000936D0BB1D06D9847E00404D50F4A136EDE
:103380000BB1506E9847A10404D50C4A936E0BB153
:10339000D06E9847620404D5084A136F0BB1506F82
:1033A0009847230404D5054A936F0BB1D06F984713
:1033B000BDE81040FEF7F8BE003C0140282D00207B
:1033C000062108B50846FFF7B5FB06210720FFF7E1
:1033D000B1FB06210820FFF7ADFB06210920FFF70E
:1033E000A9FB06210A20FFF7A5FB06211720FFF7FE
:1033F000A1FBBDE8084006212820FFF79BBB000089
:1034000008B5FFF743FE00F00BF8FDF7E5FEFDF70A
:10341000BDFDFFF7F7FDBDE80840FFF76BBD0000FD
:103420000023054A19460133102BC2E9001102F1AD
:103430000802F8D1704700BF282D0020034611F87C
:10344000012B03F8012B002AF9D1704753544D3357
:1034500032463F3F3F00000053544D333246343034
:10346000780053544D3332463432780053544D3340
:103470003246343436585800000000004C340008FE
:103480003F00000013040000583400083F00000013
:1034900019040000623400083F000000210400000D
:1034A0006C3400083F00000000000000090F000815
:1034B000F50E0008310F00081D0F0008290F000845
:1034C000150F0008010F0008ED0E00083D0F000861
:1034D0000000000001000000000000006D61696E46
:1034E0000000000069646C6500000000E43400081E
:1034F000D8230020502500200100000059180008A2
:10350000000000004172647550696C6F74002542C0
:103510004F415244252D424C002553455249414CC0
:103520002500000002000000000000002511000836
:103530009111000840004000E8290020F8290020EF
:103540000200000000000000030000000000000076
:10355000D51100080000000010000000082A00201B
:10356000000000000100000000000000B02C00205E
:1035700001010200491C0008591B0008F51B000846
:10358000D91B0008430000008C35000809024300E5
:10359000020100C0320904000001020201000524FA
:1035A0000010010524010001042402020524060084
:1035B00001070582030800FF09040100020A000058
:1035C00000070501024000000705810240000000DD
:1035D00012000000D835000812011001020000405E
:1035E000091241570002010203010000040309040B
:1035F00025424F41524425007370656564796265C8
:103600006566347633003031323334353637383905
:103610004142434445460000004000000040000095
:103620000040000000400000000001000000020017
:103630000000020000000200000002000000020082
:103640000000020000000200000000000D1300084E
:10365000C51500087116000840004000102D00201C
:10366000102D002001000000202D0020800000000F
:103670004001000003000000000180420000000043
:10368000AAAAAAAA00010040FFFF00000000000053
:1036900000A00A000000000100000000AAAAAAAAD7
:1036A00000000001FFFF000000000000000000001B
:1036B0000000010000000000AAAAAAAA0000000061
:1036C000FFFE0000000000000000000000000000FD
:1036D00000000000AAAAAAAA00000000FFFF000044
:1036E00000000000000000000000000000000000DA
:1036F000AAAAAAAA00000000FFFF00000000000024
:10370000000000000000000000000000AAAAAAAA11
:1037100000000000FFFF00000000000000000000AB
:103720000000000000000000AAAAAAAA00000000F1
:10373000FFFF00000000000000000000000000008B
:10374000000000000A00000000000000030000006C
:103750000000000000000000000000000000000069
:103760000000000000000000000000000000000059
:1037700000000000000000003A040000000000000B
:1037800000400F0000000000FF009600000000084D
:10379000009600000000080004000000EC3500085E
:1037A0000000000000000000000000000000000019
:1037B0000000000000000000FFFFFFFFFFFFFFFF11
:1037C000FFFFFFFFFFFFFFFFFFFFFFFFFFFFFFFF09
:1037D000FFFFFFFFFFFFFFFFFFFFFFFFFFFFFFFFF9
:1037E000FFFFFFFFFFFFFFFFFFFFFFFFFFFFFFFFE9
:1037F000FFFFFFFFFFFFFFFFFFFFFFFFFFFFFFFFD9
:10C000000006002099D2000871250A08CD240A08EC
:10C0100039250A08CD240A0805250A089BD20008FC
:10C020009BD200089BD200089BD2000875640C08C4
:10C030009BD200089BD200089BD200089BD200082C
:10C040009BD200089BD200089BD200089BD200081C
:10C050009BD200089BD200080D700C0835700C08AC
:10C060005D700C0885700C08AD700C080D190C087B
:10C0700035190C0861190C088D190C08B9190C0830
:10C08000E1190C080D1A0C0891180C089BD2000835
:10C090009BD200089BD200089BD20008D5700C08E8
:10C0A0009BD200089BD200089BD200089BD20008BC
:10C0B0009BD2000821720C0835720C089BD2000834
:10C0C0009BD20008991F0C0841210C089BD2000844
:10C0D0009BD20008A9710C08BD710C08D1710C0825
:10C0E00039710C089BD200089BD2000859720C08C9
:10C0F0005D720C0871720C0875720C08391A0C0804
:10C100009BD200089BD2000849720C089BD2000801
:10C11000E5710C08F9710C089BD200089BD200084D
:10C12000651A0C088D1A0C08B91A0C08E51A0C08C7
:10C13000111B0C089BD200089BD200089BD2000860
:10C140009BD200089BD200089BD20008A16B0C0870
:10C15000391B0C08651B0C08911B0C080D720C0890
:10C160009BD200089BD200089BD200089BD20008FB
:10C170009BD200089BD200089BD200089BD20008EB
:10C180009BD200089BD200089BD200089BD20008DB
:10C190009BD200089BD200089BD200089BD20008CB
:10C1A0009BD200089BD200089BD200089BD20008BB
:10C1B0009BD200089BD200089BD200089BD20008AB
:10C1C0009BD200089BD200089BD200089BD200089B
:10C1D0009BD200089BD200089BD200089BD200088B
:10C1E0001126010835FE020889710408D5F80508F2
:10C1F000F9FE0508AD7E060839E10608FDE80608E7
:10C2000035EC0608494C070891710708C108080871
:10C210008D5C0808E569080839170A08F91B0A083F
:10C22000C1FB0A0819680B08318E0B08D9980B0856
:10C23000E9C40B08B1CA0B080000000000000000B0
:10C2400081F0004102E000BF83F0004330B54FEAC7
:10C2500041044FEA430594EA050F08BF90EA020F34
:10C260001FBF54EA000C55EA020C7FEA645C7FEAC7
:10C27000655C00F0E2804FEA5454D4EB5555B8BFEA
:10C280006D420CDD2C4480EA020281EA030382EA5B
:10C29000000083EA010180EA020281EA0303362DED
:10C2A00088BF30BD11F0004F4FEA01314FF4801CC0
:10C2B0004CEA113102D0404261EB410113F0004FD2
:10C2C0004FEA03334CEA133302D0524263EB430389
:10C2D00094EA050F00F0A780A4F10104D5F1200E27
:10C2E0000DDB02FA0EFC22FA05F2801841F1000182
:10C2F00003FA0EF2801843FA05F359410EE0A5F156
:10C3000020050EF1200E012A03FA0EFC28BF4CF086
:10C31000020C43FA05F3C01851EBE37101F000453C
:10C3200007D54FF0000EDCF1000C7EEB00006EEB49
:10C330000101B1F5801F1BD3B1F5001F0CD34908D3
:10C340005FEA30004FEA3C0C04F101044FEA44522A
:10C3500012F5800F80F09A80BCF1004F08BF5FEAB1
:10C36000500C50F1000041EB045141EA050130BD91
:10C370005FEA4C0C404141EB0101013C28BFB1F5A3
:10C38000801FE9D291F0000F04BF01460020B1FAEE
:10C3900081F308BF2033A3F10B03B3F120020CDAC1
:10C3A0000C3208DD02F1140CC2F10C0201FA0CF09F
:10C3B00021FA02F10CE002F11402D8BFC2F1200C04
:10C3C00001FA02F120FA0CFCDCBF41EA0C019040BA
:10C3D000E41AA2BF01EB0451294330BD6FEA040403
:10C3E0001F3C1CDA0C340EDC04F11404C4F12002EE
:10C3F00020FA04F001FA02F340EA030021FA04F300
:10C4000045EA030130BDC4F10C04C4F1200220FA56
:10C4100002F001FA04F340EA0300294630BD21FA94
:10C4200004F0294630BD94F0000F83F4801306BF5A
:10C4300081F480110134013D4EE77FEA645C18BF4E
:10C440007FEA655C29D094EA050F08BF90EA020FE5
:10C4500005D054EA000C04BF1946104630BD91EADD
:10C46000030F1EBF0021002030BD5FEA545C05D1E0
:10C470004000494128BF41F0004130BD14F580041F
:10C480003CBF01F5801130BD01F0004545F0FE4193
:10C4900041F470014FF0000030BD7FEA645C1ABFC8
:10C4A000194610467FEA655C1CBF0B46024650EAFF
:10C4B000013406BF52EA033591EA030F41F400212B
:10C4C00030BD00BF90F0000F04BF0021704730B5B1
:10C4D0004FF4806404F132044FF000054FF0000186
:10C4E00050E700BF90F0000F04BF0021704730B547
:10C4F0004FF4806404F1320410F0004548BF40421C
:10C500004FF000013EE700BF42004FEAE2014FEA70
:10C5100031014FEA02701FBF12F07F4393F07F4F4B
:10C5200081F06051704732F07F4208BF704793F04E
:10C530007F4F04BF41F40021704730B54FF4607461
:10C5400001F0004521F000411CE700BF50EA010264
:10C5500008BF704730B54FF000050AE050EA01020D
:10C5600008BF704730B511F0004502D5404261EB7D
:10C5700041014FF4806404F132045FEA915C3FF4BE
:10C58000D8AE4FF003025FEADC0C18BF03325FEA5B
:10C59000DC0C18BF033202EBDC02C2F1200300FA0C
:10C5A00003FC20FA02F001FA03FE40EA0E0021FA31
:10C5B00002F11444BDE600BF70B54FF0FF0C4CF41F
:10C5C000E06C1CEA11541DBF1CEA135594EA0C0FD1
:10C5D00095EA0C0F00F0DEF82C4481EA030621EA0C
:10C5E0004C5123EA4C5350EA013518BF52EA033547
:10C5F00041F4801143F4801338D0A0FB02CE4FF0F9
:10C600000005E1FB02E506F00042E0FB03E54FF028
:10C610000006E1FB03569CF0000F18BF4EF0010E20
:10C62000A4F1FF04B6F5007F64F5407404D25FEA1C
:10C630004E0E6D4146EB060642EAC62141EA5551CF
:10C640004FEAC52040EA5E504FEACE2EB4F1FD0C11
:10C6500088BFBCF5E06F1ED8BEF1004F08BF5FEA8F
:10C66000500E50F1000041EB045170BD06F0004641
:10C6700046EA010140EA020081EA0301B4EB5C04EE
:10C68000C2BFD4EB0C0541EA045170BD41F48011E6
:10C690004FF0000E013C00F3AB8014F1360FDEBF0B
:10C6A000002001F0004170BDC4F10004203C35DAE7
:10C6B0000C341BDC04F11404C4F1200500FA05F36A
:10C6C00020FA04F001FA05F240EA020001F000420B
:10C6D00021F0004110EBD37021FA04F642EB060181
:10C6E0005EEA430E08BF20EAD37070BDC4F10C04AB
:10C6F000C4F1200500FA04F320FA05F001FA04F26F
:10C7000040EA020001F0004110EBD37041F100015A
:10C710005EEA430E08BF20EAD37070BDC4F1200565
:10C7200000FA05F24EEA020E20FA04F301FA05F2CD
:10C7300043EA020321FA04F001F0004121FA04F275
:10C7400020EA020000EBD3705EEA430E08BF20EA45
:10C75000D37070BD94F0000F0FD101F0004640007F
:10C7600041EB010111F4801F08BF013CF7D041EA01
:10C77000060195F0000F18BF704703F00046520005
:10C7800043EB030313F4801F08BF013DF7D043EAD6
:10C790000603704794EA0C0F0CEA135518BF95EA8C
:10C7A0000C0F0CD050EA410618BF52EA4306D1D113
:10C7B00081EA030101F000414FF0000070BD50EA32
:10C7C000410606BF1046194652EA430619D094EABC
:10C7D0000C0F02D150EA013613D195EA0C0F05D1A6
:10C7E00052EA03361CBF104619460AD181EA0301FA
:10C7F00001F0004141F0FE4141F470014FF00000B2
:10C8000070BD41F0FE4141F4780170BD70B54FF04C
:10C81000FF0C4CF4E06C1CEA11541DBF1CEA1355CC
:10C8200094EA0C0F95EA0C0F00F0A7F8A4EB0504AE
:10C8300081EA030E52EA03354FEA013100F08880A5
:10C840004FEA03334FF0805545EA131343EA12636E
:10C850004FEA022245EA111545EA10654FEA002623
:10C860000EF000419D4208BF964244F1FD0404F5DC
:10C87000407402D25B084FEA3202B61A65EB030538
:10C880005B084FEA32024FF480104FF4002CB6EBF5
:10C89000020E75EB030E22BFB61A754640EA0C0075
:10C8A0005B084FEA3202B6EB020E75EB030E22BFB5
:10C8B000B61A754640EA5C005B084FEA3202B6EBF6
:10C8C000020E75EB030E22BFB61A754640EA9C00B5
:10C8D0005B084FEA3202B6EB020E75EB030E22BF85
:10C8E000B61A754640EADC0055EA060E18D04FEA43
:10C8F000051545EA16754FEA06164FEAC30343EAE3
:10C9000052734FEAC2025FEA1C1CC0D111F4801FAF
:10C910000BD141EA00014FF000004FF0004CB6E7A8
:10C9200011F4801F04BF01430020B4F1FD0C88BF47
:10C93000BCF5E06F3FF6AFAEB5EB030C04BFB6EB52
:10C94000020C5FEA500C50F1000041EB045170BD45
:10C950000EF0004E4EEA113114EB5C04C2BFD4EB72
:10C960000C0541EA045170BD41F480114FF0000EF6
:10C97000013C90E645EA060E8DE60CEA135594EA72
:10C980000C0F08BF95EA0C0F3FF43BAF94EA0C0F75
:10C990000AD150EA01347FF434AF95EA0C0F7FF4EA
:10C9A00025AF104619462CE795EA0C0F06D152EA3E
:10C9B00003353FF4FDAE1046194622E750EA410622
:10C9C00018BF52EA43067FF4C5AE50EA41047FF433
:10C9D0000DAF52EA43057FF4EBAE12E74FF0FF3C98
:10C9E00006E000BF4FF0010C02E000BF4FF0010C69
:10C9F0004DF804CD4FEA410C7FEA6C5C4FEA430CE2
:10CA000018BF7FEA6C5C1BD001B050EA410C0CBF30
:10CA100052EA430C91EA030F02BF90EA020F002092
:10CA2000704710F1000F91EA030F58BF994208BFF9
:10CA300090422CBFD8176FEAE37040F001007047B6
:10CA40004FEA410C7FEA6C5C02D150EA013C07D10D
:10CA50004FEA430C7FEA6C5CD6D152EA033CD3D058
:10CA60005DF8040B704700BF8446104662468C4652
:10CA70001946634600E000BF01B5FFF7B7FF002885
:10CA800048BF10F1000F01BD4DF808EDFFF7F4FFAE
:10CA90000CBF012000205DF808FB00BF4DF808ED39
:10CAA000FFF7EAFF34BF012000205DF808FB00BF5C
:10CAB0004DF808EDFFF7E0FF94BF012000205DF87E
:10CAC00008FB00BF4DF808EDFFF7CEFF94BF012033
:10CAD00000205DF808FB00BF4DF808EDFFF7C4FF2C
:10CAE00034BF012000205DF808FB00BF4FEA410C75
:10CAF0007FEA6C5C02D150EA013C0AD14FEA430C58
:10CB00007FEA6C5C02D152EA033C02D14FF0000094
:10CB100070474FF0010070474FEA410212F50012D2
:10CB200015D211D56FF47873B3EB625212D94FEA74
:10CB3000C12343F0004343EA505311F0004F23FA5E
:10CB400002F018BF404270474FF00000704750EAB3
:10CB5000013005D111F0004008BF6FF00040704770
:10CB60004FF00000704700BF4A0011D212F50012CA
:10CB700011D20DD56FF47873B3EB62520ED44FEA35
:10CB8000C12343F0004343EA505323FA02F07047B5
:10CB90004FF00000704750EA013002D14FF0FF30F3
:10CBA00070474FF0000070474FEA4102B2F1E04396
:10CBB00024BFB3F5001CDCF1FE5C0DD901F0004C84
:10CBC0004FEAC0024CEA5070B2F1004F40EB8300D4
:10CBD00008BF20F00100704711F0804F21D113F100
:10CBE0003872BCBF01F00040704741F480114FEA39
:10CBF0005252C2F11802C2F1200C10FA0CF320FAC2
:10CC000002F018BF40F001004FEAC1234FEAD323DE
:10CC100003FA0CFC40EA0C0023FA02F34FEA430348
:10CC2000CCE77FEA625307D150EA01331EBF4FF0D1
:10CC3000FE4040F44000704701F0004040F0FE40EC
:10CC400040F40000704700BF80F0004002E000BFE9
:10CC500081F0004142001FBF5FEA410392EA030FE7
:10CC60007FEA226C7FEA236C6AD04FEA1262D2EB31
:10CC70001363C1BFD218414048404140B8BF5B4236
:10CC8000192B88BF704710F0004F40F4000020F0CF
:10CC90007F4018BF404211F0004F41F4000121F0E5
:10CCA0007F4118BF494292EA030F3FD0A2F101022F
:10CCB00041FA03FC10EB0C00C3F1200301FA03F16D
:10CCC00000F0004302D5494260EB4000B0F5000F90
:10CCD00013D3B0F1807F06D340084FEA310102F14F
:10CCE0000102FE2A51D2B1F1004F40EBC25008BF01
:10CCF00020F0010040EA03007047490040EB0000CB
:10CD0000013A28BFB0F5000FEDD2B0FA80FCACF1CB
:10CD1000080CB2EB0C0200FA0CF0AABF00EBC250F8
:10CD200052421843BCBFD0401843704792F0000FE6
:10CD300081F4000106BF80F400000132013BB5E739
:10CD40004FEA41037FEA226C18BF7FEA236C21D0AF
:10CD500092EA030F04D092F0000F08BF0846704714
:10CD600090EA010F1CBF0020704712F07F4F04D1E2
:10CD7000400028BF40F00040704712F100723CBFF5
:10CD800000F50000704700F0004343F0FE4040F41F
:10CD9000000070477FEA226216BF08467FEA2363DD
:10CDA0000146420206BF5FEA412390EA010F40F4C8
:10CDB000800070474FF0000304E000BF10F0004314
:10CDC00048BF40425FEA000C08BF704743F09643FB
:10CDD00001464FF000001CE050EA010208BF704716
:10CDE0004FF000030AE000BF50EA010208BF70479D
:10CDF00011F0004302D5404261EB41015FEA010CB2
:10CE000002BF84460146002043F0B64308BFA3F1A9
:10CE10008053A3F50003BCFA8CF2083AA3EBC2538B
:10CE200010DB01FA02FC634400FA02FCC2F12002AA
:10CE3000BCF1004F20FA02F243EB020008BF20F0E1
:10CE40000100704702F1200201FA02FCC2F1200247
:10CE500050EA4C0021FA02F243EB020008BF20EA3C
:10CE6000DC7070477BB972B90029BEBF00204FF05B
:10CE7000004106E008BF00281CBF6FF000414FF0E2
:10CE8000FF3000F007BAADF1080C6DE904CE0029BF
:10CE900009DB002B1ADB00F095F8DDF804E0DDE992
:10CEA000022304B07047404261EB4101002B1BDBC1
:10CEB00000F088F8DDF804E0DDE9022304B0404228
:10CEC00061EB4101524263EB43037047524263EB13
:10CED000430300F077F8DDF804E0DDE9022304B055
:10CEE000404261EB41017047524263EB430300F063
:10CEF00069F8DDF804E0DDE9022304B0524263EB97
:10CF00004303704753B94AB9002908BF00281CBF22
:10CF10004FF0FF314FF0FF3000F0BCB9ADF1080C1D
:10CF20006DE904CE00F04EF8DDF804E0DDE90223FF
:10CF300004B07047430803F05533C01A830803F068
:10CF4000333300F03330184400EB101000F00F3092
:10CF500000EB002000EB0040000E704707EE900A47
:10CF6000F5EEC07AF1EE10FA01D400F00BB8F1EE54
:10CF7000677A08B517EE900A00F004F8404261EBBA
:10CF8000410108BDD0B5FFF7BFFA0C4B00220646A1
:10CF90000F46FFF711FBFFF7E7FD0446FFF792FA94
:10CFA000074B0022FFF708FB02460B463046394686
:10CFB000FFF74AF9FFF7D8FD2146D0BD0000F03D4C
:10CFC0000000F0412DE9F047089D04468E46002BF5
:10CFD0004DD18A42944669D9B2FA82F252B101FA2D
:10CFE00002F3C2F1200120FA01F10CFA02FC41EA3D
:10CFF000030E94404FEA1C48210CBEFBF8F61FFAC2
:10D000008CF708FB16E341EA034306FB07F199425C
:10D010000AD91CEB030306F1FF3080F01F8199420F
:10D0200040F21C81023E63445B1AA4B2B3FBF8F0E9
:10D0300008FB103344EA034400FB07F7A7420AD970
:10D040001CEB040400F1FF3380F00A81A74240F298
:10D0500007816444023840EA0640E41B00261DB103
:10D06000D4400023C5E900433146BDE8F0878B4238
:10D0700009D9002D00F0EF800026C5E900013046F7
:10D080003146BDE8F087B3FA83F6002E4AD18B42D1
:10D0900002D3824200F2F980841A61EB030301207B
:10D0A0009E46002DE0D0C5E9004EDDE702B9FFDE67
:10D0B000B2FA82F2002A40F09280A1EB0C014FEA12
:10D0C0001C471FFA8CFE0126200CB1FBF7F307FB6F
:10D0D000131140EA01410EFB03F0884208D91CEB12
:10D0E000010103F1FF3802D2884200F2CB804346AF
:10D0F000091AA4B2B1FBF7F007FB101144EA01448E
:10D100000EFB00FEA64508D91CEB040400F1FF311C
:10D1100002D2A64500F2BB800846A4EB0E0440EA0A
:10D1200003409CE7C6F12007B34022FA07FC4CEA13
:10D13000030C20FA07F401FA06F31C43F9404FEA06
:10D140001C4900FA06F3B1FBF9F8200C1FFA8CFE1B
:10D1500009FB181140EA014108FB0EF0884202FA6F
:10D1600006F20BD91CEB010108F1FF3A80F0888030
:10D17000884240F28580A8F102086144091AA4B2ED
:10D18000B1FBF9F009FB101144EA014100FB0EFE6E
:10D190008E4508D91CEB010100F1FF346CD28E459D
:10D1A0006AD90238614440EA0840A0FB0294A1EB2E
:10D1B0000E01A142C846A64656D353D05DB1B3EB8B
:10D1C000080261EB0E0101FA07F722FA06F3F140BB
:10D1D0001F43C5E9007100263146BDE8F087C2F162
:10D1E0002003D8400CFA02FC21FA03F391400143DA
:10D1F0004FEA1C471FFA8CFEB3FBF7F007FB103613
:10D200000B0C43EA064300FB0EF69E4204FA02F4BE
:10D2100008D91CEB030300F1FF382FD29E422DD911
:10D22000023863449B1B89B2B3FBF7F607FB163346
:10D2300041EA034106FB0EF38B4208D91CEB0101C6
:10D2400006F1FF3816D28B4214D9023E6144C91A46
:10D2500046EA004638E72E46284605E70646E3E656
:10D260001846F8E64B45A9D2B9EB020864EB0C0E60
:10D270000138A3E74646EAE7204694E74046D1E76F
:10D28000D0467BE7023B614432E7304609E764441D
:10D29000023842E7704700BF02E000F000F8FEE706
:10D2A00072B6374880F30888364880F309883648D4
:10D2B0003649086040F20000CCF200004EF63471AE
:10D2C000CEF200010860BFF34F8FBFF36F8F40F2C3
:10D2D0000000C0F2F0004EF68851CEF20001086066
:10D2E000BFF34F8FBFF36F8F4FF00000E1EE100AD6
:10D2F0004EF63C71CEF200010860062080F31488DF
:10D30000BFF36F8FB9F014F9B8F0ECF94FF0553066
:10D310001F491B4A91423CBF41F8040BFAE71D49E3
:10D32000184A91423CBF41F8040BFAE71A491B4ADC
:10D330001B4B9A423EBF51F8040B42F8040BF8E72E
:10D3400000201849184A91423CBF41F8040BFAE703
:10D35000B9F0F2F8B8F01AFA144C154DAC4203DAF1
:10D3600054F8041B8847F9E701F098FB114C124D63
:10D37000AC4203DA54F8041B8847F9E7B9F0DAB88D
:10D38000000600200022002000C0000808ED00E098
:10D39000000000200006002050180F080022002086
:10D3A0007C2B0020802B0020205B0120E0C10008A6
:10D3B00038C2000838C2000838C200082DE9F04F12
:10D3C0002DED108AC1F80CD0C3689D46BDEC108AC3
:10D3D000BDE8F08F002383F311882846A047002082
:10D3E000B7F006FFFEE7B7F073FD00DFFEE70000D1
:10D3F00001F0FF01102A2BDB10F0070F08D010F806
:10D40000013B013A8B422DD010F0070F42B3F6D109
:10D41000F0B441EA012141EA014122F007047FF022
:10D4200000070023F0E80256083C85EA010586EA79
:10D43000010685FA47F5A3FA87F586FA47F6A5FAB5
:10D4400087F68EB9EED1F0BC01F0FF0102F00702C1
:10D4500032B110F8013B013A83EA010313B1F8D16C
:10D460000020704701387047002D06BF354603384D
:10D47000073815F0010F07D1013015F4807F02BF86
:10D48000013015F4C03F0130F0BC0138704700BFD7
:10D4900010F8012B11F8013B012A28BF9A42F7D05E
:10D4A000D01A7047034613F8012B002AFBD1181A33
:10D4B0000138704738B50022002304460D46FFF7B7
:10D4C000EDFA28B920462946BDE8384000F00AB8F0
:10D4D000204605F1004100F005F8404261EB4101B2
:10D4E00038BD00BFD0B50C4B002206460F46FFF7F3
:10D4F00063F8FFF739FB0446FEF7E4FF074B002211
:10D50000FFF75AF802460B4630463946FEF79CFEB6
:10D51000FFF72AFB2146D0BD0000F03D0000F0419E
:10D52000036800221B68184710B503685B6804464F
:10D53000984708B194F84D0010BD00002DE9F04166
:10D54000664B03F5C04490B094F9A42106460F46FB
:10D55000002A00F0C08094F8EC5135B9604A83F09D
:10D5600093F9284610B0BDE8F081B3F9A4201AB9A8
:10D57000B3F8A220A3F8A420B3F8A430632B05D8F5
:10D58000584A3946304683F07FF9002500212E2283
:10D5900004A80391BCF0EEFED4F80401036803AACA
:10D5A0001B6832219847804630B94F4A03AB394651
:10D5B000304683F069F94546B4F8E030A3F57A7354
:10D5C0009BB241F65832934206D9484B3A46202145
:10D5D000304682F051FF002594F91433002B69DDA9
:10D5E00094F9CC32002B59DD414B3A46202130468C
:10D5F00082F042FF00253F49D4F81001322303AAEC
:10D600008EF04CF9804640B903AB00933A463A4B52
:10D610002021304682F030FF45463849D4F80C01CD
:10D62000322303AA8BF06CF9804640B903AB009318
:10D630003A46314B2021304682F01EFF45462021DC
:10D64000304682F011FFB8B1D4ED587A9FED2C7AB4
:10D65000F0EEE77AF4EEC77AF1EE10FA0CD594F911
:10D660001433002B02DD94F878332BB9254A394660
:10D67000304683F009F9002594F91433002B7FF725
:10D6800070AF94F9D131002B3FF46BAF1E4B3A468B
:10D690002021304682F0F0FE002562E794F878837E
:10D6A000B8F1000F06D1194B3A462021304682F0DE
:10D6B000E3FE454694F9CC32002B9CDD94F8FD82C4
:10D6C000B8F1000F97D1124B3A462021304682F034
:10D6D000D3FE45468FE7012543E700BF902B00208E
:10D6E00034E80C0856E80C087DE80C0888E80C08BB
:10D6F0009AE80C080BE90C080FE90C0821E90C0862
:10D700000000003425E90C083FE90C08C0E80C08CB
:10D71000E6E80C0838B5044682F08AFE114B93F80F
:10D72000B012114B1D68EB6A1A68002908BF014648
:10D730001268184690475CF037FBEB6A93F89C1030
:10D740005BF01EFB94F837305BB194F047FFEB6A57
:10D75000D3F8A030C01AB0F5FA6F24BF002384F8C4
:10D76000373038BD908B00208C2B002008B5FFF798
:10D77000D1FF054B05481B68DB6A93F89C10BDE898
:10D78000084011F013BB00BF8C2B0020688C0020D8
:10D7900070B50E46054667F077FC67F039FC10B9A6
:10D7A0000124204670BD0A4B93F90A32012BF7D1B0
:10D7B00067F06AFC437A002BF2D167F065FC847A4B
:10D7C000002CEDD1034A3146284683F05DF8E8E7A6
:10D7D000904B002058E90C08034BD3F874320BB976
:10D7E00082F0DCBD01207047904B00202DE9F0470E
:10D7F0002DED028BC47F90B006460F468CB990F990
:10D800000430002B00F00581834B1D68A86A036873
:10D810005B6B9847044650B9804A3946304683F0DE
:10D8200033F8204610B0BDEC028BBDE8F087B3683A
:10D830004BB933685B6B3946304610B0BDEC028B98
:10D84000BDE8F0471847E86AFFF76EFE0446002877
:10D85000E7D13946304683F0B5FEDFF8F48105465E
:10D860003946304683F038F898ED877AD8ED867AD5
:10D87000B4EEE77A2840F1EE10FAC5B209D598F96E
:10D880001432032B05D0664A3946304682F0FCFF3D
:10D890002546D8ED6F7AB0EE088AF4EEC87AF1EE3C
:10D8A00010FA0BD517EE900AFEF72EFE5D4ACDE971
:10D8B00000013946304682F0E7FF0025D8ED707A46
:10D8C000F4EEC87AF1EE10FA0BD517EE900AFEF7D7
:10D8D0001BFE554ACDE900013946304682F0D4FF9F
:10D8E0000025D8ED717AB8EE087AF4EEC77AF1EE39
:10D8F00010FA0BDD17EE900AFEF706FE4B4ACDE953
:10D9000000013946304682F0BFFF0025B8F9A83142
:10D91000042B07DC052200923946454A304682F046
:10D92000B3FF0025D8F8300C67F00AFC80B198F9F5
:10D930000A326BB1D8F8303CB8F90C22B3F90E308A
:10D940009A4205DA3B4A3946304682F09DFF00256F
:10D9500039463046FFF71CFFDFF8F8A0814639460C
:10D960003046FFF7EBFD9AF8353F002B4AD109EA24
:10D97000050500EA050430484FF4806101F070F8B5
:10D9800078B1D8F8303CB3F90C30A3F2E24292B24D
:10D99000B2F5FA7F05D9294A3946304682F074FF3C
:10D9A0000024274890F888355BB100F5B06038F066
:10D9B0006BFC054628B9234A3946304682F064FF9D
:10D9C0002C4600212E2204A80DF10C080391BCF076
:10D9D000D1FCDAF8200F4246322109F053FE054609
:10D9E00000287FF41EAFDAF8200F03689B68984781
:10D9F000154ACDF8008003463946304682F044FF90
:10DA00002C460EE7114A3946304682F03DFF00248D
:10DA1000B1E7012405E700BF8C2B002068E90C0862
:10DA20007FE90C08A2E90C08C2E90C08E4E90C083B
:10DA300006EA0C0825EA0C08902B002060EA0C0886
:10DA4000907B002088EA0C08D0B80D084BEA0C083F
:10DA5000904B0020906B002070B505460E46FFF7F6
:10DA600097FE31460446284683F058FC2040C0B259
:10DA700070BD0000F0B591B005460E4682F0CCFFB7
:10DA80000446D8B11021284682F0EEFCB0B1002146
:10DA90002E2204A803AF0391BCF06CFC1CF0CAF862
:10DAA00032233A4601211BF085FB044630B9054B71
:10DAB000009732461021284682F0DEFC204611B045
:10DAC000F0BD00BF9CEA0C0870B505460E46B1B922
:10DAD00090F910408CB1164814F096F8DFED157AE5
:10DAE000B0EEC00AB4EEE70AF1EE10FA07D4124A1B
:10DAF0000121284682F0C8FE3446204670BDAB683E
:10DB00009BB10E4B1B68D86AFFF70EFD044630B17F
:10DB100066F018F80A4A04215FF0B4F9EDE73146DF
:10DB20002846BDE8704083F043BA0124E5E700BF12
:10DB3000902B002000000034A8EA0C088C2B002059
:10DB4000BAEA0C0838B5044683F0F6FD0546A8B1DC
:10DB50000B4806F061FC38B10A490B481BF082FC07
:10DB600010B1074800F050FF2046FFF7FFFD0123EA
:10DB7000064984F83730204683F0F4FC284638BD47
:10DB8000902B0020948B0020503E0020DCEA0C08F3
:10DB9000F8B505460E461746C2B1232901D0012922
:10DBA00014D8254809F02EF8044668B10024204610
:10DBB000F8BD95F91030022B08D065F0C3FF1F4A5D
:10DBC00006215FF05FF9F2E7002EF2D03A463146C7
:10DBD000284683F067FE04460028E7D0184ED6F8A2
:10DBE000202F06F548639A4203D006F5AC5038F072
:10DBF00081FFD6F8200F134F03689B6B984787F877
:10DC0000580507F58057D7F82831012B07D167F061
:10DC10003BFA542168F0FCF908B9C7F828012846F6
:10DC2000FFF7A4FD4FF0FF330749C6F8583F2846D9
:10DC300083F098FCBBE700BF902B0020ECEA0C08B7
:10DC4000906B0020907B002004EB0C082DE9F04F36
:10DC50002DED028BDFF8489191B00746884682F09F
:10DC6000AFFC99F9DF510446D5B9BD2109F55650ED
:10DC700038F0D6FE38B1434B42464FF48041384627
:10DC800082F0FAFB2C464048BC2138F0C9FE38B17E
:10DC90003E4B42464FF48041384682F0EDFB002473
:10DCA0003B4E96F8EC31002B66D0A6F580531C2233
:10DCB000002102A8B3F8B4A5DFED368ABCF05AFB08
:10DCC00004A821F08BFCA6F5286B0125A6F5C0461B
:10DCD000554551D20BA821F081FC09AA2946584686
:10DCE00036F03EFB002847D0BDF82610304608F03D
:10DCF000A1F880B3BDF80A30102B2CD104A90BA8D1
:10DD000021F0CEFF09F64853B0EE408A93ED000AA9
:10DD10002148B4EEE80AF1EE10FAB8BF99ED6B0AAB
:10DD200020EE000A0FF058F9F6EE087A60EE277A36
:10DD3000B4EEE78AF1EE10FA0DD517EE900AFEF771
:10DD4000E3FB164BCDE9000142464FF480413846D3
:10DD500082F092FB00240DF1240CBCE80F000DF1C1
:10DD6000080EAEE80F009CE80700AEE8030001359E
:10DD70008EF80020ADB2ABE7204611B0BDEC028BAF
:10DD8000BDE8F08F18EB0C081081002044EB0C0864
:10DD9000908B002000000034688C002077EB0C088A
:10DDA000904B002000207047014800F0ADBD00BF3F
:10DDB000902B002003685B68184700006AF0A6BB40
:10DDC00067F0B0B830F090BA5BF05CB909F06CB8AD
:10DDD00059F048BA0DF028BD15F088B903F04CBBD6
:10DDE00057F0DCBD1FF010BE69F036BF15F0E4B986
:10DDF00013F088BF1FF06CB96CF03CB966F0ACBD95
:10DE000064F070BF08F0F8B905F082BA0CF0D8BF22
:10DE10000DF068BC14F0A4BF15F07CBA13F0A6BDD9
:10DE200015F0DEB801F0BABB00F2545022F0A0BCED
:10DE300008F078BD90F8C432B02202FB030390F8DA
:10DE4000082393F8A13012B1012B28BF01231846F3
:10DE50007047000090F814310BB190F8413118462A
:10DE600070470000034808602A21117008221A60D8
:10DE7000704700BFA8EE0C08F8B5044600F5C14095
:10DE8000103004F59656FFF745FC002130461BF094
:10DE900043FE8021204615F0ADFC18B131F018FE8C
:10DEA0002FF0F8FE04F50055D5ED6F7A9FED317A2D
:10DEB00067EE877A05F64447FDEEE77A04F5C6403B
:10DEC00017EE903AC5F8403CD5F8C4313B601030AD
:10DED00015F092FEF8B9D5F8403C07EE903A04F5FB
:10DEE000805303F20C5292ED007AF8EEE77A03F5D4
:10DEF000A16367EE877AFDEEE77A17EE902AC5F800
:10DF0000402CD3ED007A97ED007AF0EEE77A67EED9
:10DF1000877AC7ED007A04F5AF51183106F54570E0
:10DF200035F09CFC04F5A94594ED467AD5ED167ABA
:10DF3000E7EE007AC5ED167AB0EE670A32F0F0FA35
:10DF400004F5C14085ED160A58300EF055F904F578
:10DF5000C1400021643087F0E5FB4FF400112046FA
:10DF600015F048FC20B13046BDE8F84019F0FEBE7F
:10DF7000F8BD00BF0000C842FFF77EBF70B500F5D6
:10DF800080430546D3F8200F03689B6B984705F53F
:10DF9000C14458340646204610F0CAFE05F5A04399
:10DFA000002893F8173518BF00262BB926B105F5C0
:10DFB0003350183087F01AFB204610F04FFB18B989
:10DFC0002046FFF747FF20B12046BDE8704011F022
:10DFD000FDB870BDFFF7D2BF38B54FF480110546CC
:10DFE00015F008FC044620B90121284615F002FC72
:10DFF00004460221284615F0FDFB48B114B9284615
:10E0000003F060F905F59650BDE8384019F0ACBD55
:10E01000002CF7D138BD0000FFF7DEBF38B54FF454
:10E020008011044615F0E6FB01210546204615F057
:10E03000E1FB18B115B9204603F044F91021204640
:10E0400015F0D8FB60B1204603F02EFA4FF48001A2
:10E05000204615F0CFFB18B931F03AFD2FF00CFF38
:10E060002021204615F0C6FB28B1204603F092FA85
:10E07000204603F0A9FB4FF40051204615F0BAFBEF
:10E0800010B1204603F088FB8021204615F0B2FB3A
:10E0900028B131F01DFDBDE838402FF01FBE38BD5E
:10E0A000FFF7BCBF10B5044622F052FC90F92130B6
:10E0B0008BB190F8403373B194F978355BB1064B6E
:10E0C0001B68DB6A93F89C302BB904F25450BDE80E
:10E0D000104022F065B910BD8C2B0020FFF7E2BF85
:10E0E0002DE9F843434B1B68DB6A93F89C300446E8
:10E0F000002B7CD000F5805797F8C935002B76D0DF
:10E1000008F080FD002872D004F5F75507F5805916
:10E11000083599F83610284619F0CAF8002866D054
:10E1200004F590763046FFF785FE02285FD994F813
:10E13000E4334FF0B00808FB034393ED777AF1EE38
:10E14000007AB4EEE77AF1EE10FA50D499F836106E
:10E15000284619F05DFB04F50053B3F9A82107EE3A
:10E16000902AB8EEE77AB4EEC07AF1EE10FA0CDD40
:10E1700094F8E42308FB0242F8EE677A92ED777A8E
:10E18000F4EEC77AF1EE10FA31DCD7F8B824D3F800
:10E19000401C002AB8BF52428A4228DC07F2BC4227
:10E1A000D2ED007AD3ED706A9FED136AF8EEE77A4C
:10E1B00066EE866AF4EEE67AF1EE10FA17DC03F604
:10E1C000444292ED007A27EE067AF4EEC77AF1EE39
:10E1D00010FA0CD494F8E413B02202FB0161284633
:10E1E000B3F9AA21D431BDE8F84318F0DFBEBDE889
:10E1F000F88300BF8C2B00200000C842FFF770BFDF
:10E200002DE9F04190F8E4332C4E00EB031337680E
:10E21000D3F8948100F5907504462846FFF70AFE6E
:10E22000474512D0022812D904F58047C6F800806D
:10E2300097F8503F012B13D815D104F5C046F36869
:10E24000DBB93369CBB905230BE0022810D804F5FC
:10E25000804393F8502F5AB1052283F8502F07E0DE
:10E26000013B87F8503F04F5B7501C301CF096FE78
:10E270002046BDE8F0410CF08DBF114B1B68D86AF9
:10E2800003685B68984780460028ECD194F8E41353
:10E29000B02303FB015104F5A045AC31204606F044
:10E2A0002BF9D5F8F03F0FCB05F6F475143685E859
:10E2B0000F0086E80F0087F8508FD4E7802B0020EE
:10E2C0008C2B0020FFF79CBF70B500F5C0430446BF
:10E2D00093F8EC3100F58056BBB100F5C640103024
:10E2E00015F090FF18B1012386F8C93570BD04F50B
:10E2F000C1455835284610F0B1F908B10023F3E7BD
:10E300002846FFF7A7FD0028F8D104F5A04393F8AD
:10E310001725002AF2D1D3F85C35042BE3D104F59C
:10E32000BE40343090F09EFB86F8C905DEE7000061
:10E3300010B500F5804400F59943D4F8201F9942A8
:10E3400000F5A04308D000F59C42083291421CBF62
:10E350004FF0FF32C3F8D02403F5986207491160EB
:10E3600003F2C443064A1A60FFF7AEFFD4F8200F49
:10E370000368BDE810401B69184700BF0000C84291
:10E380000000C8C2FFF7D4BFF7B500F5A0470446A8
:10E39000D7F85C358B420D4624D00B1F00F5BE46E6
:10E3A000594206F1340659413046019190F04AFA3B
:10E3B0000199304690F046FA072D0BD104F54F50E5
:10E3C000D7F8E0246423052192FBF3F32830064AB2
:10E3D0005EF058FD2046C7F85C5503B0BDE8F0403C
:10E3E00003F040B903B0F0BD08EC0C0870B500F5BF
:10E3F00080460446D6F8200F03689B6B9847B0B15F
:10E4000004F5A04595F858358BB9D6F8202F04F5BA
:10E4100099439A424CD104F5C146583630460FF024
:10E4200039FB60B995F810357BB9012108E004F596
:10E43000C1455835284610F011F900283ED0022178
:10E440002046BDE87040FFF79FBFB5F8BE35152BDD
:10E4500027D195F8381F11F0010120D1D5F85C358E
:10E46000072B1CD095F9AE3F0BB90421E8E72046F5
:10E4700013F0CAFBDFED127AB4EEE70AF1EE10FA00
:10E48000F3DB04F5BE40343090F02CFA0028ECD0D9
:10E4900004F54F500B4A062128305EF0F3FC0721AB
:10E4A000CEE73046FFF7D6FC0028C8D10321C7E7E6
:10E4B00004F59C4308339A42F8D170BD2846F1E731
:10E4C0000000B4422CEC0C0838B5314CD4F8202FA5
:10E4D00004F548639A422DED028B0546B0EE408A62
:10E4E00003D00020BDEC028B38BD2A480FF0D2FAD1
:10E4F00040B1BDEC028B05F5C1405830BDE8384055
:10E5000010F0E4BB04F58055D5F85C35042B35D10B
:10E5100094F8513F33B12049A1F6842038F062FDD0
:10E520000028DFD11D4C94F8EC315BB104F1D80028
:10E530000FF0B0FA0028D4D104F1D8000FF06AFA35
:10E540000028CED19FED167AF0EEC87AF4EEC77AA5
:10E55000F1EE10FA09D49FED130A28EE008ABDEE01
:10E56000C88A18EE103AC5F8E0340F4890F0BAF9AE
:10E570000028B6D0002385F81335B3E7B5F8BE15EB
:10E58000A4F5804007F056FC0028C1D1A9E700BFE0
:10E59000906B0020688C0020948B0020908B0020D2
:10E5A000000000340000C842C48A002010B52DEDE0
:10E5B000028B00F5A0430446D3F85C35042B0BD145
:10E5C00005F024F92046B0EE408A05F03FFA38EE17
:10E5D000400ABDEC028B10BD00F5C04494ED100A5A
:10E5E000F7E700002DE9F0412DED028B00F586657F
:10E5F0008AB0044628461DF089FE002307A904F5C9
:10E6000096500793089309931BF012F9002800F025
:10E6100092809DED090ADFED5F7A04F5A04505F5CE
:10E620009E6393ED007A20EE270ADFED5B7AA7EE7A
:10E63000270A04F5AC40783004F5804783ED000AE2
:10E640006BF06CFE2046FFF7D1FED7F8200F036871
:10E650009B6B9847064604F5C140583010F068FBA4
:10E6600095F81735002818BF0026002B5ED1002E24
:10E670005CD095F85835002B58D1D5F85C35042B73
:10E6800070D09FED468A204605F002FA04F5C0429C
:10E6900004F59943C2F83C04D7F8201F2C33994263
:10E6A0001CD192F88830CBB904F50053B3F90C3C77
:10E6B000002B04DC3A49D1F8EC1BC9060ED5D5F87D
:10E6C000F06FD5F8F81F76680A33891B6426734308
:10E6D0008142ACBF5B181B18C2F83C34D5F85C35DE
:10E6E000D2F83C14D7F8542F059120460492039396
:10E6F00016F088FDB7F9627F06462046FFF756FF01
:10E70000CDE9006704F50050D0ED911A059905F5A3
:10E71000AF6504F53350F0EE400ADDE9033295EDC4
:10E72000001AB0EE480A183086F004FC0AB0BDECBE
:10E73000028BBDE8F08104F59070FFF77BFB0228A7
:10E740000AD994F8E433B02202FB034393F8102271
:10E7500012B193ED7F0A5EE728461DF071FCB1EE21
:10E76000400A58E704F5C04604F5C048043608F1ED
:10E77000140804F5BF4142467431304621F0FCF9DB
:10E7800000283FF47EAF4146304621F089FAB0EED2
:10E79000408A78E7CDCC4C3ECDCC4C3F0000000009
:10E7A000904B0020FFF71EBFF8B500F5804200F542
:10E7B0009A43D2F8202F20339A4204460E4623D0A3
:10E7C00000F5C147583738460FF048FF0546A8B155
:10E7D00038460EF0C9FB70B104F5C044D4F81401FA
:10E7E00003689B689847DFED097A20EE270A86EDDB
:10E7F000000A2846F8BD9FED060AF8E704F5A9448B
:10E800000125A36F3360F4E70025F2E70AD7233C24
:10E8100000000000F8B500F5804200F59A43D2F8F8
:10E82000202F20339A4204460E4630D000F5C147CF
:10E83000583738460FF012FF0546A8B138460EF09B
:10E8400093FB70B104F5C044D4F814010368DB688D
:10E85000984707EE900AF8EEE77AC6ED007A284668
:10E86000F8BDDFED0C7AF8E704F540540125D4F843
:10E87000040603681B69984707EE900A9FED067A25
:10E88000F8EEE77A67EE877AC6ED007AE7E70025CB
:10E89000E5E700BF000000000AD7233CF8B500F50B
:10E8A000804200F59A43D2F8202F20339A42044642
:10E8B0000E4624D000F5C147583738460FF0CEFE3B
:10E8C000054688B138460EF04FFB50B104F5C04400
:10E8D000D4F8143118698BF04BFF86ED000A2846F6
:10E8E000F8BD9FED080AF8E704F540540125D4F877
:10E8F000040603685B69984786ED000AEFE7002588
:10E90000EDE700BF0000000030B505460FC985B037
:10E910006C4684E80F0040F279322146284605F023
:10E9200087FC0C4B03F6E442D3F8203F93420ED110
:10E930009DF8001011F0040102D1204620F018FFCC
:10E940000548214605F024FD012005B030BD00201A
:10E95000FBE700BF906B0020902B002010B5044611
:10E9600006480FF0AFFC40B904F58044D4F8200FFE
:10E970000368BDE810409B6C184710BD688C0020F0
:10E9800010B5044606480FF0F3F840B904F580448A
:10E99000D4F8200F0368BDE81040DB6C184710BDA9
:10E9A000688C002070B5044600F5C14058300E4612
:10E9B00015460EF03BFC50B104F5C044D4F88C333E
:10E9C0009B682B60D4F88C335B68336070BD04F5B2
:10E9D000805303F5996203F2C44312682A601B68EE
:10E9E000336004F50054D4F8EC3B9B05EED4D4ED31
:10E9F000916AD5ED007A9FED037AE6EEC77AC5ED10
:10EA0000007AE3E735FA8E3C38B50C4D04462946CA
:10EA10000B481AF039FE04F5804305F13C0183F8F8
:10EA2000510F04F5965004F5C0441AF0C5FCD4ED1E
:10EA3000107AF1EE677AC4ED107A38BD948B00201D
:10EA4000503E002010B5044600F590702AF002FBFD
:10EA50002046BDE81040FFF7D7BF0000FFF7F2BF28
:10EA600000F50050D0F8EC3B194214BF0120002003
:10EA70007047000010B500F580430446D3F8200F1E
:10EA800003689B6D9847014604F59C406030BDE8E3
:10EA9000104092F095B90000FFF7ECBF38B5054B78
:10EAA0001C6823680A461D68034B01462046A84798
:10EAB000002038BD8C2B0020902B002070B52DED50
:10EAC000028B0446036804F500559B6D9847D5F802
:10EAD000EC3B1B0617D5B5F9A831B5F9AA11CA1A2E
:10EAE0000B4402EBD27203EBD37352105B1000EEB7
:10EAF000902A00EE103AF8EEE00AB8EEC00A04F5EB
:10EB000096501AF0DFF9604BB5F8DA211A7004F567
:10EB1000C14568F037FB103567F0C6FF0021284675
:10EB2000FEF764FE594E0123B0712846F37181F05F
:10EB30007FFC28B9284682F029FDB0FA80F0400910
:10EB400030710421204614F055FE20B104F5AD408B
:10EB5000183058F039FC284681F06AFC04F5C045AD
:10EB6000D8B994F8E43304EB031341F28832D3F8B4
:10EB70009461D5F88C30F31A93420ED904F5907055
:10EB8000FFF758F9022808D9C5F88C60204605F02F
:10EB900043FC04F5BE4300225A63B4F9A4301BB908
:10EBA000B4F8A230A4F8A430B4F8A430DFED388A69
:10EBB00007EE903AF8EEE77AB7EE008A88EE270A79
:10EBC000D4ED2B7AF0EEE77AF4EEE87AF1EE10FA73
:10EBD00009D5B4F9A23007EE903AF8EEE77A88EE5C
:10EBE000277A84ED2B7AD4ED2B0A31F09BFB70BB96
:10EBF00059F0C8FA40F27D124FF4801159F07AFAB8
:10EC000056F082FF56F0EAFB95F8EC31B0EE408A00
:10EC100023B1D5F80C0103681B6F984704F53E50EB
:10EC2000B0EE480A143079F0FDFB04F54350B0EE25
:10EC3000480A303079F0F6FBB0EE480ABDEC028BA2
:10EC400004F548502430BDE8704079F0EBBBD4EDBA
:10EC50002B7A94ED460AF0EEE77AF4EEE87AF1EEDC
:10EC600010FA09D5B4F9A23007EE903AF8EEE77A37
:10EC700088EE277A84ED2B7AD4ED2B0A31F052FB03
:10EC80000028B5D0BCE700BF942300207D90002071
:10EC900000000034FFF712BF70B500F5A04604462F
:10ECA00096F9AC3F002B28DD07F0ACFF28BB04F53C
:10ECB000C1451035284682F069FCF0B1284681F044
:10ECC000B7FBD0B193F08AFCD6F80035C01A96F99C
:10ECD000AC3F4FF47A72534398420ED301221C2169
:10ECE0002846FEF755FF40B104F54F50034ABDE8F2
:10ECF0007040062128305EF0C5B870BD4CEC0C08A1
:10ED000000B52DED028B9FED0B8AD0ED4E7A67EEAC
:10ED1000887A83B0C0ED4E7A3830019079F0E0FB0C
:10ED2000019820EE080A03B0BDEC028B5DF804EBFD
:10ED300079F0EEBC52B87E3F00B52DED028B9FED11
:10ED40000B8AD0ED4F7A67EE887A83B0C0ED4F7AA8
:10ED50003C30019079F0C4FB019820EE080A03B022
:10ED6000BDEC028B5DF804EB79F0D2BC52B87E3F6B
:10ED700030B52DED048B83B0044601A900F5965003
:10ED80001AF028FD002800F0B98004F5A94595ED9A
:10ED90001A7ADDED017AB4EEE77AF1EE10FA05F1B8
:10EDA000680507D504F5C140103081F04BFB08B170
:10EDB000019B2B6004F5005595ED7F7AB5F9A831DC
:10EDC000DFED606A052BB8BF052307EE903AB5F971
:10EDD000AA31F8EEE78A07EE903AF8EEE77AB6EE57
:10EDE000009A77EEA77A1820C7EE270ADFED567A49
:10EDF00068EEA77AF4EE490A87EE271AF0EE007A59
:10EE0000F1EE10FAB4EE671AC8BFF0EE490AF1EE5F
:10EE100010FA48BFB0EE671ADDED017AF4EEE67A3B
:10EE2000F1EE10FACCBF87EE270AB0EE410A31F0BE
:10EE30008BFB04F5C1405830B0EE408A0FF00EFC59
:10EE400038B904F5C04393F8EC21D2B393F81932E2
:10EE5000BBB304F5C140103081F0F4FA88B328EE5A
:10EE6000892A9DED011AB4EEC21AF1EE10FA28D5E6
:10EE7000D5ED7F0ADFED351A9FED350AC0EE820A27
:10EE800031F094FA04F53D501C30B4EE408AF0EEB7
:10EE9000408AF1EE10FA48BFF0EE488AFFF730FFE3
:10EEA00004F54250343004F54054FFF745FFD4EDEB
:10EEB000D97A9FED287A67EE877AB0EE688AC4ED3A
:10EEC000D97A254819F034FC90B924484021FFF73D
:10EED000C7FD68B1224BD3F85C35012B08D1F7EEA2
:10EEE000007AB4EEE78AF1EE10FA58BFB0EE678A06
:10EEF000B0EE480A03B0BDEC048B30BD04F5C14050
:10EF0000103081F09FFAB7EE008A0028D9D0462051
:10EF100067F0E0FBB4EEC80ADFED127AF1EE10FA0A
:10EF2000D8BFB0EE480A87EE800AB9F073F92F20F7
:10EF30009FED0D1ADFED0D0A31F006FBB0EE408AB1
:10EF4000BFE700BF17B7D1383333333F00000000AD
:10EF50006F12833A52B87E3F503E0020902B002023
:10EF6000907B0020000034428FC2D53F9A99193F10
:10EF7000F8B5044666F088F80368DB6898470546EC
:10EF800010B900252846F8BD04F58046204607F054
:10EF9000B7FCD6F8202F04F59B4330339A4207463E
:10EFA00005D104F5C04393F8AC32022BE9D804F53F
:10EFB000C14058300FF078FD0028E2D1D6F8200F7C
:10EFC00003689B6B984758B996F8343F002BD9D00B
:10EFD00004F5005494F91452023D18BF0125D1E7FD
:10EFE000084BD3F8200F03685B6B98470028EBD0E1
:10EFF00004F5005494F95132002BC2D0032BC0D039
:10F000003D46BFE7906B002070B52DED028B0446A6
:10F0100000F5804600F5C14006F5776382B05830B0
:10F0200093ED008A0FF054FC04F53D551C35002883
:10F0300046D104F5C046D6F80C0103689B68984792
:10F04000D6F89C335B0225D5D6F80C3193ED437A84
:10F05000D3ED097A67EE877A9FED327AF4EEC77ABC
:10F06000F1EE10FA16DB04F5005404F5766393ED27
:10F07000007A67EE877AF7EE006A86EEA77A04F6E2
:10F080005C74B4EE667AF1EE10FAC8BFB0EE667A40
:10F0900084ED497ADFED247A90ED250AF0EE480AF6
:10F0A00020EE270A284683F015F928468DED010A3F
:10F0B000FFF726FE9DED010A02B0BDEC028B70BD8C
:10F0C000D6F8202F04F5974310339A4228D104F53F
:10F0D0000053D3F8283CB3F90860003E18BF01265E
:10F0E00004F5A04204F58054D2F87035D4F8B84441
:10F0F0001C1B92F86C353BB10C484FF40061FFF7D4
:10F10000AFFC80F00100C3B23246B0EE480A21469F
:10F11000284602B0BDEC028BBDE8704083F0DEB83B
:10F120000026DDE700000034E02E6542902B002031
:10F1300010B5044606F0A4FF98B104F5A042D2F839
:10F14000703503F58C415031C2F8701504F58051CB
:10F15000D1F8B8140029BEBFA3F58C43503BC2F8C8
:10F1600070352046FFF750FFBDE81040042067F0DF
:10F170009DBA00002DE9F04700F5C1442DED048B48
:10F1800000F580495834054609F577632046D3EDEC
:10F19000008A0FF09DFB05F542563436002844D115
:10F1A00005F5C044D4F80C010368DB689847D4F82F
:10F1B0009C335B0221D5D4F80C3193ED447AD3ED26
:10F1C0000B7A67EE877A9FED537AF4EEC77AF1EE09
:10F1D00010FA12DB05F5405595ED2E7A67EE877A29
:10F1E000F7EE006A86EEA77AB4EE667AF1EE10FAD0
:10F1F000C8BFB0EE667A85ED777A90ED250ADFED2F
:10F20000467AF0EE680A20EE270A304682F0BCFC0F
:10F210003046B0EE408AFFF78FFDBDEEC80ABDEC68
:10F22000048BB8EEC00ABDE8F087204605F500580B
:10F230000DF0C8FE9FED399A98ED918A28EE098A63
:10F2400005F5A047BDEEC88AD7F8743518EE102A28
:10F250001A4408EE102A8246462067F03BFAB8EEC0
:10F26000C88AD8ED7B7AD9F8200FA0EE278A05F559
:10F27000974310339842FDEEC87A17EE904A45D175
:10F28000D8F82C3CB3F90880B8F1000818BF4FF04B
:10F290000108BAF1000F1ED103685B699847D0B925
:10F2A000D9F8200F03689B6B9847A0B905F5C043B8
:10F2B000D3F83434022B0ED1284612F0EFFA50B1B5
:10F2C00007F68C73D3ED007A67EE897AFDEEE77A64
:10F2D00017EE903A1CB205F58055D5F8BC34E41A07
:10F2E00097F86C353BB10E484FF40061FFF7B8FB5F
:10F2F00080F00100C3B2B0EE680ABDEC048B424658
:10F3000021463046BDE8F04782F024BD4FF00008AA
:10F31000BFE700BF00000034E02E65420000C84295
:10F32000902B002010B5044616F0B4F868B100B276
:10F3300000EB4000C0EB001300EE103AB8EEC00A3C
:10F34000BDE81040132067F0B1B92046FFF712FF67
:10F35000F6E7000010B51048FFF70AFED0B10F48DD
:10F360000FF0DCFCB0B10E4C042067F0B3F9D4F818
:10F37000280C66F0F9F8042067F098F9132067F07C
:10F38000A9F9D4F82C0C66F0EFF8BDE81040132072
:10F3900067F08CB910BD00BF902B0020688C002056
:10F3A000904B0020F8B52DED028B0446FFF7E0FDF1
:10F3B000002800F0AB8004F5804704F59742D7F8A9
:10F3C000203F4832934200F0A18004F59842043275
:10F3D000934200F09B8004F598426432934200F01F
:10F3E000958004F598422032934200F08F8004F516
:10F3F00098423C32934200F0898004F59A423C32B4
:10F40000934200F0838004F59A42583293427DD0B3
:10F4100004F59A427432934278D004F59B42143238
:10F42000934273D004F59B42503293426ED004F560
:10F43000C14058300FF072FC002867D0D7F8202F59
:10F4400004F597432C339A4260D004F50055F6EE4C
:10F45000008AD5F8280C65F047FFB4EEE80AF1EE13
:10F4600010FA40DDB0EE087AFFEE007AE0EE077A9F
:10F47000B0EE670AD5F8402C04F5A04607EE902AB6
:10F48000D6F87035B8EEE77A07EE903AF8EEE77AFC
:10F490005142E7EE007AFDEEE77A17EE900AC6F8E1
:10F4A000700531F0F1F8C6F87005D7F8202F04F593
:10F4B000994348339A4222D0D5F82C0C65F014FFBA
:10F4C000B4EEE80AF1EE10FAB0EE408A21DCFEEE6E
:10F4D000007AB4EEE70AF1EE10FA22D5B0EE087A1F
:10F4E000F7EE007A19E0FEEE007AB4EEE70AF1EEEC
:10F4F00010FABFD5B0EE087AF7EE007AB6E72548E5
:10F500004FF48051FFF7ACFA0028D5D0BDEC028B48
:10F51000F8BDB0EE087AFFEE007AE8EE077AB0EEBA
:10F52000678A204606F0ACFD08B1B1EE488AD6F8ED
:10F530007435D5ED706A9FED186A05F6444595ED72
:10F54000007AB5EEC08A07EE903AF1EE10FACCBF21
:10F5500028EE268A27EE488AF8EEE77A66EE866A73
:10F56000E8EE067A27EE067AFDEEE77AFDEEE66A29
:10F5700017EE903ABDEEC77A16EE902A17EE101AE3
:10F5800017EE900AC6F8743531F07EF8C6F87405A7
:10F59000BCE700BF902B00200000C842F8B504462D
:10F5A00004F5C04793F01AF897F8EC31064653B1CA
:10F5B000D7F81402036804F5AA4204F5AA411B6AAD
:10F5C00070327431984704F58045D5F8303FF31A0E
:10F5D000B3F5FA6F03D9D5F8200F08F06DF82C4B6E
:10F5E000C5F8306FD3F8200F0268136898470021E0
:10F5F000204612F009FBDFED277AB0EEC00AB4EE28
:10F60000E70AF1EE10FA42D5D7ED107AB1EE047A9E
:10F61000F0EEE77AF4EEC77AF1EE10FA37D504F59A
:10F6200086601CF00DFDF6EE007AB0EEC00AB4EE76
:10F63000E70AF1EE10FA2AD504F5B65595ED017AF0
:10F64000F0EE087AB4EEE77AF1EE10FA05F104056F
:10F650001DD504F53D501C3082F0B0FE04F542503B
:10F66000343082F027FC04F548500C3083F054FB12
:10F6700095ED007AF7EE007AB4EEE77AF1EE10FA43
:10F6800005D504F54E50BDE8F84083F09BB8F8BDB1
:10F69000906B00200000003400F5005090F99F317D
:10F6A000012BC3BF00F6D84090ED290ADFED047AA4
:10F6B0009FED040AC8BF20EE270A462066F0F6BF79
:10F6C0000000C842000000002DE9F8432DED028B38
:10F6D00000F5804909F57763D3ED008A054611F0FE
:10F6E000E1FE8046D9F8200F03681B6A984705F5AC
:10F6F00048560C3698B14F4CD4F83C35002B0EDDF3
:10F7000092F06CFFD4F83C35C01A40F6B7339842FB
:10F7100005D8B4F93045304683F00AFB7AE005F5A8
:10F72000C04305F5005793F8293443B1B7F9303297
:10F73000002B04DD05F5405393F9223203BBD9F8C1
:10F74000203F05F597451035AB426DD00021B0EE56
:10F75000680A304683F084F80546042066F0BAFF54
:10F760002BB207EE903A97ED797AF8EEE77AE0EE71
:10F77000077AFDEEE77A17EE904A444424B2CAE7CE
:10F780002846012112F080F89FED2B7AB7F930322C
:10F79000C0EE077A05F5A04505F27C5508EE103A53
:10F7A00055F80C3C9FED250AB8EEC88A28EE278A4A
:10F7B00007EE903AF8EEE77A67EE807A9FED200A3E
:10F7C00027EE800AB8F04AFBB7F9A831DFED1D7AC1
:10F7D00095ED007A20EE270A07EE903AF8EEE77AE8
:10F7E0000021B4EEE77AF1EE10FA58BFF0EE477A56
:10F7F00080EE277A3046DFED147AB0EE480AA7EEA5
:10F80000270AF0EE680A83F087F9BDEEC00A10EE11
:10F81000103A1CB2BDEC028B20460C49BDE8F843FF
:10F8200041F2941230F040BFB8F1000118BF01213D
:10F830008DE700BF907B002000A08C450AD7233CB9
:10F8400035FA8E3C0AE81C41E02E65426CEEFFFF63
:10F8500038B500F540530546D3F804060368DB6865
:10F860009847014605F54E5082F08EFF04B22846B7
:10F87000FFF77EFB70B107EE904A05F50055B8EE34
:10F88000E70AD5F8340C65F06FFEBDEEC00A10EE45
:10F89000103A1CB220460349BDE8384041F29412A8
:10F8A00030F002BF6CEEFFFF38B590F8E433B022C1
:10F8B00002FB030393ED777AF7EE007AB4EEE77A72
:10F8C000F1EE10FA054600F5A0441DD5002112F016
:10F8D0009BF9DFED417AB0EEC00AB4EEE70AF1EE33
:10F8E00010FA11D5D4F85C35012B0DD0072B0BD0B5
:10F8F000002384F8D43404F59B6400232360284655
:10F90000BDE8384011F0CEBD92F068FED4F8DC348A
:10F91000C4F8DC04C31AB3F57A7F84BF002384F8EB
:10F92000D434284611F0BEFDD4F85C35012B07EE27
:10F93000100A2CD0072B2AD0B8EEC77ADFED276A41
:10F94000C7EE267A05F50052B2F9F42100EE102A2E
:10F95000B8EEC00A27EE800ADFED1F7AB0EEC07A5B
:10F96000B4EEE77AF1EE10FA13D4002384F8D4341D
:10F9700094F8D43405F54E50DBB982F0EDFDBDE8C6
:10F980003840174900B241F2941230F08DBE9FED1D
:10F99000150A94F8D424002AEAD10122934284F86B
:10F9A000D424E5D0072B1EBF04F59B6300221A6008
:10F9B000DEE704F59B6494ED007ADFED0B7A67EEE9
:10F9C000C77A9FED0A7A67EE877AFDEEE77A17EE3F
:10F9D000901A82F0D9FED2E70000003400A08C45D6
:10F9E0006CEEFFFF00000000E02E65420000C84200
:10F9F00070B52DED028B00F5BE46343682B004465C
:10FA000030468EF09FFE0546D8B904F50053D3F872
:10FA1000282CB2F9082072B904F5C042D2ED107A50
:10FA200093ED7C7AF0EEE77AF4EEC77AF1EE10FA15
:10FA30004CBF0125002530468EF098FE002808BFF7
:10FA4000002530468EF07EFE50BB04F5A043D3F86F
:10FA5000D03401331ED01DBB9FED1C8A2046FFF71A
:10FA600033FE07EE900AB8EEE70A8DED010AFDB904
:10FA7000152066F01BFE9DED010A1A2066F016FEA9
:10FA800004F5C240603002B0BDEC028BBDE87040AE
:10FA900003F010BC002DDFD02046FFF705FF02E089
:10FAA0002046FFF7D5FE07EE900AB8EEE78AD5E7C5
:10FAB0001A2067F0A7F89DED010A08B9B0EE480AD0
:10FAC000152066F0F3FDB0EE480AD6E7000000000E
:10FAD00010B500F5005303F64442D3ED706ADFED34
:10FAE000127A92ED007A9FED116A03F6D84366EE22
:10FAF000A76A27EE277AD3ED2A7A67EE867AFDEE9B
:10FB0000E66ABDEEC77AFDEEE77A044616EE902A65
:10FB100017EE101A17EE900A30F0B6FD04F5A04467
:10FB2000C4F8740510BD00BF0000C842A00CB34566
:10FB300010B5044613F062FE031E2ADB04F50051E3
:10FB400091F99F219A4224DD04F5A040D0F85C454C
:10FB5000022C1ED0D1ED7E7ADFED0E6AD31A66EE4E
:10FB6000E76A07EE102A07EE903AB8EEC77AF8EE89
:10FB7000E77AD0F8743587EE876A07EE903AF8EEA8
:10FB8000E77AE6EE867AFDEEE77A17EE903AC0F86D
:10FB9000743510BD0000C84270B52DED028B00F524
:10FBA000A0459FED550AD5F870359FED547A07EEC4
:10FBB000903AF8EEE77A044667EE807A9FED500AB5
:10FBC000F0EEE76AF4EE476AF1EE10FAC8BFF0EE25
:10FBD000477A27EE800AB7F0B1FF30F0D7FBB7EED7
:10FBE000008AC8EE007A05F5AF6304F50056C3ED50
:10FBF000007A04F5C04393F8EC219AB1D3F81402CB
:10FC0000036804F531515B6A984758B1D6F8402C27
:10FC1000D5F87005514230F037FDC5F87005BDECE0
:10FC2000028B70BD96F9D031002BF8D0204606F03B
:10FC300027FA0028F3D104F5C640103013F0DCFF9A
:10FC40000028ECD1B6F9A831012BB8BF012307EE8B
:10FC5000903A05F27C52F8EEE77AD2ED006A86EE31
:10FC6000A77AB4EEC87AF1EE10FA13D840F6C412AF
:10FC70002449D5F8700530F007FDC5F87005D6F8B1
:10FC8000402C40F6C4139A42D4BFC6F8402CC6F8A4
:10FC9000403CC4E705F5AF63D3ED007AF4EEC77AD4
:10FCA000F1EE10FABBDD88EE070A20EE000AB8F08C
:10FCB000FFF8DFED157AD5F8700520EE270ADFEDA5
:10FCC000137A20EE270A40F6C413FDEEC07A17EE31
:10FCD000904A9C42B8BF1C462246614230F0D4FC98
:10FCE000C5F87005D6F8403CA342D4BFC6F8403CE6
:10FCF000C6F8404C93E700BF0AD7233C0000AA4255
:10FD000035FA8E3C3CF6FFFFE02E65420000C8420B
:10FD100010B500F540530446D3F8040603681B6889
:10FD2000984704F50053D3F8402C514230F0ACFC16
:10FD300004F5A043C3F870052046BDE81040FFF766
:10FD40002BBF00007047000001207047082070475B
:10FD500001207047014B93F8DC017047904B002065
:10FD6000034B93F9E409003818BF0120704700BF26
:10FD7000904B0020014B93F9DE017047904B00201F
:10FD800013B5064BD3F8200F4B6904680093083174
:10FD90000EC9646CA04702B010BD00BF906B00207C
:10FDA000704700007047000038B5264DD5F8200F89
:10FDB00003685B68984719283CD8DFE800F00D39E4
:10FDC000370D0D373737373B3939393939393B3703
:10FDD000373737393B0D393940241B4B93F8E12332
:10FDE00012B193F8E0330BB944F01004174BD5F877
:10FDF000202F9A42A3F11C0303D09A4218BF44F06B
:10FE00001004134991F95102B0B19A4216D0032857
:10FE100003D101F532518A4201D144F040040D482A
:10FE200080F006FB50B144F0800407E01024D4E7D2
:10FE30001824D2E70124D0E79A42F0D144F001001F
:10FE400038BD00BF906B0020905B0020B078002090
:10FE5000904B0020208C002008B5044806F0D2FE0C
:10FE600000280CBF0120022008BD00BF902B0020FD
:10FE7000F0B52DED028B8BB0054619F0DBFE4FF48B
:10FE80008071D0F8047290ED828AD0F80C6204463A
:10FE90001948FEF7E5FD30B9184BDFED197A93EDFF
:10FEA000917AA7EE678A17480DF0C0F930B1164B6A
:10FEB000D3F88C335F6893ED028ADE682D7C92F074
:10FEC0008DFBD4F81823D4F81C33D4F814130892FB
:10FED000099327221C23CDE900320390079103AA3E
:10FEE0001E21284604978DED058A06965DF0E8FFF1
:10FEF0000BB0BDEC028BF0BD902B0020904B00208E
:10FF000035FA8E3C688C0020908B002038B5C5787F
:10FF10000B46352D044628BF3525352200211846CD
:10FF2000BAF028FA2A4604F10C01BDE83840BAF0CC
:10FF3000D7B9000008B5024813F060FC00B208BD54
:10FF4000902B002037B50D46134840F2EF2204F005
:10FF50006FF92C7814F004040AD0696803220F4862
:10FF60001FF042FB0C4803B0BDE8304003F0C0BABC
:10FF700001AA214628461FF00BFC0028F2D0DDED37
:10FF8000017A9FED077A67EE877A2246FDEEE77ADF
:10FF900017EE901AE3E700BF902B0020A48B0020FF
:10FFA0000000C84210B5054C012384F8E3335FF02C
:10FFB00009FC002384F8E33310BD00BF905B0020F0
:10FFC00062F03EBD2DE9F0412DED028B4FF00008AF
:10FFD00082B0CDE900281E4F9FED1E8A0C461546C3
:10FFE000B0EE480AB1F90220D7F8281C4FF47A7312
:10FFF000064662F0FFFF0123CDE90053B4F900206B
:020000040801F1
:10000000D7F82C1CB0EE480A30464FF47A7362F0F1
:10001000F1FFB4F90420D7F8301C9FED0F0A4346D6
:100020003046CDE9005862F0E5FFCDE90058B4F95B
:100030000620D7F8341CB0EE480A4FF47A733046E5
:1000400062F0D8FF02B0BDEC028BBDE8F08100BFCA
:10005000904B00200000FA4400007A4410B5074B92
:1000600093F9982640F24D3440F24D13002A08BF10
:100070001C465FF09FF9204310BD00BF907B00201D
:1000800010B504461FF0E4FE204610BD10B50B4C21
:10009000002384F8133560F08FF854F8E02CA4F5B1
:1000A00060739A4208D194F884352BB904F5B06096
:1000B000BDE8104036F0F0BE10BD00BF907B0020C0
:1000C00013B5124C94F83610A4F58C7017F0F0F8B4
:1000D00078B194F83610A4F58C7017F057FB40B146
:1000E00094F83610A4F58C7002B0BDE8104017F0FB
:1000F0008FBB19F09FFD01A919F06CFB18B19DEDA4
:10010000010A02B010BD9FED020AFAE7904B0020F1
:1001100000000000044B93F8EC0120B1D3F8140266
:1001200003681B6B18477047908B002008B5084B7D
:10013000D3F8D02B002A03DCBDE808405FF07EB97D
:1001400003F52F605CF0ECFA90ED000A08BD00BFEB
:10015000904B002008B51248D0F8202F00F6045329
:100160009A4216D0B0F9383FABB900F5805393F8F6
:100170009D2482B990F8352F6AB993F8493563B94F
:10018000A0F5804006F03EFD00280CBF03200420AF
:1001900008BD0220FCE70520FAE70620F8E700BFCB
:1001A000906B002010B5214B03F55262D3F8203F2D
:1001B000934290B0044636D000231D4802931FF0AE
:1001C000FDF9014618B91A4802AA1FF043FA247C27
:1001D00092F004FA174BDDED027A9FED177AD3E91E
:1001E000072305930023F8EEE77A07930893099312
:1001F0000A930B930C930D930E934FF6F853ADF8AF
:100200003C300023CDE9030267EE877A96228DF811
:100210003E303323CDE90032572103AA2046CDEDED
:10022000067A5DF04DFE10B010BD00BF906B00204F
:10023000A48B0020908B00200AD7233CF0B58DB012
:10024000044692F0CBF9184AD2F81032C31A642B44
:1002500028D8D2F80C310290D3F88C10D3F8902023
:10026000D3F88460D3F88850D3F8DC70D3F894E0E6
:10027000D3F898C0D3F89C30099300238DF82C3024
:10028000069225231622CDE900320591207CCDF877
:100290001CE002AA5321CDF820C00A9703960495CA
:1002A0005DF00EFE0DB0F0BD908B002010B55FF03C
:1002B000CBFA044678B9094850F8E02C80F8134589
:1002C000A0F560739A4206D190F884351BB900F509
:1002D000B06036F0E1FD204610BD00BF907B0020ED
:1002E0002DE9F0472DED088B8B4CD4F8202F04F529
:1002F00052639A4290B0054600F0E7808748DFEDF0
:10030000888ADFED889A9FED889A0CF08FFF00288D
:1003100067D082480CF028FE002862D004F500580F
:100320009FED820AD8F80C016C3033F01BFA08F10B
:10033000E400B0EE60AAB0EE418ACDED070A8DED83
:10034000081AF0EE40AA8DED060A85F03FFAD8F8BB
:1003500010310146D3F85C23D3F85833059204A832
:10036000049332F0FFFF09A88DED090AB0EE680A88
:10037000CDED0A0A33F006F828EE288A02A8BDEE71
:10038000C88A95F81090CDED030A18EE103A8DED5D
:10039000020A1EB233F06AF8DFED657A20EE270A12
:1003A00002A8BDEEC00A6AEEA8AA10EE103A1FB26B
:1003B00033F0A6F8B4EEE90AF1EE10FA58BFB0EE49
:1003C000690ABCEEC00AD4F8202F10EE103A9DB294
:1003D00004F63C539A422AEE28AA7BD1DFED558AD7
:1003E0007EE0DFF854A195F81090DAF804760AF56B
:1003F00000583846D8F8703507EE903AD8F874357A
:10040000B8EEE7BA07EE903A3B689B68F8EEE7AAC9
:10041000984707EE900AF8EEE77A384667EEA87A32
:1004200008F59F68FDEEE77A04F65C7417EE903AE3
:100430001EB23B681B69984707EE900AF8EEE77A10
:1004400098ED00AA67EEA87AB4EEE9AAFDEEE77A85
:10045000F1EE10FA17EE903ADFED327AAAF540503D
:1004600058BFB0EE67AA1DB203F026F93B68D4ED81
:10047000007A5B6908EE100A384627EE899A984799
:10048000B8EEC88ABCEECAAA2BEE28BA6AEEA8AAB1
:100490001AEE103A68EE288A8DED09BACDED0AAA57
:1004A000CDED0B8A8DED0C9A8DED0D0AADF838600F
:1004B000ADF83A50ADF83C30B7221A23CDE90032FE
:1004C0003E2109AA48465DF0FBFC10B0BDEC088B4C
:1004D000BDE8F087D8F81031D3ED0F7A67EEA88A1F
:1004E000D8F8143104F65C74D4ED007A186927EE5C
:1004F000899A8AF03DF9CDED09AA8DED0AAACDEDD4
:100500000B8A8DED0C9A8DED0D0AADF83860ADF8C3
:100510003A70ADF83C50CFE7906B0020688C00201B
:100520000AD7233C00FF7F470000C8429F0CB34519
:10053000E02E654200000000905B002001480CF0B6
:1005400025BD00BF688C002008B5034BD3F8200FF1
:1005500003685B68984708BD906B002030B587B092
:10056000054619F067FB04462D7C92F02BF8D4F871
:100570008422D4F888320492059300211023CD22DE
:10058000CDE900320290039102AA42F60C312846CE
:100590005DF096FC07B030BD30B52DED028B89B013
:1005A000054619F047FB00F55A7393E8070002ACC3
:1005B00084E80700DDED020A9DED030A2D7CF1EED3
:1005C000600AB1EE400AB7F0DBFC2046B0EE408A8C
:1005D00033F04CFDDFED0B7A049B079328EE278A5E
:1005E0000C230122CDE90032A82105AA28468DED71
:1005F000058A8DED060A5DF063FC09B0BDEC028B47
:1006000030BD00BFE02E6542282938B5054623D00D
:1006100007D824292BD0272911D01B2908D1012440
:1006200013E0432937D008D84029F8D0422928D0F0
:100630002846BDE8384063F00FB85329EEE7122191
:100640005CF03CFE044610B90024204638BD297CED
:10065000134855F0F9FDF8E716215CF02FFE04462B
:100660000028F1D0297C0E4855F0C8FEEDE70C219A
:100670005CF024FE04460028E6D02846FFF78CFFF5
:10068000E3E710215CF01AFE04460028DCD028467F
:10069000FFF764FFD9E7017C02488EF051F8BEE70E
:1006A00028820020C48A0020F0B52DED028B05467B
:1006B0008DB01646B0EE408A0C46002930D0007C42
:1006C0005DF094FB0746287C5EF094FA00F121036C
:1006D0009F4207D2287C0DB0BDEC028BBDE8F040F4
:1006E0005CF0DABD63690893636A2269CDF825304E
:1006F000236AA069E1680792CDF82930622221239C
:1007000027680590CDE900320691287C03971923CC
:1007100003AAC2218DED048A8DF824605DF0D0FB20
:100720000DB0BDEC028BF0BDF8B54B4CD4F8202FCA
:1007300004F552639A42054600F08C80A4F50056F9
:10074000B6F88232DF0713D544480DF087FF002842
:1007500079D004F50054D4F80C0103689B689847DD
:1007600000F1940191ED010A01222846FFF79CFF58
:10077000B6F882329C0712D538480DF06FFF00287A
:1007800064D0374BD3F80C010368DB68984700F15D
:10079000940191ED010A02222846FFF785FFB6F881
:1007A0008232580712D52D480DF058FF00284FD03F
:1007B0002B4BD3F80C0103681B69984700F1940197
:1007C00091ED010A03222846FFF76EFFB6F8823248
:1007D000190708D52349052291EDED0A284601F5B0
:1007E0006C71FFF761FFB6F88232DA0616D51E4F3C
:1007F000D7F85C35042B11D119F01CFA044607F622
:1008000034708DF0CDFF94EDC70ADFED187A014604
:1008100020EE270A06222846FFF746FFB6F8823266
:100820009B0617D50D480DF019FF98B10C4BD3F866
:100830001011284691EDAB0ABDE8F840042201F5FD
:100840002A71FFF731BFA4F67C718BE70849A0E756
:100850000849B5E7F8BD00BF906B0020688C002008
:10086000908B0020905B0020907B0020E02E654262
:10087000705D0020E45E002070B504460E4628F04E
:1008800027FC90F8C412B02303FB0101AC312046D1
:1008900003F032FE0546C0B13EB119F0CBF990F835
:1008A0007C3243F0020380F87C3204F58043D3F8B5
:1008B000200F04F599432C33984204D004F59B444F
:1008C0003034A04201D106F01BFE284670BD000066
:1008D00073B516460191044619F0ACF9019918F068
:1008E000C1FD0546C0B13EB119F0A4F990F87C32C3
:1008F00043F0020380F87C3204F58043D3F8200FE4
:1009000004F599432C33984204D004F59B443034C9
:10091000A04201D106F0F4FD284602B070BD0000EF
:1009200030B5054685B00C46D1E9040130F010FF22
:1009300040B168461EF052FE6A462146284662F0E3
:10094000C9FA08B9022067E0344840F24F326946DC
:1009500003F06EFCD4ED037AF4EE677AF1EE10FA50
:1009600022D69FED2F7AF0EEE77AF4EEC77AF1EE19
:1009700010FA54BF012200229DF80030294962F389
:10098000410368468DF800301EF092FF0028D9D14F
:10099000254869466EF012FC40B959F005FA052267
:1009A000162158F0B9FFCDE70022E5E7D4ED017A32
:1009B000FDEEE77A17EE903ADB0706D41B4B03F601
:1009C000E442D3F8203F934225D11949134802222B
:1009D00012F022FD9DF8001011F0040102D16846CA
:1009E0001EF0C6FE0D48694603F0D2FC94ED020AE3
:1009F000B4EE400AF1EE10FA0BD6B5EEC00AF1EEF5
:100A000010FA06DD9DF800100948C1F3400107F017
:100A100065FF002000E0042005B030BD902B0020D1
:100A200000000034948B0020304C0020906B00209C
:100A30007478002010B52DED028BD1ED017A91ED87
:100A4000008AFCEEE77A8AB0CDED037A9DF80C10AF
:100A500005AA044662F028FAC8B1DFED0E7A059BBC
:100A6000009368EE277A0022FDEEE77A114617EE32
:100A7000903A06A81EF0D2FD23682046D3F8C43071
:100A800006A9984700200AB0BDEC028B10BD0220D9
:100A9000F9E700BF0000C84237B5124DD5F8200F66
:100AA00003681B6A0C46984740B9D5F8202F05F516
:100AB00048639A4202D0042003B030BDD4ED007ADE
:100AC000D4ED020A94ED010A0748FCEEE77ACDED79
:100AD000017A9DF8041004F0B7F90028EBD000204B
:100AE000EAE700BF906B0020902B0020134610B562
:100AF00024220C4618460021B9F03CFCA27F8277E4
:100B0000E27FC277072280F82020A28B8283D4ED77
:100B1000067AF1EE677AC0ED067A10BD10B48C8BC0
:100B2000162C03D15DF8044BFFF7E0BF5DF8044BD2
:100B300061F0F8BB08B591F82030072B0DD10948BA
:100B400090F8EC313BB191ED060AD830B1EE400A95
:100B50000DF04CFB18B9042008BD0220FCE7002072
:100B6000FAE700BF908B002008B5D1ED007A9FED29
:100B7000087A0848F0EEE77AF4EEC77AF1EE10FA58
:100B800054BF0121002105F075FA002008BD00BF07
:100B900000000034902B002010B5D1ED007AFCEE5F
:100BA000E77A17EE903A9CB2012C02D0022C06D0C4
:100BB00084B91148214669F01FFB002010BD0F4881
:100BC00090F88C365B0707D562F0BCFF0C4A052114
:100BD0005CF058F90420F1E790F978361BB962F01F
:100BE000B1FF084AF3E7A0F5A0400AF049FE00284B
:100BF00014BF00200420E1E708820020907B002041
:100C0000F8F10C0813F20C081FB5D1ED017AFCEED7
:100C1000E77A0B46CDED027AD1ED007A1A7C017CA1
:100C20000192FCEEE77A0B48CDED037AD3ED027A20
:100C3000FCEEE77A17EE902A92B2009293ED030A47
:100C40009DF80C209DF8083009F062FF05B05DF8B2
:100C500004FB00BF688C002007B5D1ED007A08487E
:100C6000FCEEE77ACDED017A9DF804100BF096FDCD
:100C700000280CBF0420002003B05DF804FB00BF77
:100C8000688C002070B58B8BC02B05460C4633D882
:100C9000B12B0DD8142B00F0B080162B59D0112B8E
:100CA00000F0A78021462846BDE8704063F06CBB89
:100CB000B23B0E2BF6D801A151F823F0410D0108EB
:100CC000A50C0108A50C0108A50C0108A50C01083C
:100CD000A50C0108A50C0108A50C0108370D010899
:100CE000A50C01086B0D0108A70D0108A50C010852
:100CF0005B0D01082D0D0108D42B13D007D8D02B84
:100D000023D0D12BCED1BDE87040FFF77DBFB3F526
:100D1000967F53D040F6B836B342C3D1BDE8704099
:100D2000FFF79ABFBDE87040FFF71EBF2146BDE840
:100D30007040FFF7F5BD2146BDE87040FFF77ABE71
:100D40002146BDE87040FFF7A7BEBDE87040FFF741
:100D500023BFBDE87040FFF7EDBE94ED000A2948BF
:100D6000FDF7B2FBE8B100201CE0274C94F8513F9E
:100D7000BBB1264904F5AC5036F08CF988B104F5C6
:100D80008053012283F8B92504F548610222A4F5B5
:100D9000804012F041FB0028E5D11D4B002283F872
:100DA000B925042070BD184C94F8513F002BF8D0A1
:100DB000164904F5AC5036F0F1F8DFE7D1ED007AD2
:100DC0009FED147AF0EEE77AF4EEC77AF1EE10FABE
:100DD00016D5D1ED017AF0EEE77AF4EEC77AF1EEAE
:100DE00010FA0DD50C490222A1F5994012F014FB1E
:100DF000B9E70A4902220348F8E709490222FAE75B
:100E00000220CFE7902B0020906B0020948B0020D5
:100E1000907B0020000000341078002058780020DB
:100E20003C78002070B5434B03F6E442D3F8203FF2
:100E300093428EB00C467BD1CD78272D28BF272535
:100E40002722002104A8B9F095FA2A4604F10C01E2
:100E500004A8B9F045FA059B9DF836400093069B1F
:100E60000193E443079B0293E4B2089B03938DF83C
:100E7000364091F0B3FB14F0810F04F0870506466D
:100E800001D1802D13D1684631F0D6FFDFED2A7AEB
:100E90002A4B20EE270ADFED2A7AC3F8346520EECC
:100EA000270ABDEEC00A10EE102AC3F8282514F058
:100EB000820F01D1802D13D1684631F0D7FFDFEDCD
:100EC0001E7A1E4B20EE270ADFED1D7AC3F8386527
:100ED00020EE270ABDEEC00A10EE102AC3F82C251A
:100EE00014F0840F01D1802D13D1684631F0CEFF6C
:100EF000DFED117A114B20EE270ADFED117AC3F8EE
:100F00003C6520EE270ABDEEC00A10EE102AC3F899
:100F1000302563060CD5DDED0C7A9FED097A074B81
:100F200067EE877A03F5A862C2ED007AC3F84465DC
:100F30000EB070BD906B0020E02E6542907B0020CB
:100F40000000C84270B51F4C90B0084602A9FEF7D9
:100F5000DDFFD4F8202F04F6E4439A4230D19DF807
:100F60003C30072B2CD104F50056D6ED067ADDED8A
:100F7000056A9FED157AF8EEE77A04F58054E6EEFF
:100F8000C77AFDEEE77AC6ED067A62F0DBFDD4F8AB
:100F9000F02FB36952689FED0D7A9B1A07EE903AD5
:100FA000F8EEE77A054667EE877A17EE900AFBF7C8
:100FB000ABFA074ACDE90001062128465BF062FF43
:100FC00010B070BD906B00200000C8420AD7233CCF
:100FD0002CF20C0810B51D4B03F6E442D3F8203F69
:100FE0009342044696B008460FD108A9FEF78EFF3B
:100FF0009DF8541003AA204661F056FF38B962F0FC
:10100000A1FD134A04215BF03DFF16B010BDBDF8F1
:10101000503023F004039BB2002BF6D0DDED0B7AA9
:101020009FED0C7A039B009367EE877A0022FDEE1A
:10103000E77A114617EE903A04A81EF0EFFA2368FB
:1010400004A9D3F8C43020469847DEE7906B00200F
:1010500040F20C080000C84230B48D7A4B7A43EA63
:101060000523CD7A43EA0543562B04460A461BD096
:1010700008D8522B12D0542B13D02046114630BC26
:1010800062F01AB803F18073863B23F07F43012B93
:10109000F3D8017C064830BC55F078BA30BCFFF775
:1010A000C1BE30BCFFF74EBF30BCFFF793BF00BFDF
:1010B0002882002000207047C82070470120704718
:1010C000002070470020704790F890308B4286BF18
:1010D00000EB8100D0F894000020704790F8903029
:1010E0008B4286BF00EB8100D0F89400002070474F
:1010F00003207047014B93F8DA017047904B0020B2
:1011000070B504464C4810F079FD18B1236A43F4D9
:1011100000032362484810F071FD88B1462065F055
:10112000D9FADFED467AB4EEE70AF1EE10FA07D805
:10113000636A43F400036362A36A43F40003A36297
:10114000236A43F4F84323623D4BD3F8200F03682E
:101150005B6898470138182815D8DFE800F03B4352
:101160000D4543434343143B3B3B3B3B3B14434311
:1011700043433B14453B3B00324A92F8E0338BB388
:1011800092F8E1238AB3304B93F8303F012B3DD0E6
:10119000022B44D02D4B1D68DDB12D4E284696F80C
:1011A0001A1C4FF0F3F8A0B1236A43F48073236252
:1011B00096F980321BB1636A43F48073636296F8D8
:1011C0001A1C28464FF01AF918B1A36A43F4807329
:1011D000A36270BDD4E9092342F4E04243F4E04342
:1011E0006262A362012300E00023616A41F480622D
:1011F0006262A26A42F48060A062002BC3D041F414
:10120000406142F440626162A262BCE7236A43F437
:1012100080032362636A43F480036362BAE7236A4C
:1012200043F480032362636A43F480036362A36A26
:1012300043F48003A362ADE7902B0020000000B4CC
:10124000906B0020905B0020907B00202491002078
:10125000904B002013B54FF44470CDE900211EF0EF
:10126000EFFD044628B1DDE9002162F089FC024B64
:101270002360204602B010BD3CF40C0800207047EB
:1012800000207047002070470020704700F508508C
:101290003C30704700487047781A0D0800F58040D0
:1012A000D0F8200F03685B681847000000F5804302
:1012B00000F59940D3F8203F1B1A58425841704717
:1012C000A22070472DE9F04100F5A04303F27453CA
:1012D00053F8042CDFED666A07EE902AB8EEE77A41
:1012E000D3ED007AF8EEE77A00F5C14890B027EE2A
:1012F000267A67EEA67A08F158080446002340468D
:101300008DED017ACDED027A03930BF08FFF04F59A
:10131000C046002800F0A680D6F80C3184330FCBED
:101320000CAF87E80F0008AD04AF87E80F0085E831
:101330000F0001A9384603AB02AA31F0C1FD9FEDB1
:101340004D0AD6F88C7301A832F00CFA29463846BB
:101350008DED080ACDED090A8DED0A1A16F064FD2F
:1013600091F03CF9D6F81032C01A632804F57C6578
:101370002DD8D6F80C0103689B689847042100F12A
:101380009402284657F0DCFBD6F80C010368DB68B2
:101390009847052100F19402284657F0D1FBD6F872
:1013A0000C0103681B699847062100F19402284646
:1013B00057F0C6FBD6F81021284602F52A720721FD
:1013C00057F0BEFB04F5C640103013F07DFC4046DC
:1013D0000DF044F990B1D6F8100188F0A5FE68B17F
:1013E000D6F810216E219032284657F0A9FBD6F886
:1013F00010216F21BC32284657F0A2FB04F542525F
:1014000004326921284657F09BFB04F547522032ED
:101410006A21284657F094FB04F5405393F92222A1
:1014200032B9D3ED867AF5EEC07AF1EE10FA06DD28
:1014300004F54D5214326B21284657F081FB04F518
:101440004E54204681F0C2F928B104F130026D21DA
:10145000284657F075FB18F0EDFB18F0FFF810B0B8
:10146000BDE8F08101A904F5965016F0A5FB77E7D9
:101470000AD7233CE02E654210B54FF48011044694
:1014800012F0B8F910B12046FFF71CFF4FF48001AD
:10149000204612F0AFF928B12EF01AFBBDE810403B
:1014A0002CF0EABC10BD000030B591B0002300F56F
:1014B0009655029302A9002304460DF1070228461F
:1014C0008DF8073018F08CF903A9284617F080F939
:1014D00008B92E4B03933022002104A8B8F04AFF2C
:1014E000A3238DF8103095238DF8113091F07EF8FC
:1014F00004F5A042CDF81300D2F87035ADF81B30DA
:1015000004F58053D2F87425CDF817104620D3F88F
:10151000B814D3F8BC34ADF81D10ADF81F20ADF8E9
:10152000213065F0D7F810EE103A1520CDF82330B1
:1015300065F0D0F810EE103ACDF8273004F53353AB
:101540009FED137AD3ED2F7A67EE877A284617EE50
:10155000903ACDF82B30029BCDF82F309DF8073014
:101560008DF83330039B0D9318F040FB04F5804356
:101570003022D3F8643F8DED0E0A04A904F57C6097
:101580000F9357F019FC11B030BD00BF2292CA7FF3
:101590000000C84230B58FB03522044600216846AD
:1015A000B8F0E8FEA3238DF8003095238DF80130C4
:1015B00001238DF8023091F019F804F5A94304F5E0
:1015C00040557833CDF803001B68D5F80406CDF8F4
:1015D0000710CDF80B3003681B699847ADF80F0072
:1015E000D5F8040603689B689847ADF811001C48BD
:1015F00002F062F8ADF81300D5F8040603685B69E1
:10160000984710EE103AD5F80406CDF81530036867
:101610009B69984710EE103A04F58041CDF81930D7
:1016200001F65C7335221B68CDF81D3004F5C0430C
:10163000D869CDF82100186ACDF825009869D3F84B
:101640003C34CDF82900CDF82D3004F57C60D1F87C
:10165000543FCDF83130694657F0AEFB0FB030BD86
:10166000902B002030B587B0162204460021684632
:10167000B8F080FEA3238DF8003095238DF801305B
:1016800002238DF8023090F0B1FF04F5A045CDF8AB
:1016900003002046CDF8071005F0B4FA05F5AC6359
:1016A0008DF80B001B680393124B1B68D86A90F8E7
:1016B0009C308DF810300368DB69984795F8493500
:1016C0008DF812308DF811002EF002FA2DF050FB3B
:1016D000D5F85C358DF813008DF81430162295F886
:1016E0004A358DF81530694604F57C6057F064FB87
:1016F00007B030BD8C2B002010B58AB027220446DD
:1017000000216846B8F036FEA3238DF800309523FB
:101710008DF8013009238DF8023090F067FFCDF885
:1017200003000420CDF8071064F0D4FF10EE103A47
:101730001320CDF80B3064F0CDFF10EE103A4620A8
:10174000CDF80F3064F0C6FF10EE103A1520CDF83A
:10175000133064F0BFFF10EE103A0320CDF81730BD
:1017600064F0C8FF10EE103A1A20CDF81B3064F078
:10177000B1FF10EE103ACDF81F3004F59E437033E0
:1017800027221B68CDF82330694604F57C6057F0AA
:1017900013FB0AB010BD000013B5044600F57C60D1
:1017A000019056F03BFE019856F0D2FE04F58053AE
:1017B000019893F9D4300BB156F072FF204602B075
:1017C000BDE81040FFF798BF7047000030B500F546
:1017D000C04389B093F8EC21044600F57C6552B112
:1017E000D3F804011E2269468AF0CEFD0F496A46ED
:1017F000284657F07DFC04F58043D3F8200F03689A
:101800005B68984704F50053014693F85C2128462D
:1018100057F092FC04F5965018F086FC04F5907091
:1018200009B0BDE8304026F0BDBC00BF48F50C084B
:101830009FED020A00224CF095BE00BF0AD7233C60
:10184000134B70B5044640F8043B63F09DFA114E0B
:10185000114B63605425601963F04CFC66513035C0
:10186000B5F5557FF7D104F5557065F029FB0B4AA6
:1018700004F5EC6002F63C318DF0EEFD01232046CC
:10188000074984F891394DF06BFA204670BD00BFCE
:10189000D0370020BC450D08D0450D082C4D002048
:1018A00090350D082DE9F04100F507519AB00D2251
:1018B0001831044655F09EFE0022C04827214CF006
:1018C000C9FD0421002065F085FA1321012065F08F
:1018D00081FA4621022065F07DFA1521032065F08A
:1018E00079FA65F047F804F5C04393F9A43123B1C0
:1018F0009FEDB30AB3484DF0DBFD4DF037FCB24A23
:10190000B24E138843F0040313804FF000080AAF6F
:10191000002110223846B8F02DFD01238DF830301B
:101920003388ADF8283005A973680B9338464CF01E
:1019300099FCC8B19DF91430002B15DD63F0A4FBB0
:101940009DF81410036801391B68C9B2984758B153
:10195000051D28464CF024FC30B9B368ADF81830AA
:1019600006A928464EF0BEF808F10608B8F12A0F7D
:1019700006F10C06CCD1964800220DF10B014CF07B
:10198000F7F906AD064620B34CF00AFC08BB914BB4
:101990000FCB85E80F0004A928464CF063FC002813
:1019A00040F03B814FF004088B4B0FCB87E80F00D2
:1019B00005A938464CF056FC28B105A84CF0F0FBC0
:1019C00008B148F0010803A930468DF80C804EF0AC
:1019D00037F8824B0FCB85E80F0003A928464CF05F
:1019E00041FC002846D00998002204A94CF0C0F917
:1019F000064600283ED04CF0D3FB0546002839D1DE
:101A00009DF80C30013BDBB2032B96BF744A0346B2
:101A1000D35C8DF82830304639464EF011F87148C5
:101A2000002205A94CF0A4F906466DF009FE78B134
:101A30006DF004FE90F8302090F8281090F84830AF
:101A4000114490F840200A44D34214BF01250025D8
:101A500086B130469DF90C804CF0A2FB50B91DB107
:101A6000B8F1000518BF0125394630468DF82850D9
:101A70004DF0E6FF04F509500022B7EE000A0121FF
:101A800034304CF06FFD04F508500022B7EE000A28
:101A9000022110304CF066FD012304F5F75100934C
:101AA000514A002308318E204CF0D8FC94F974C9B7
:101AB000BCF1000F1AD14D4E0FCE3D460FC50FCED3
:101AC0000FC50FCE0FC596E80F0085E80F006246E0
:101AD000042138464CF0BEFC9FED450A45484DF0C8
:101AE000E7FC4548B7EE000A4DF0E2FC012504F59D
:101AF0000251424A00950023203140F205104CF07B
:101B0000ADFC04F5095002210430FFF791FE04F505
:101B1000065003212C30FFF78BFE04F506500321FD
:101B20003430FFF785FE032104F50950FFF780FEEE
:101B300004F5095002210830FFF77AFE022104F56E
:101B40000750FFF775FE04F5075002210430FFF738
:101B50006FFE04F5065002213C30FFF769FE04F5E4
:101B6000BE4034308CF080FF254A1368D90705D475
:101B70002449156004F5015308330B6004F50A503D
:101B800020490122083001254CF0BAFC1E4A00957C
:101B9000002304F57C61FD204CF060FC1B4B1A68AF
:101BA000D20705D41A4A1D6004F58F540834146016
:101BB000174801214CF0C0FC2CE000BFCC320D08CE
:101BC0000000964324200E08089100203C350D08A3
:101BD00090320D08F8E50C0808E60C0818E60C0829
:101BE000C8320D089B320D0824770D0828E60C0832
:101BF00000000000A8320D08B7320D08A4850E08B9
:101C0000842B00200022002068060E08882B00206C
:101C10000C2200201AB0BDE8F08104A84CF0C0FAF4
:101C200000283FF4BFAE4FF00C08BDE6704700003F
:101C30000020704700207047002070470020704748
:101C40000020704770470000002070470020704758
:101C500084B001A880E80E0004B0002070470000A6
:101C60000020704700207047704700001020704728
:101C700000487047B8410D0800487047C8410D083A
:101C80000020704770470000012070470120704716
:101C900000207047002343608360C3600361436199
:101CA000002303767047000010B50446FFF7F2FFEB
:101CB0000023637610BD0000027E531CDBB2042BB0
:101CC000037600EB820288BF002382ED010A88BF01
:101CD0000376704710B50446FFF7EEFFD4ED017AA6
:101CE0009FED107A94ED020A637E77EE877A042BDB
:101CF00077EE807A94ED030A94BF0133052377EEE3
:101D0000807A94ED040A637677EE807A637E94EDB0
:101D1000050A77EE807A00EE103AB8EEC00A87EE38
:101D2000800A10BD0000000010B504461EF090F8B7
:101D3000204610BD04F080BC03F098BA04F060B8EF
:101D400003F0A0BA01F0B8BF01F016BB01F09EBCD1
:101D500001F0DEBCFCF7A0BFFCF748BB70B51F4B21
:101D6000036000F540530446D3F898051C4AC3F8B5
:101D7000E82308B11EF070F81A4B236004F5805375
:101D800093F8842E42B9D3F8805E2DB128462BF00B
:101D9000FBF828461EF05CF804F58E500C307DF000
:101DA0008DFE04F58650143066F08AF904F6C445B9
:101DB00004F66446B54204D0183D28462AF038FDA2
:101DC000F8E7094BC4F8983804F694105AF084F9EF
:101DD00004F510605AF080F9204670BD10290D08F6
:101DE00038210E084CFF0D08FCC40D0838B5474BD0
:101DF000044640F8043B66F0A9FC04F110001BF017
:101E00008DFA04F1680053F057FB04F5907025F04B
:101E1000ABFD04F586601AF0E9F804F254501EF0A8
:101E20001DF804F698002CF013F904F5446066F0F0
:101E30006BFA04F551604EF0CFF904F57C6056F072
:101E4000EFFE04F58650143066F022F904F5885050
:101E500010301CF077FD04F58E500C307DF01AFE2A
:101E600004F58F50083053F0E9FE04F591501C3012
:101E700067F04AFE04F5805304F59352002510469E
:101E800083F86052224B10301A6049F0B5FD2946A4
:101E900004F5965016F07EF904F5C850103076F02F
:101EA000F5FC04F5E85014307AF03AFE04F5F150F0
:101EB0000C307CF049FF04F5F45010307DF07EFBCF
:101EC00004F5F750083015F087F804F50150083094
:101ED00077F03AF904F5025020306CF087FE04F5F3
:101EE000005304F5055083F85C510A4D34307EF000
:101EF000A5F92B6813B1084890F03EFB204607492E
:101F00004CF02EFF2C60204638BD00BF4CFF0D0862
:101F1000FC9900205C910020D0410D0874FE0D0852
:101F20002DE9F04F2DED028B04469FB0FFF75EFFC9
:101F3000E24B236004F50A500830FFF781FC04F5FA
:101F40003050203004F500577FF0CCFC04F50853E6
:101F50002233C7F8483C04F53150062387F84C3C3F
:101F6000343065F0A7FC04F5BE433433C7F8F03CC9
:101F70000E934FF40063C7F8F43C5A2387F8743D7E
:101F800004F5065807F6D84308F11C08CC4AC7F8F0
:101F9000EC8C04F5965BC7F8E8BCC3F86021C94A2D
:101FA000C3F86421B7EE008AC74AC3F8682104F574
:101FB0003A50C3F8CC2183ED578A34305AF0ACFB49
:101FC00004F5335A04F53B505AF0A6FB0026BF4BEC
:101FD000C7F8D03E0AF1180A87F8E86E0AF5FC70D7
:101FE000FFF758FEBA4BBB49C7F8D03E87F8E96EF9
:101FF00050464CF0B5FEB84BC7F8F03E07F56F639E
:102000000022C7F8F4BEC7F8F8AE04F53B555A6392
:10201000DA6304F53D50012387F8343F303508304A
:102020001DF0DCFA87F8586FAC4928464CF098FE52
:1020300004F53D5041461C3080F00AF804F542504A
:10204000414634307FF068FC04F54850414604F5C1
:1020500040570C3080F0C6FB2C22314607F56C70DF
:10206000B8F088F904F54F569D4904F54E504CF0F0
:1020700077FE28369B4BC7F8E83306F108008FF04F
:10208000E9F904F5505904F5515309F114093833AD
:1020900048460F935FF054F80F9B09F114094B4524
:1020A000F6D10723C7F89C350023A7F8A0354FF4D5
:1020B000CB701DF0CBFEC7F8980504F556502430C0
:1020C0008FF0C8F904F5575028308FF0C3F9864BCC
:1020D0001A6802B91E60854BC7F8E83304F55850FA
:1020E0004FF48051C7F8045608301BF013FA04F57A
:1020F0005A5008304DF0ACFD04F55A501C306EF0CB
:102100001BFE04F5964004F58045743005F0CCF9CB
:10211000774BC5F8743B04F59740103005F0C4F9CF
:10212000744BC5F8903B04F597402C3005F0BCF992
:10213000714BC5F8AC3B04F59740483005F0B4F955
:102140006E4BC5F8C83B05F53F63002204F5984087
:10215000DA609A605A6083ED008A043005F0A4F9D1
:10216000674BC5F8043C04F59840203005F09CF915
:10217000644BC5F8203C04F598403C3005F094F9D8
:10218000614BC5F83C3C04F59840643005F08CF98F
:102190005E4BC5F8643C04F5994005F085F95C4B4D
:1021A000C5F8803C04F599402C3005F07DF9594B79
:1021B000C5F8AC3C04F59940483005F075F9564B2C
:1021C000C5F8C83C04F59940643004F59A4605F01A
:1021D0006BF90436514BC5F8E43C304605F064F920
:1021E0004F4BC5F8043D04F59A40203005F05CF9EA
:1021F0004C4BC5F8203D04F59A403C3005F054F9AD
:10220000494BC5F83C3D04F59A40583005F04CF96F
:10221000464BC5F8583D04F59A40743005F044F932
:10222000434BC5F8743D04F59B40143005F03CF970
:10223000404BC5F8943D04F59B40303005F034F92F
:102240003D4BC5F8B03D04F59B40503005F02CF9EE
:102250003A4BC5F8D03D04F59B406C3005F024F9AD
:10226000374BC5F8EC3D04F59C40083008F0A2F966
:1022700004F59C40443005F017F9324BC5F8443E54
:10228000314BC5F8603E04F59C404FF4C053A5F8AF
:10229000B43E2E4960304CF063FDFE2385F82C3FA0
:1022A000052385F8503F4FF0FF33C5F8583F284BC2
:1022B000C5F8206FC5F8246F11934BE010290D0865
:1022C000000080BF0000B4420000B4C208420D0804
:1022D00018420D08DCBF0E083CBD0E08E4BC0E0819
:1022E0003CBB0E0838210E087894002010F50C082D
:1022F000704D0D086C540D088C570D086C4B0D0873
:10230000804E0D08084F0D08E84D0D08F04C0D08E3
:102310006C4C0D08FC530D08F84F0D08884F0D0844
:1023200050420D0878500D0884530D0878510D085F
:1023300068520D08E8510D0800530D08F8500D08BB
:10234000FC4A0D0808570D0840420D089CE00E0895
:10235000351D010805F577658F4B85ED008A04F57D
:102360009E4004F5A0454FF40071009322468B4B2C
:10237000109474301AF03AFB4FF0FF33C5F8D034A4
:1023800005F59C63864ADA6003230026C5F85C35B0
:1023900005F5AF63C5F82865C5F82C65C5F8306547
:1023A000C5F83465C5F83865C5F83C6583ED008A25
:1023B0007C4BC5F8A03504F5AB497B4BC5F8A83577
:1023C00048467A4BC5F8B035C5F89C45C5F8A445D4
:1023D000C5F8AC4544301DF001F9484660301DF0A9
:1023E000FDF848467C301DF0F9F8714BC5F8103601
:1023F0004FF0FF33A5F8143609F198001DF0EEF800
:102400004FF0FF326B4BC5F874266B49C3F8009050
:1024100048464CF0A5FC4FF6FF73A5F8BC354FF0CD
:10242000FF33A5F8D83504F5AC40644B64497830E7
:1024300018604CF095FC04F5AD40183054F0CEFC1B
:10244000604BD7F804261294CDE913345E4BCDE9E6
:1024500015345E4BCDE917345D4BCDE919345D4B36
:10246000CDE91B345C4B1D931EA911E903000CAB95
:1024700083E80300DDE91A010AAB83E80300DDE924
:10248000180108AB83E80300DDE9160106AB83E819
:102490000300DDE9140104AB83E80300DDE9120168
:1024A00002AB83E803004946CDE9002853465A466B
:1024B0000E988CF0E3F80BF51B7304F5BF40C5F8DC
:1024C000F03F74301DF08AF804F5C04004301DF070
:1024D00085F804F5C04004F5C047143004F5C14840
:1024E0001DF07CF808F110081C22314607F1240089
:1024F000B7F040FF40467DF05BFF384B3849C7F8E6
:10250000903040464CF02CFC364A3749116004F5B7
:10251000C14348334FF0140CB0B20CFB001201362B
:10252000127C002AF8D1314A1080314A166816B15F
:10253000304890F021F804F5C1404C3013607DF034
:1025400021FF2D4BC7F8CC3004F5C1405946583017
:1025500009F05EFB294BC7F8D033642387F8D433E6
:10256000274BC7F8083404F5C740264BC7F80C348E
:10257000254950304CF0F4FB244BC7F8D0332046AB
:102580000123C7F8306487F8386485F810351FB028
:10259000BDEC028BBDE8F08FF0F10C08351D010891
:1025A0000000B442391D01083D1D0108411D01080C
:1025B0000000FFFF5090002034D30D08009A002047
:1025C000542F0E08451D0108491D01084D1D010825
:1025D000511D0108551D0108591D0108C0EB0C08CB
:1025E00098EB0C081891002040370D081691002038
:1025F000D4900020E4410D0800EC0C0828420D089E
:1026000078730D08D0730D0830280E0850750D082A
:1026100010B58FF0EDFA064C064B18602046FFF718
:102620007FFC2046044A0549BDE81040B5F060B97A
:10263000902B00208C2B002020F200205D1D010833
:102640000069C0F3401070470F299DBF302303FB82
:102650000100503000207047014B93F92102704770
:10266000904B0020014BD3F8340C7047904B002066
:1026700008B503689B68984730B9044B93F83A0F44
:10268000B0FA80F0400908BD0020FCE7906B002004
:1026900008B504480FF022F810B9034B93F8340F33
:1026A00008BD00BF902B0020906B0020022A10B5BF
:1026B0000C4605D1BDE810400948352210F084BF12
:1026C000084BD3F8200F03685B689847A04205D1F8
:1026D00062F0DAFCBDE8104062F060BC10BD00BFE3
:1026E000902B0020906B0020012910B50C4610D0D3
:1026F000022904D061B961F025FA084A02E061F0CC
:1027000021FA074A06215AF0BDFB064BC3F8704177
:1027100010BD61F017FA044AF4E700BF68430D08E2
:1027200040430D08908B002057430D08012910B538
:102730000C4614D0022907D0D1B90E4BC3F830147F
:1027400061F000FA0C4A05E00A4BC3F8301461F05E
:10275000F9F90A4ABDE8104006215AF093BB61F02E
:10276000F1F9074A06215AF08DFB024BC3F83044B9
:1027700010BD00BF908B0020A7430D087C430D08BF
:1027800090430D08012903D0022914BF0021022122
:10279000014BC3F8D41B7047904B0020012902D095
:1027A000022900D011B9024BC3F83414704700BF9E
:1027B000908B00206C2910B400F3A6803F290FDC19
:1027C000162900F39980032940F39A807E4B012457
:1027D0008C402340002B00F093805DF8044B704741
:1027E000A1F140032C2B00F28B8001A454F823F0BC
:1027F000A929010801290108012901080129010865
:1028000001290108012901080129010801290108FC
:10281000DB27010801290108012901080129010814
:1028200001290108DB270108012901080129010804
:1028300001290108012901089F290108012901082E
:102840009F290108012901089F2901089F290108E2
:102850009F290108DB270108012901089F29010898
:10286000DB2701080129010801290108DB270108EC
:10287000DB27010801290108DB27010801290108DC
:10288000012901080129010801290108012901087C
:10289000012901080129010801290108DB27010894
:1028A000DB270108112B2BD801A454F823F000BF1B
:1028B000DB27010801290108012901080129010874
:1028C000DB27010801290108012901080129010864
:1028D000012901080129010801290108012901082C
:1028E000DB270108DB27010801290108012901086C
:1028F000DB270108DB270108A1F12703112BD1D920
:102900005DF8044B63F0D2B9A0291FDC9529F7DDEF
:10291000A1F196030A2BF3D801A454F823F000BFC9
:10292000DB27010801290108012901080129010803
:10293000DB270108DB27010801290108DB27010843
:1029400001290108012901089F290108B52921DC75
:10295000A929D5DDA1F1AA030B2BD1D801A454F8E4
:1029600023F000BFDB270108012901080129010824
:10297000DB2701080129010801290108DB270108DB
:10298000012901080129010801290108012901087B
:10299000DB270108A1F1D003022BB1D81DE75DF8B8
:1029A000044B002363F054B9084B012283F82C2414
:1029B000A3F58043D3F8300C00283FF40EAF5DF848
:1029C000044B642162F0A6BB10004100908B0020F4
:1029D0006C2938B50346154600F3A2803F2912DC66
:1029E00038290ADC26296FDC102900F00581162918
:1029F00000F08A81042900F016812A461846BDE8B5
:102A0000384062F01BBFA1F140022C2AF5D801A08A
:102A100050F822F0D12B0108FB290108FB290108FD
:102A2000FB290108FB290108FB290108FB290108F2
:102A3000FB290108012C0108FB290108FB290108D9
:102A4000FB290108FB2901082B2C0108FB2901089F
:102A5000FB290108FB290108FB290108732C010847
:102A6000FB290108C72C0108FB2901087D2C01085E
:102A7000BD2C0108692C0108FF2C0108FB29010865
:102A8000E72C0108312C0108FB290108FB2901086A
:102A9000BF2B0108172D0108FB2901080F2C010885
:102AA000FB290108FB290108FB290108FB29010872
:102AB000FB290108FB290108FB290108FB29010862
:102AC0009F2D0108372C0108A1F12702112A94D863
:102AD00001A050F822F000BFBF2B0108FB2901081C
:102AE000FB290108FB290108C32B0108FB29010868
:102AF000FB290108FB290108FB290108FB29010822
:102B0000FB290108FB290108212C0108092C0108D7
:102B1000FB290108FB2901081B2C0108152C0108C1
:102B2000A02921DC95297FF768AFA1F196020A2A36
:102B30003FF663AF01A050F822F000BF212D01083D
:102B4000FB290108FB290108FB290108272D0108A1
:102B5000792D0108FB290108872D0108FB290108AF
:102B6000FB290108472D0108B52923DCA9297FF796
:102B700044AFA1F1AA020B2A3FF63FAF01A050F8E3
:102B800022F000BF3D2C0108FB290108FB290108A8
:102B9000672D0108FB290108FB290108432C0108C6
:102BA000FB290108FB290108FB290108FB29010871
:102BB000BF2D0108A1F1D002022A3FF61EAF012469
:102BC0008FE0A91E864B4D424D4183F82D5FF6E7FD
:102BD000AA1E5542834C554184F82B5460F0B2FF35
:102BE000814A94F82B14814B002908BF1346804A70
:102BF00006215AF047F9E2E70A21FFF757FDDEE721
:102C00002A4601211846F8E72A460421FAE72A460F
:102C10000321F7E72A460C21F4E72A460F21F1E7C2
:102C20002A460021EEE70B21E7E72A460D21E9E7D6
:102C30002A460521E6E72A461521E3E72A4611211F
:102C4000E0E7AB1E5A425A41664B93F8D0119142CD
:102C5000B5D083F8D02160F075FF664A664B022D2F
:102C600008BF1346654AC3E729461846FFF78AFDA1
:102C7000A5E729461846FFF737FDA0E7594CD5B11F
:102C8000022D0DD1012384F82834A4F50053D3F884
:102C9000200F03685B6A984710B1594800F09EFF07
:102CA00060F050FF534A94F82814534B002908BF92
:102CB0001346544A9CE784F82854E6E72946184608
:102CC000FFF734FD7BE7012445B1022D09D1454BC7
:102CD000C3F82841002283F8182202E0414BC3F8D0
:102CE0002851204638BD01242DB1022DF9D1464B83
:102CF00083F83440F5E7444B83F83450F1E7294634
:102D00001846FFF74BFD5AE7022A7FF458AF3C48BC
:102D100008F0B6FD53E762F0B7F962F03FF94EE70D
:102D20002A4607216EE71846294662F0B7FC374865
:102D30007DF07EFB044600283FF441AF294B012281
:102D4000C3F82821C6E7274BD3F8E831002B3FF41E
:102D500036AF012425B1022DC3D183F82C40C0E742
:102D600083F82C50BDE7022D7FF429AF9FED280A90
:102D70002348FBF7A9FB22E7022D7FF420AF204870
:102D80000EF0BAFB1BE701242DB1022DA9D1154B82
:102D900083F82A44A5E7134B83F82A54A1E7022DB0
:102DA00012D10F4DD5F8200F0368DB6B984704460E
:102DB00078B10121A5F5804003F05CF991E7154851
:102DC00029468DF0D9FCFAE60D48002103F052F9AE
:102DD000F5E660F0B7FE104A04215AF053F8EEE62B
:102DE000906B0020908B0020BC430D08A32B0D0896
:102DF000C4430D08B3150D08D8540D08D4430D086D
:102E0000902B0020E0430D08904B0020208C0020E8
:102E100000000000F0790020F3430D0810B599B1CF
:102E200004681168416004B90160126801681B6898
:102E3000521A9A4202D80021084610BD017A012395
:102E400081F001010372F7E7037A3BB144682CB1CA
:102E50001368029A12681B1B9342ECD90023C0E945
:102E60000033EFE70023C0E90533C0E90833838569
:102E7000037780F828307047F0B52DED028B0446BB
:102E800087B09F48B0EE408A0E467DF0DBFA40B135
:102E9000236933B1206B00F50E7010F08FFE0546EC
:102EA00038B12046FFF7DEFF002007B0BDEC028BF3
:102EB000F0BD236B93F93C22002A1EDD93F8A0326B
:102EC000DBB1904BD3F83424002AEAD12369D4ED46
:102ED000007A991E4842F5EEC07A4841F1EE10FAA8
:102EE00084F82C0027D8C4E90822C4E9052284F814
:102EF0002D2084F828202277D7E7834FD7F8200F9A
:102F000003689B6B984728B107F5805797F85835A9
:102F1000002BD6D07D4800210EF076FEDFED7C7AC6
:102F2000B4EEE70AF1EE10FACBDA784803F06AFE65
:102F30000028C6D1B5E76EB1F4EEC87AF1EE10FA0A
:102F40003CDD236BD3F8C432DB0403D5714815F0A4
:102F5000EFFB064684F82D608FF040FBD4ED027A3B
:102F60009FED6D7A039067EE877AFCEEE77A17EEB5
:102F7000903A5B000593B4F90630CDED047A002B4E
:102F80001EDC0023C4E9083384F8283094F90430A7
:102F9000002B41DC0023C4E90533237794F82C008F
:102FA000002882D194F82D0000287FF47EAF94F899
:102FB000280000287FF479AF207F76E71646C9E71E
:102FC0000421524800F0B4FCB4F9063007EE903A00
:102FD000F8EEE77A05ABF4EEC07AF1EE10FA009362
:102FE000CCBF0121002104AB03AA04F12000B0EE04
:102FF000408AFFF713FF0028C8D060F0A3FD064603
:1030000018EE100AF9F780FA444ACDE900010421CC
:10301000304659F037FFB9E7414E9FED427AD6F876
:10302000B824DFED416A06F58051D1ED6F7A82EA6E
:10303000E270B0EE476AA0EBE270A7EEA66A07EE78
:10304000900AF8EEE77AF4EEC67AF1EE10FA53D869
:10305000D6F8BC0491ED706A07EE900AA6EE267AC7
:10306000F8EEE77AF4EEC77AF1EE10FA44D591ED76
:10307000716A9FED2E7AA6EE267AF4EEC77AF1EE0B
:1030800010FACCBF01270027642113FB01F1284B64
:10309000D3F87005121A002AB8BF52428A422DDABC
:1030A000D6F8BC24D3F87435D31A002BB8BF5B42D2
:1030B0008B42ACBF0023012304F114000FB983F04D
:1030C000010505AB009303AA04AB2946FFF7A6FE52
:1030D00000283FF463AF60F035FDD6F8B814D6F899
:1030E000BC24642392FBF3F291FBF3F300920421DE
:1030F000104A59F0C7FE51E70027C5E70023DBE778
:10310000208C0020908B0020906B0020902B0020C2
:1031100000000034503E002000007A44EC450D08C9
:10312000903B00200000FA430000C8420000FAC3B0
:10313000907B0020FD450D0873B58289036BD20793
:1031400004466CD493F93C22002A03DD93F8A022B4
:10315000002A64D1524DD5F8201F05F55D629142D9
:103160005DD0A5F54055B3F90860D5F8B83407EE41
:10317000903AD5F8BC34B8EEE77A07EE903AF8EE1C
:10318000E77A6846CDED017A8DED007A30F0B8F936
:10319000730007EE903AF8EEE77AB0EEC00AF4EE6C
:1031A000C07AF1EE10FA42D4236B93F8F1223AB3CD
:1031B00007EE906AF8EEE77AF4EEC07AF1EE10FAD4
:1031C0001EDB002183F8F112236B586B85F0A8FEFB
:1031D000236B9FED347ADA6BD2ED067A05F2C46286
:1031E00067EE877A92ED007AF4EEC77AF1EE10FA84
:1031F00006D5986B88F0F4F8236B986B87F08AFEFD
:10320000A389226B13F0020302D192F8F11299B94B
:10321000002382F8F232236B93F8F10205E00020DC
:1032200083F8F102236B83F8F20202B070BD236BC6
:10323000012283F8F122B7E705F2DC51D1ED007AE3
:103240009FED197AF0EEE76AF4EEC76AF1EE10FA34
:10325000DFDD05F2D451D1ED006A9FED146AB0EEC6
:10326000E67AB4EEC67AF1EE10FAD2DD05F5BB616E
:1032700091ED007AB0EEC77AB4EEC67AF1EE10FAAC
:10328000C7DD67EEA67AF5EEC07AF1EE10FAC0D58A
:10329000D5F8BC3406498B42ACBF00230123B8E704
:1032A000906B00200AD7233CC2B8323E920A063FF8
:1032B0006CEEFFFF08B5036B93F8F2223AB1DA6ABD
:1032C00092F8A020022A03D0002283F8F22208BD3F
:1032D0000B4B9FED0C0AD3ED007AF5EEC07ADFEDD3
:1032E0000A7AF1EE10FAD8BFB0EE670A152063F043
:1032F000DDF9BDE808409FED050A132063F0D6B95B
:103300006C41002000A08CC500A08C45000000008E
:1033100000F58040D0F8200F03681B6C18470000B0
:1033200000F5005393ED907AB5EEC07AF1EE10FA05
:1033300003D500F5C0408068704700F5A040DFED80
:10334000076AD0F8F03FD3ED017AF8EEE77AE7EEBE
:10335000267AFDEEE77A17EE900A70470000C84221
:1033600000F5005090F8800228B141F001010842B8
:1033700014BF01200020704710B54B68516800F55C
:10338000C0448B42D8BF0A46606ACCBF1A46194671
:103390002DF07AF9606210BD10B5044650486BF00C
:1033A00081FD10F0080117BF4E4BDFED4F7A93ED12
:1033B0002B7AD3ED2D7A1FBF77EE877A9FED4B7A6C
:1033C000012167EE877A10F0010317BF454B9FED8F
:1033D000467AD3ED2D6A93ED2A7A1CBF37EE667AD2
:1033E000DFED426A04F5005218BF27EE267AD2EDCF
:1033F000926AF5EEC06A18BF0123F1EE10FA34DDCF
:10340000384A9FED3A6AD2ED926A66EE866A0121E9
:10341000F4EE676AF1EE10FA58BFF0EE667A04F542
:10342000C04292F82C0028B373B1D2ED0C6AF8EECA
:10343000E66AF4EEC76AF1EE10FA58BFF0EE476A9A
:10344000FDEEE66AC2ED0C6A99B192ED0C7AB8EE27
:10345000C77AB4EEE77AF1EE10FAD8BFB0EE677A29
:10346000BDEEC77A82ED0C7A03E00029D7D1002B9C
:10347000D5D110BDC3B104F5A043D3F8F03FD3EDCF
:10348000016AF8EEE66A76EE876A92ED097AB8EE9E
:10349000C77AF4EEC76AF1EE10FAD8BFB0EE667ADA
:1034A000BDEEC77A82ED097A0029E2D004F5A04486
:1034B000D4F8F03F93ED017AB8EEC77A77EE277A29
:1034C00092ED097AB8EEC77AF4EEC77AF1EE10FA07
:1034D00058BFB0EE677ABDEEC77A82ED097AC8E7C9
:1034E000304C0020904B0020000000000000C8423B
:1034F00000F5C040002383627047000073B5164694
:10350000044600236A46304600931CF055F948B142
:10351000DDED007A9FED267A67EE877AFDEEE77A99
:1035200017EE900A04F5C045A86233785B0718D5FA
:1035300095F82C30ABB104F5AD40012201A918304B
:1035400053F0D2FD68B1D5ED0C7ADDED016A9FED47
:10355000187AF8EEE77AE6EEC77AFDEEE77AC5ED7F
:103560000A7A04F5A043D3F85C35042B1DD004F58A
:103570000054B4F97A22002A15DDAB6A9FED0D7A6A
:1035800083EAE371A1EBE37107EE901AF8EEE77AB4
:1035900067EE877A07EE102AB8EEC77AF4EEC77A9C
:1035A000F1EE10FA01D50023AB6202B070BD00BF8E
:1035B0000000C8420AD7233C37B50B780D4659079F
:1035C00004461DD500F5AD40012201A9183053F085
:1035D0008BFDA8B1D5ED017A2B78DFED1B6AF8EEF3
:1035E000E77ADA0767EEA67A18D59DED017AB4EE90
:1035F000E77AF1EE10FACCBF0120002003B030BD15
:103600002B78D5ED017ADB07F8EEE77A11D404F5D3
:10361000C04494ED027AB8EEC77AE8E704F5A04416
:10362000D4F8F03F93ED017AB8EEC77AE7EE667A08
:10363000DBE704F5A043D3F8F03F93ED017AB8EE51
:10364000C77A77EE877AE2E70AD7233C00F5005382
:1036500000F58042B3F92A32D2F8202F00EE103A5A
:1036600000F599439A42B8EEC00A0ED100F5A04089
:10367000D0F85C35042B02D090F811352BB100F650
:103680003470D0ED007A30EE270A7047014608B555
:1036900001F5C041FFF7DAFFD1ED027A9FED057A1F
:1036A000F8EEE77AE0EE477AFDEEE77A17EE900A59
:1036B00008BD00BF0000C84237B500F5C04504464C
:1036C00095F82C30DBB100F5AD40012201A918308E
:1036D00053F00AFD98B1D5ED0C7AD5ED0D6A9FED4A
:1036E0000B7AF8EEE77AE6EE877ADDED016AE6EE30
:1036F000C77AFDEEE77A17EE900A03B030BD204698
:10370000FFF7C4FF6B6A181AF7E700BF0000C84252
:10371000014608B5FFF79AFF01F5C041D1ED107AD7
:1037200037EEC00ADFED047A20EE270AFDEEC07AFC
:1037300017EE900A08BD00BF0000C8422DE9F04115
:1037400000F5C04800F5C04508F1040814350446EA
:10375000294640461CF0A4FA04F5A04704F5BF46EC
:1037600007F59F6374362A46314683ED000A4046CA
:103770001CF0CCF907F2FC47DFED220A87ED000AC6
:10378000B7EE001A76202CF0DFFE04F5335383EDFC
:10379000770A2046FAF72AFE04F58043D3F8200F73
:1037A00003685B6898470B280CD007D80A2810D00C
:1037B00004F5C0440023A362BDE8F0810E38C0B216
:1037C0000128F5D829462046FFF7F6FE0028EFD05D
:1037D00011E029462046FFF7EFFE30B90A484FF4C2
:1037E0008041FBF73DF90028E2D12046FFF790FF2A
:1037F000B0F5FA6FE6DD2A4631462046BDE8F041D5
:10380000FFF77CBE00000000902B002010B52DEDCE
:10381000028B00F5C043D3ED067A1B7DDFED1C8AD9
:10382000B8EEE78ADA0728EE288A82B0044609D47F
:1038300000F5805202F5A662D2ED007AF8EEE77A42
:10384000A7EEE88A5B070FD504F5AD40012201A978
:10385000183053F049FC38B19DED010A30EE480AAA
:1038600002B0BDEC028B10BD204604F58054FFF77A
:103870000DFF04F5A66393ED000A07EE900AB8EE7B
:10388000C00AF8EEE77A28EEC00AA7EEA80AE5E734
:103890000AD7233C73B504461646FFF761FD78B995
:1038A00066BB04F5C145583528460AF00BFDB8B390
:1038B00028460AF0AFF898BB2046FFF7A7FF09E0BB
:1038C00004F5005595F8503CDB0705D505F66C4529
:1038D00095ED000A02B070BD04F5C14058300AF001
:1038E00017FD0028DCD095F81A1C04F551604CF047
:1038F00043FD0228D4D19FED0D0AEBE704F5A04368
:1039000093F8303F022BCCD104F5AD40012201A940
:10391000183053F0E9FB0028C3D09DED010AD9E728
:1039200004F5C04494ED100AD4E700BF0000000085
:1039300000F5C04393F82C20FFF7ACBF38B52DED50
:10394000028B00F5804200F59843D2F8202F2033F7
:103950009A4204464CD100F58053D3F8C05400F588
:103960000053B3F97832002B65DD04F5B65292EDC1
:10397000017AF7EE007AB4EEE77AF1EE10FA5AD453
:1039800004F53452D2ED007AF6EE006A67EEA67ABC
:1039900087EE871AB5EEC01AF1EE10FA4BD907EE92
:1039A000905A9FED278AB8EEE70A07EE903A04F5A1
:1039B000AD4004F5C044F8EEE70A20EE080A1830DE
:1039C00053F09EFCA36A9FED1F1ADFED1F0A002B28
:1039D000BCBF07EE903AF8EEE77A4FF42970B8BF13
:1039E000A7EE880ABDEC028BBDE838402CF0ACBDD8
:1039F00007F0BEFDF8B904F54053D3F80406036898
:103A00001B69984704F50053DFED0F0AB3F97832CC
:103A100001EE103A04F5A94393ED1E0AB8EEC11A5F
:103A2000054640F27F202CF08FFDBDEEC00A10EE5F
:103A3000103A1BB297E7BDEC028B9FED030A38BD2D
:103A40000AD7233C00007A440000000010B5044669
:103A50008EF0C4FD04F50053D3F8642C801A41F2B3
:103A6000883290420FD802212046FFF779FC50B1EE
:103A700004F5A044D4F85C25042A04D103F6584385
:103A800093ED000A10BD9FED010AFBE70000000066
:103A900030B52DED028B00F5C045DFED278A95F896
:103AA0002C3083B004465BB3D5ED0C7A9FED230A2E
:103AB000F8EEE77A00F5AD4027EE800A012201A971
:103AC000183053F049FBD8B12046FFF737FFDDED42
:103AD000017A85ED0D0A37EE800A20468DED010A48
:103AE000FFF7B4FFDDED017A30EE270A20EE280A59
:103AF000BDEEC00A10EE100A03B0BDEC028B30BD63
:103B000004F5A0432046D3F8F02F6B6A52689B1A45
:103B100008EE103AFFF79AFDB8EEC88A2046A0EEEC
:103B2000288AFFF793FFBDEEC88AB8EEC88AA0EED8
:103B3000288ABDEEC80ADDE70000C8420AD7233C48
:103B400010B500F580430446D3F8200F03685B6A84
:103B5000984718B104F5C04494F8280410BD00003B
:103B600038B500F5C0440D46636A0B44636294F8AF
:103B70002C302BB1FFF7E4FF10B9216B29442163EE
:103B800038BD000030B500F50050D0F87422D307DE
:103B90000FD4094B0B201D785C688D4204D1224262
:103BA00014BF0120002030BD013803F10803F2D119
:103BB000F9E70120F7E700BF54460D0810B500F5FE
:103BC00080430446D3F8200F03685B68984701469A
:103BD0002046BDE81040FFF7D5BF000037B500F51F
:103BE000C0440546A36863620023A362FFF7E6FFB3
:103BF000D0B105F5AD40012201A9183053F074FA97
:103C000090B12846FFF79CFF70B9DDED017A9FED7A
:103C1000087A67EE877A0123FDEEE77A84F82C3084
:103C2000C4ED0C7A03B030BD002384F82C30F9E7E2
:103C30000000C84238B504460D46FFF7BFFF30B15B
:103C4000032128461BF094FD80F00103D8B204F54F
:103C5000C04484F82D0038BD73B500F5C0454A68EE
:103C60006A620B780E46D907044606D500F5A043D4
:103C7000D3F8F03F5B6813446B6295F82D302BB19D
:103C800004F5C04114312046FFF7D4FF33785B07B9
:103C90000ED504F5AD40012201A9183053F024FAE5
:103CA00030B1012385F82C3073682B6302B070BDEE
:103CB000002385F82C30F9E7F0B52DED028B044692
:103CC00083B004F5C0450E468DED010AFFF7C4FF31
:103CD000DFED320A9DED010A40F24310B7EE001A03
:103CE0002CF032FCAB6A5B4207EE903AF8EEE77AD2
:103CF000204667EE807A04F50057FDEEE77AB0EED5
:103D0000408A17EE901AFFF72BFFD7ED9F7AF5EE5A
:103D1000C07AF1EE10FA3CDDAB6A002B39DD2046AB
:103D2000FFF7CAFC07EE900ADFED1D6AB8EEE77AEE
:103D3000D7ED9F7A67EEA67AB4EEE77AF1EE10FA45
:103D400027D531462046FFF787FF29463246043102
:103D50002046FFF7D3FBAB6A5B4207EE903AF8EEE2
:103D6000E77A204667EE887AFDEEE77A17EE901A3A
:103D7000FFF7F6FEB5EEC08AF1EE10FA09DDD5EDDB
:103D80000A7AB8EEE77AC7EE087AFDEEE77AC5ED73
:103D90000A7A03B0BDEC028BF0BD00BF000000004A
:103DA0000000C8C2F0B500F5C04487B0237D03F021
:103DB0000503052B07460BD054F0E4F94FF4AE721F
:103DC0004FF4801154F096F90025284607B0F0BD55
:103DD0001E486A4603211BF0DBFC0028F4D01C4877
:103DE00001AA03211BF0D4FC05460028ECD0194B96
:103DF000DFED190A93ED000A40F26D10B7EE001ADC
:103E00002CF0A2FB04F114030FCBB0EE401A02AE6B
:103E1000DFED111ADDED010A9DED000AB7EE002A73
:103E200086E80F002CF0C2FADFED0C7A20EE270AAC
:103E30003046FDEEC07A032217EE901A1BF0D4FB39
:103E400031463846FFF708FFBFE700BF848B0020EC
:103E5000A48B00208C800020000000000000C842DD
:103E6000F7B50E4602210446FFF77AFA70B304F55F
:103E7000A045D5F85C35042B28D12046FFF79EFEDF
:103E800020B304F5AD47183704F5C04101236A4655
:103E90000431384653F012F8C0B104F5C041012393
:103EA00001AA1431384653F009F878B19DED017A32
:103EB000DDED007A77EEC77A96ED007A37EE277A55
:103EC00005F21C5586ED007AC5ED007A03B0F0BD11
:103ED000F0B52DED048B00F5005489B000F5516666
:103EE00094F81A1C0391054630464CF045FA0399A4
:103EF000074630464CF052FA042F0399B0EE408A40
:103F000020D1002305A88DED050A069307932FF015
:103F100077FD05A905F5AF502DF040FCDFEDAC7A3B
:103F20008DED050AB4EEE71AF1EE10FACDED060AB2
:103F30008DED071A06DB05F5805393F83C7517F0F5
:103F400001070CD194F8503C002262F3000384F87E
:103F5000682C84F8503C09B0BDEC048BF0BD94F89B
:103F6000503C9A075FBF43F0020384F8503C04F6CC
:103F7000544383ED008A05F5315104F66C4383ED1B
:103F8000001A2C312846FFF76BFF94F8683C092B88
:103F900000F2898004F54763D3ED000A9FED8D9A06
:103FA000B0EE480A2CF0BEF900BB04F6544394F876
:103FB0001A1CD3ED008A30464CF00EFA07EE900A38
:103FC0009FED857AF8EEE77A78EEC88A67EE877A11
:103FD000F0EEE88A67EE897AF4EEE78AF1EE10FAFD
:103FE000C2BF94F8683C013384F8683C04F5476329
:103FF00094F81A1CD3ED008A30464CF0EDF907EE28
:10400000900AF8EEE77A9FED757A67EE897A78EE96
:10401000C88A67EE877AF0EEE88AF4EEE78AF1EE76
:1040200010FA02DD002384F8683C04F5476383ED51
:10403000008A94F8503CDA078DD52846FFF7E6FB56
:1040400004F66C4393ED008A05F5C04330EE488AD0
:1040500093F82C30002B70D005F5AD40012205A956
:10406000183053F041F800286DD18EF0B7FAD4F82B
:10407000642C41F28831821A8A42034604F658427F
:1040800004F65C4168D982ED008A284681ED008AF9
:104090000221FFF765F918B105F5BE452A6CEA6300
:1040A000C4F8643C57E794F8503C43F0010384F8AB
:1040B000503C05F5A04305F59B42D3F85C6505F53A
:1040C0008043301FD3F8203F464202F1140246419C
:1040D000934211D005F59B42303293420CD005F546
:1040E0009942934209D13E4B05F5C140B3F8BE1544
:1040F000583009F0ABFC00B13E4694F8503C5907EB
:1041000093D4002E91D002212846FFF729F90028E8
:104110008BD043F0040384F8503C04F66C4305F55F
:104120004F561868F8F7F0F92836CDE900012D4A06
:104130000621304658F0A6FE77E72846FFF73EFDF9
:10414000002889D191E704F66C4393ED000A9DEDB8
:10415000058A38EE408A88E79FED200A92ED007AC2
:10416000DFED217A28EE008AA7EE278A82ED008A09
:10417000C4F8640CD1ED007A38EE678AF3EE0E7A5B
:10418000B0EEC88AB4EEE78AF1EE10FA7FF7E3AE3C
:1041900094F8503C5B070ED504F66C4405F54F5679
:1041A0002068F8F7B1F92836CDE900010F4A062159
:1041B000304658F067FE05F53150242200211030BA
:1041C00009B0BDEC048BBDE8F040B6F0D3B800BF39
:1041D000000000340AD7233CCDCC4C3DCDCC4C3E26
:1041E000907B002014460D08CDCC4C3F31460D0885
:1041F00038B52DED028B0D460446FFF707FB002373
:1042000020462B70B0EE408AFFF720FC02212046AA
:1042100038EE400AFFF7A4F828B104F5005494F8EA
:10422000500C00F00100BDEC028B287038BD00007E
:1042300070B50B7803F00503042B05460C461646B3
:1042400015D105F5A04553F09DFFB2B24FF4801192
:1042500053F050FFD5F8F02F636852689B1A13F59E
:10426000FA7FC8BF6360237843F00103237070BDF9
:10427000F8B500F5805300F5A047D3F83065D7F8BE
:104280002055B542044619D00E4A1268D26A92F8F7
:104290009C209AB100F5C041751B25221431FFF70F
:1042A000C7FF07EE905AB8EEE70ADFED077A04F58C
:1042B000335020EE270A183080F0CAFFC7F8206577
:1042C000F8BD00BF8C2B00200AD7233CF8B500F5C1
:1042D000A046054696F813E58C4600F5C04406F660
:1042E000F477BEF1000F49D004F114030FCB87E837
:1042F0000F00012386F814359CE80F0004F1140721
:1043000087E80F00E36905F5C04714375BB9236AF6
:104310004BB9E368A269E361236923621AB9A16812
:1043200038461BF061F9394628222846FFF780FFFE
:10433000217D11F0040102D138461BF019FA05F570
:10434000BF4105F5C0403A46743104301BF014FCFF
:1043500030B1043494E80F0006F6F47686E80F00D6
:10436000284606F0DDFC2846FFF7E8F9284607F066
:10437000C5F82846BDE8F840FEF7CABF231D0FCB9D
:1043800087E80F00012386F8133586F814E5B3E7B4
:104390002DE9F04100F500530446B3F9D231002B6A
:1043A0000D4635DB0B7813F0020F14BF4FF0FF33CF
:1043B000012304F5A04604F5C04886F8CC3F08F177
:1043C00004030FCB06F6F47787E80F0095E80F009B
:1043D00008F1140787E80F00572239462046FFF7F7
:1043E00027FF2046FFF7FAFB20460025FFF7A6F936
:1043F000204607F083F886F81455C6F8D05F86F893
:104400001955204606F08CFC88F81A52BDE8F08158
:104410004FF0FF33CDE700002DE9F043354B1B682B
:1044200085B00546D86AF9F77FF800285FD105F511
:10443000005393F9E83B5A1C52D0002B05F58666D1
:1044400011DD95F84124242107EE903A01FB026228
:1044500092ED0B7AF8EEE77AB0EEC77AB4EEE77A2F
:10446000F1EE10FA3CDC05F5805305F5965793F80C
:104470003C3513F0010429D0C3F340089B0732D424
:1044800095F8E41395F828444FF0B00909FB015161
:1044900091F8C1314CBB022B18D968461BF09EF82D
:1044A0006946384615F0F0F8044678B195F8E433DB
:1044B00009FB03534246D3F8D01168461BF094F829
:1044C00015F0B8FB694614F0CDFF0446304617F0EE
:1044D00061FE384614F0E4FE2846FAF795FA2046C5
:1044E00005B0BDE8F0830024F0E74446EEE7002085
:1044F000F6E700BF8C2B002038B50C4B1B68054637
:10450000D86A0C46F9F710F810B10024204638BDDF
:1045100015F090FB214614F0A5FF04460028F4D0C6
:1045200005F5AB4030F086F8F0E700BF8C2B00209B
:10453000F0B500F5A04700F5C045002387F8133516
:1045400087F814352B1D044600EE101A0FCB87B0E8
:1045500007F6F47686E80F0002AE2A46B8EEC00AE7
:104560003046164904324BF07BFC96E80F001435B8
:1045700085E80F0040F25712294620460195FFF7C3
:1045800057FE01992046FFF755FB01992046FFF79A
:1045900063FB04F500532046B3F9D231002BB4BFBE
:1045A0004FF0FF33012387F8CC3FFFF7C7F82046D1
:1045B00007B0BDE8F04006F0A1BF00BF18620020C0
:1045C00010B5034904464BF04BFC204610BD00BF1C
:1045D00018620020F8B500F5C046331D00F5A04470
:1045E00005460F460FCB04F6F47C8CE80F0007F16C
:1045F00008012846FFF76AFEBB8803EB830303EB41
:1046000083039B001BB2002BD8BF4FF4C873A4F8E0
:104610000E35D4F8F03FB2695968521AC4F8E02454
:104620009A680A32F261DB680A3333620023C4F805
:10463000F43484F8103584F82435C4F8E43404F5EF
:104640009B6300221A604FF0FF33C4F8D03495F812
:10465000412405F58663242101FB023304F5A1649E
:10466000DB6A2360F8BD000070B50E4608310446D1
:10467000FFF72CFEB38804F5A04543B3642213FB77
:1046800002F3C5F8E034B5F90E35002BD8BF4FF46E
:104690007A7304F53150D8BFA5F80E3524220021D5
:1046A0001030B5F067FE04F5C04304F5BE4093ED4D
:1046B000100A314634308AF0D7F8D5F85C35072B2C
:1046C0000CD120460421BDE87040F9F75DBED5F855
:1046D000E034002BD7DC40F6B833D2E770BD0000E1
:1046E00030B5083104460FC985B06D4685E80F0026
:1046F00004F5C041043128461BF0DAF8204629466B
:10470000FFF7E4FD04F580440123C4F8483F05B0F9
:1047100030BD00000B7A00F5A04013F0020F14BF6B
:104720004FF0FF33012380F8CC3F70477FB501F194
:10473000080305460E460FCB6C4684E80F0005F5CE
:10474000C041043120461BF0B3F821462846FFF74C
:10475000BDFD31462846FFF7DDFF04B070BD000007
:104760007FB501F1080304460E460FCB6D4685E880
:104770000F0004F5C041043128461BF099F8294682
:104780002046FFF7A3FD20463146FFF7C3FF3379EC
:1047900007EE903A337E9B0748BF9FED0C7AF8EE08
:1047A000677A04F5A04448BF67EE877A9FED087AE0
:1047B00067EE877AFCEEE77A17EE903AC4F8C43FCA
:1047C0000123C4F8E43F04B070BD00BF0000803B8B
:1047D00000A00C477FB501F1080304460E460FCB3D
:1047E0006D4685E80F0004F5C041043128461BF0F2
:1047F0005FF829462046FFF769FD20463146FFF75E
:1048000089FFB38804F5A0444FF47A725343C4F887
:10481000DC3F0123C4F8E43F04B070BD2DE9F3414F
:1048200000F5C0450446143500F5BF400E4674300F
:1048300029461AF0FDFF04F5A047C0B94FF0FF3339
:10484000C7F8D03406F1080840461AF0F7FE0328EE
:1048500002463AD1F16828461AF0C6FEB388C7F876
:10486000E43F204602B0BDE8F041FEF741BE24F02F
:104870002FFCF9F7DFFA012812D94FF0FF33C7F800
:10488000D03424F025FC90F8C432DFED150AB022B4
:1048900002FB030090ED300A28461BF0A7FAD1E78F
:1048A00004F58058D8F8C0042BF022FE04F5A65376
:1048B000C7F8D004D3ED007A9FED0A0ADFED080AAD
:1048C000F8EEE77A27EE800AE6E701AA00214046E3
:1048D0001AF0C0FE0028C1D001990022BBE700BF3A
:1048E00000007A440AD7233C7FB501F1080304464F
:1048F0000E460FCB6D4685E80F0004F5C04104312C
:1049000028461AF0D5FF29462046FFF7DFFC20464F
:104910003146FFF7FFFE04F5A0440023C4F8E43F4E
:1049200004B070BD37B504460D468DF057FE2062C9
:10493000D5ED027AF5EEC07AF1EE10FA15DD9FEDB5
:10494000127A67EE877AFCEEE77AC4ED077A5FF0B9
:10495000F9F8E2694FF47A73B2FBF3F30B4A0621DC
:1049600003B0BDE8304058F08DBA6AF0E9F8002392
:10497000009395F90D2095F90E3095F90C106AF019
:104980007BF8E061E3E700BF00007A44AC460D0825
:104990002DE9F0432DED028B85B0044615F04AF960
:1049A00014F030FA04F5805304F5A04793F8B837B3
:1049B0000BB9002877D0D7F8D034013373D1D7F8AA
:1049C000F434002B4BD08DF009FED7F8F434C01A24
:1049D000B0F5FA6F67D394F8E423DFED5F7A9FEDCB
:1049E0005F8A4FF0B00808FB024292ED780A20EE91
:1049F000270A2BF095FD07F59B69D9ED007A30EE7B
:104A0000670A2BF08DFDDFED567A20EE080A04F5DB
:104A10004F5620EE270A2BF02BFDFDEEC07A2836EC
:104A200017EE905AC7F8D054D9ED007A67EE887A1D
:104A300017EE900AF7F768FDCDE9020194F8E43328
:104A400008FB0343D3F8DC01F7F75EFD454ACDE9E7
:104A500000012B460621304658F014FA23E004F5F5
:104A60009070F9F7E7F902281DD994F8E433B022E1
:104A700002FB034393ED777AF1EE047AB4EEE77A22
:104A8000F1EE10FA0FDD384B1B68D86A0368DB695A
:104A90009847012803D08DF0A1FDC7F8F404D7F89A
:104AA000F434002B8FD104F54053D7F8D014D3F849
:104AB00004064A1C036845D01B6B98472B4810F02E
:104AC0004FFD18B104F5AB4032F014F82046FEF764
:104AD0001FFED7F8E0348342054636DA07EE905AD7
:104AE0009FED237AF8EEE77A04F54F5667EE877A62
:104AF000283617EE900AF7F707FD1E4ACDE90001A8
:104B00003046062158F0BEF901254FF0FF3304F579
:104B1000C044C7F8D03487F81055231D0FCB07F6D3
:104B2000F476143486E80F0084E80F0012486AF027
:104B300083F9002387F81335284605B0BDEC028BB6
:104B4000BDE8F0835B6B9847B8E7084810F0E8FCD5
:104B50000028C3D1F1E700BF35FA8E3CE02E654254
:104B60000000C842BC460D088C2B0020902B002072
:104B70000AD7233CE0460D08304C00202DE9F041D7
:104B800000F5BF4600F5C045743614350446294685
:104B900030461AF04DFE04F5A04704F5405830B3F6
:104BA000D7F8D0144B1C22D0D8F8040603681B6B2E
:104BB0009847D7F8E43F012B04F5C04545D0D7F816
:104BC000E43F022B05D12046FEF760FDAB69984219
:104BD00041DD2046FEF75AFDAB69C01A0028B8BF78
:104BE0004042B0F5FA7FCCBF0020012034E004F54C
:104BF000C040294604301BF053F8DFED187AB4EEBC
:104C0000E70AF1EE10FA16D5304629461AF018FFD9
:104C10009FED137ADFED130AF6EE007AE0EE077AE5
:104C200028469FED110AFDEEE77AF8EEE77A27EEC7
:104C3000800A1BF0DBF8D8F804069FED0C0A036825
:104C40002A469B6A31469847B3E72046FEF71EFD89
:104C5000AB699842B3DB0120BDE8F0810000484316
:104C6000A00CB345000096430AD7233C0000000087
:104C700073B5384CD1ED026AD4ED027A9FED367AE5
:104C8000F8EEE77A0546D7EE876A0E46F5EEC06A7B
:104C9000F1EE10FA08DD5EF055FF304A062158F0BB
:104CA000F1F8012002B070BDD1ED037AF5EEC07AC3
:104CB000A4F53164F1EE10FA94ED006A12DDF4EE21
:104CC000C67AF1EE10FA0DD55EF03CFF054620687D
:104CD000F7F71AFC224ACDE900010621284658F0D0
:104CE000D1F8DEE7DFED1F7A337CB4EEE76AF1EE50
:104CF00010FA54BFB0EE677AB0EE467A0BB90020D6
:104D0000D0E7B5EEC06AF1EE10FA0CDC86EE876AE9
:104D100003EB830307EE903AF8EEE77AF4EEC67AF7
:104D2000F1EE10FAEBD595F82440002CE7D18DF088
:104D300055FCAB6AC01A337C4FF47A7253439842E5
:104D4000DDD9012385F824308DF048FCA862204687
:104D5000A8E700BF908B00200AD7233CFC460D0833
:104D60000D470D080AD723BC38B505467CF0B4FDC5
:104D70007BF068FB044640B98DF030FC2B6AC01A0A
:104D8000EB69984284BFEC610124204638BD0000E5
:104D900038B504460D468DF021FC04F5A0439FED87
:104DA000077AC3F8E80FD5ED027A67EE877AFDEE51
:104DB000E77A17EE902AC3F8E42F38BD00007A4452
:104DC00010B504468DF00AFC04F5A043D3F8E82F93
:104DD000801AD3F8E42F90424FF0000084BFC3F84C
:104DE000E40F012010BD000000F5A04303F59F6112
:104DF000D3F8E42F91ED007A22EAE27207EE902ACE
:104E0000F8EEE77A0020B4EEE77AF1EE10FA44BF4C
:104E1000C3F8E40F0120704710B500F50053B3F953
:104E2000D231002B00F5A043B4BF4FF0FF32012276
:104E300000F5C04083F8CC2F00F1140404300FC8F3
:104E400084E80F0010BD000038B504462DED028B3C
:104E5000F0EE408AB0EE608A09B301295ED0B5EE6B
:104E6000C08AF1EE10FA69DDDFED357AB4EEE78A3B
:104E7000F1EE10FA62D8FCEEC87A04F54F5017EE46
:104E8000903A304A0621283057F0FCFFFDEEC87AF0
:104E900004F5005417EE903A84F89F313CE0F8EEA8
:104EA000000A2BF03FFA40B104F580444FF0FF3385
:104EB000C4F8583FBDEC028B38BD04F50053B3F97C
:104EC000A82107EE902AF8EEE77AF4EEE87AF1EE00
:104ED00010FAC4D8B3F9AA3107EE903AF8EEE77A9F
:104EE000F4EEE87AF1EE10FAB9DBDFED157A68EE50
:104EF000A77A04F58043FDEEE77A04F54F5017EEEC
:104F0000902AFCEEE87AC3F8582F062117EE903A63
:104F10000D4A283057F0B6FF0120CBE7FCEEC07AEF
:104F200000F54F5017EE903A084A0621283004F554
:104F3000005457F0A7FFC4ED6D8AEDE70020B9E7F4
:104F40000000C84253470D082C470D0840470D0884
:104F5000D1F80D3000EE903AD1F80930097A00EE20
:104F6000103AFFF771BF000070B58B88012B044623
:104F70000D4611D100F590763046F8F75BFF022818
:104F80000AD994F8E413B02303FB01612046AC3145
:104F9000BDE87040FFF7B0BA14F04CFE05F108010F
:104FA000BDE8704014F05EBAF0B500F5A0470024EB
:104FB000AB4B87F8194589B0054608460E4683F87D
:104FC0002D402FF049F998B3012387F8103505F5E6
:104FD0004053D3F804060368DB6B984787F81745FE
:104FE000C7F8D04F03A81AF0F9FAB7F8BC154FF676
:104FF000FF73994208BF2146013101AA89B205F524
:10500000AB4031F0F9F8F0B1BDF80630A3F115026C
:105010005342534187F8113550B105F5C140BDF8F1
:105020000610583008F012FD10B1002387F8113532
:1050300073885E2B4ED8522B07D8103B9AB20F2A9A
:1050400022D90024D5E00346E4E7533B0B2BF8D8E4
:1050500001A252F823F000BFED510108F9510108F7
:105060000952010843500108435001084350010808
:1050700043500108435001084350010843500108C0
:1050800055520108095201080F2BDAD801A252F833
:1050900023F000BF71510108AB510108B55101085F
:1050A000BF510108D35101087D5101084351010846
:1050B0004350010843500108435001084350010880
:1050C000435001084350010843500108E3510108CF
:1050D000C9510108BD2B1AD8BB2B47D8B22B00F001
:1050E000A7800DD8702B00F09E80722BA9D1D6ED31
:1050F000027AFDEEE77A17EE903AC7F8E43F35E022
:10510000B32B9ED131462846FFF72EFF2EE0D42B3D
:1051100000F0938040F6B832934200F09680D22B94
:105120008FD1B388012B21D803F0010387F8123502
:1051300005F54F50B3884B4A0621283057F0A2FEA0
:1051400014E0002305F5C14487F8493558347188C7
:10515000204607F023FF314628B1204609B0BDE8BC
:10516000F04008F01DB92846FFF734FA012440E06A
:1051700006F108012846FFF7A9F8F7E705F5C1444D
:1051800058341521204608F061FC48B1002387F807
:1051900049353146204609B0BDE8F04008F004B872
:1051A00031462846FFF760FAE0E731462846FFF728
:1051B000BDFADBE731462846FFF7D2FAD6E731469B
:1051C0002846FFF707FBD1E731462846FFF78CFB5F
:1051D000CCE705F5994129222C3128460EF01CF91F
:1051E000C4E731462846FFF719FBBFE7012487F8DB
:1051F0001745204609B0F0BD002305F5C14087F8EA
:10520000493531465830A9E705F5C1475837384682
:1052100008F000FC3146044618B12846FFF760FA52
:10522000E7E73846B7E731462846FFF7B1FD9DE787
:1052300031462846FFF78CFE98E7B188003918BF41
:105240000121284600F016FF90E7317A064807F062
:10525000A5FA8BE7314605F59940FFF763FB85E733
:10526000908B002064470D08688C002000F5804278
:1052700000F59943D2F8202F9A4201D1FFF794BE4E
:105280000120704710B500F5804200F59943D2F82F
:10529000202F9A4204460DD1194608222C310EF0D7
:1052A000BBF804F54F50044ABDE8104006212830F1
:1052B00057F0E8BD10BD00BF74470D082DE9F04F51
:1052C0002DED048B00F5C04393ED568ADFEDD77AC0
:1052D000B0EEC87AB4EEE77AF1EE10FA48BF00F506
:1052E0000053DFEDD37A42BFB3F9D23108EE103A62
:1052F000B8EEC88A00F5A048B4EEE78AF1EE10FADD
:1053000094BF4FF0FF37012700F5804588F8CC7F28
:10531000D5F8483F9BB004460E46F0EEC88A052BF0
:1053200016D8DFE813F006002C0069008800C500DD
:105330005F0100F540543A46D4F804060368B0EE25
:10534000680ADB6A08319847BA4806F011F908B9CB
:10535000002048E1B84C54F8103CB4F998115B684F
:10536000642201FB0231A4F5C040FFF7E1F8A4F587
:10537000C04005F0D5FC0123C5F8483FE8E700F53B
:1053800040533A46D3F804060368B0EE680ADB6A75
:1053900008319847D8F8C83F002BB8BF5B42012BB3
:1053A000D6DD98F8CD3F1BB998F8CE3F002BCFD073
:1053B00004F5B153D3ED020A93ED030AF1EE600A4E
:1053C000B1EE400AB2F0DCFDDFED9C7A20EE270A58
:1053D00005F64C7383ED000A10EE100AF7F794F807
:1053E00004F54F542834CDE90001954A06212046A2
:1053F00057F048FD0223BFE700F5C04901F1080A54
:1054000009F10409494650461AF04AFC30EE680A90
:10541000F1EE047AB0EEC00AB4EEE70AF1EE10FA4B
:1054200000F3E680D8F8C83F0133022B40F2EA804F
:105430000323C5F8483F04F5405306F10808D3F8A4
:10544000040603683A46DB6AB0EE480A41469847CC
:10545000DFED7C6A9FED7C7A05F64C73D3ED007A24
:10546000012F18BFB0EE667A04F5A65377EE877A5F
:1054700093ED030A9FED757AA7EEC70A2BF050F85B
:10548000DFED737AB0EEC00AB4EEE70AF1EE10FA7F
:105490007FF55EAF04F54F50062128306D4A57F076
:1054A000F1FC0423C5F8483F41462046FEF70EFFB5
:1054B00006F1080595E80F000AAF0DF1380887E8F6
:1054C0000F0088E80F0004F5804303F64C7A9FED47
:1054D000629A9AED000ADFED610A0393384630EED6
:1054E000090A1AF083FCDFED5D0A9AED000A9FEDD0
:1054F0005C8A40461AF07AFC04F540534246D3F8E1
:105500000406036839469B6AB0EE480A984795E856
:105510000F0004F5C1490DF1480B09F158098BE85A
:105520000F00DAED009A484607F05EFD79EE899AA1
:1055300004F5C048F0EE400A5846B0EE690A08F19A
:1055400004081AF053FC5A46394640461AF014FB38
:10555000834695E80F009AED000A16AF87E80F0022
:10556000F0EE680A30EE090A38461AF03FFC394678
:1055700040462A461AF0CAFA07A904F59650F0EEFA
:10558000408A8DED078A8DED088A8DED098A14F029
:105590004FF9002866D0294640461AF08DFA05A931
:1055A00007A8CDED060A8DED050A2DF0BDFFDFED54
:1055B000237A20EE270A2AF047FFB0EEC00ABBF19B
:1055C000000F3FF4C5AEF3EE0E7AB4EEE70AF1EE4B
:1055D00010FA23D5039A0523C2F8483F31464846BE
:1055E00007F0E2FD01201BB0BDEC048BBDE8F08F9D
:1055F000494650461AF054FBB4EEE80AF1EE10FAB0
:105600007FF510AF04F540543A46D4F80406036819
:10561000B0EE680ADB6A5146984799E6F6EE007AE2
:10562000F4EEE78AF1EE10FAD4DC91E600000034E3
:10563000000000B4902B0020908B0020E02E6542EB
:105640009C470D080000B4420000874335FA8E3CA9
:10565000C2B8B23DBE470D080000344300007A4492
:1056600000000000BBF1000F3FF472AEB2E700BFD4
:105670002DE9F041044600F5C1408EB058300F4688
:1056800008F008FA054638BB09AE04F5A0483046D4
:1056900019F0A4FFB8F8BC354FF6FF72934208BF6B
:1056A0000023013307AA99B204F5AB4030F0A4FD02
:1056B000B0B10FB1C8F8C85F96E80F0001AD85E83A
:1056C0000F0004F5C0441434E368009394E80E001E
:1056D000044803F0CDF9054628460EB0BDE8F08138
:1056E0000125F9E75878002070B5064606F5A04573
:1056F000002106F03DF8D5F8D04F7CB9304605F0D2
:1057000037FF10B90024204670BDD5F8C83F012BE3
:10571000F8DD8CF063FFC5F8D00FF4E7D5F8E41F8F
:1057200061B18CF05BFFD5F8D03FC01AD5F8DC3FF3
:105730009842E7D90023C5F8E43F01213046FFF73E
:1057400097FF04460028DDD006F54F50044A062195
:10575000283057F097FB002385F81935D3E700BFB1
:10576000E0470D0870B50A468B88190A137E054676
:10577000DB0748BF01EB810105F5A04448BF4900A4
:10578000002605F0F5FF84F81965284605F0F0FEBF
:1057900010B90024204670BDD4F8E41F51B1D4F8EC
:1057A000C83FD4F8C42F9342F3DD012BF1DDC4F8D8
:1057B000E46F01212846FFF75BFF04460028E8D08C
:1057C00005F54F50024A0621283057F05BFBE1E710
:1057D000F8470D0838B5054605F5A044898805F059
:1057E000C7FFD4F8E43F8BBBD4F8C83F002BB8BF49
:1057F0005B42012B02DC0024204638BD94F8CD2FFB
:1058000094F8CE3F7AB9002BF5D005F5C04305F5E5
:105810004F509A6806216423283092FBF3F30C4A18
:1058200057F030FB01E0002BEFD10121C4F8E41F59
:105830002846FFF71DFF04460028DCD005F54F5031
:10584000044A0621283057F01DFBD5E70021EFE779
:1058500010480D082E480D0810B504460B4808F0F6
:10586000FDFE48B10A4BDFED0B7AD3F8143193ED0E
:10587000090A20EE270A10BD04F50054B4F90032DD
:1058800000EE103AB8EEC00AF5E700BF688C0020C1
:10589000908B00200AD7233C38B52DED028B00F504
:1058A000005300F5A045B3F904120029ACBF012351
:1058B0004FF0FF330029B8BF494285F8CC3F04467A
:1058C00089B205F055FF05F59F65204695ED008AE4
:1058D000FFF7C2FFB5EEC00AF1EE10FAD8BF9FED98
:1058E0000E0ABCEEC00AB8EE400AB4EEC08AF1EE71
:1058F00010FA0AD804F54F502830084A062157F00C
:10590000C1FA0120BDEC028B38BD204605F030FE07
:105910000028EFD1F6E700BF0000000048480D085E
:105920002DE9F04F00F5A0472DED028B4FF0FF332E
:1059300000F5C04AC7F8D0340AF114038C46054676
:105940000FCBBCF804409CF8049089B004AE240A44
:1059500086E80F0020D005F5BF4808F174083146ED
:1059600040461AF09DF931464046B0EE408A1AF0A2
:1059700067F8DFED577AB4EEE78AF1EE10FA0BDB49
:10598000E3B200EE903ADFED537AF8EE600A20EED3
:10599000270A30461AF02AFA05F5405B97F81425D5
:1059A000DBF804069FED4C0A036805F5C0489B6AC6
:1059B00008F1040832B305F5BF4132467431984707
:1059C00005F50053B3F90232002B1EDD07EE903AC5
:1059D00007F59F62F8EEE77A92ED007AB4EEE77A87
:1059E000F1EE10FA11DD05F5BF4132467431404643
:1059F0001AF0C2F8F8B90024204609B0BDEC028BB9
:105A0000BDE8F08F32464146D9E7B9F1000F1CD10D
:105A1000002C3CD1DBF8044623682846D3F82090BC
:105A2000FFF71AFF07F2EC43D3ED000A2046C84700
:105A3000B0EE408A0DE0002CDDD10AF104030FCB5B
:105A400007F6F47787E80F00D6E707EE909AB8EEEE
:105A5000678A314640461AF023F9B4EEC08AF1EE67
:105A600010FA17DBB7F8BC350393314640461AF0FD
:105A700017F9BCEEC00A05F54F50039B174A8DED90
:105A8000000A0621283057F0FDF90124B4E79FED04
:105A9000128ADEE705F5BF413246743140461AF0FE
:105AA0006BF804460028A6D0B7F8BC3503933146FE
:105AB00040461AF0F5F8BCEEC00A05F54F50039BBE
:105AC000074A8DED000A0621283057F0DBF993E7ED
:105AD00000000034E02E65420000000060480D0820
:105AE0007E480D082DE9F0474B881F2B8AB00446ED
:105AF0000D466BD80F2B41D804F54F50BE4A0421F8
:105B0000283057F0BFF99BE0A3F1BC02182AF3D864
:105B100001A151F822F000BF415C0108415C01087D
:105B2000F95A0108F95A0108F95A0108F95A010805
:105B3000F95A0108415C0108F95A0108415C010861
:105B4000F95A0108F95A0108F95A0108415C01089B
:105B5000F95A0108F95A0108F95A0108415C01088B
:105B6000415C0108415C0108F95A0108F95A010831
:105B7000415C0108F95A0108415C0108A3F11002D7
:105B80000F2AB9D801A151F822F000BF7D5C0108AD
:105B9000635D01086D5D0108795D01088F5D010895
:105BA000895C0108535C0108F95A0108F95A010897
:105BB000F95A0108F95A0108F95A0108F95A010875
:105BC000F95A0108995D0108835D01085E2B21D80F
:105BD000522B91D9A3F153020B2A8DD801A151F870
:105BE00022F000BFA35D0108B35D0108BD5D01089F
:105BF000F95A0108F95A0108F95A0108F95A010835
:105C0000F95A0108F95A0108F95A0108E75D010833
:105C1000BD5D0108722B00F0E18007D8702B7FF486
:105C20006BAF0AB0BDE8F047FFF7CAB8D42B09D86C
:105C3000BB2B3FF669AFA3F1B202012A3FF65CAF7E
:105C4000012052E0DF2BFBD040F6B8329342F7D070
:105C500052E700F5C14658361621304607F09EF946
:105C600030B1294630460AB0BDE8F04707F084BCA1
:105C700020460AB0BDE8F047FEF78ABE29460AB0C2
:105C8000BDE8F047FFF74CBE00F5C145583515217A
:105C9000284607F0DBFE28B128460AB0BDE8F047E9
:105CA0000BF0CCB904F5A04504F5BE46D5F85C353B
:105CB00004F5BF4704F5C04804F5C049072B06F1B9
:105CC000340607F1740708F1140809F104090FD12B
:105CD00004F5AA4458340194D5F8E03400934246C0
:105CE0004B463946304688F083FE0AB0BDE8F0875F
:105CF0000DF127018DF827004048FEF779FA05F2EB
:105D00001C53D3ED007AD5F800A505F59E63D3EDBD
:105D1000000A05F2FC4330EE670A93ED001A8DEDA0
:105D2000070A04F5C1401030CDED060A8DED051AC5
:105D30007AF07EFB0546204600F064FF9DF8273090
:105D40009DED051ADDED060A9DED070ACDE902037A
:105D5000CDE900A54B4642463946304688F09EFDC7
:105D6000C3E7A98805F004FD0020BEE729460AB074
:105D7000BDE8F047FFF7F6BC0AB0BDE8F047FFF713
:105D8000B3BC29460AB0BDE8F047FFF723BD0AB00F
:105D9000BDE8F047FFF780BD0AB0BDE8F047FEF769
:105DA000EDBE294604F599400AB0BDE8F047FEF77C
:105DB0005FBF04F5C1402946583054E704F5C14699
:105DC0005836304607F026FE08B9304665E72946C2
:105DD0002046FFF773FA0028F7D186E70AB0BDE83E
:105DE000F047FFF701B8294604F599400AB0BDE82D
:105DF000F047FEF7B9BF00BF9C480D08902B00206C
:105E000070B500F5804200F59943D2F8202F9A42F0
:105E100005460E4602D00024204670BDFFF762FE04
:105E200004460028F7D005F54F50318828305BF044
:105E300069F9F1E721F04003152B04D0A1F15E03CD
:105E400058425841704701207047000000F58042D9
:105E500000F59943D2F8202F9A4207D100F5A040CF
:105E6000B0F8BE355B1A5842584170470020704761
:105E7000192962D8DFE801F00D1115191D21252817
:105E80002C613033365539393C3F4246494D6151DA
:105E9000595D00F59A402030704700F59640743007
:105EA000704700F597401030704700F597402C3050
:105EB000704700F597404830704700F5984004302F
:105EC000704700F59840E6E700F598403C30704791
:105ED00000F598406430704700F59940704700F530
:105EE0009940E4E700F59940E5E700F59940F1E7CE
:105EF00000F59A40E3E700F59A40E7E700F59A409D
:105F00005830704700F59A40C9E700F59B401430BF
:105F1000704700F59B403030704700F59B40503093
:105F2000704700F59C400830704700F59C404430B5
:105F3000704700F59B406C307047002070470000B0
:105F400000290DDB074890F84C2CCBB29A4207D3BE
:105F5000D0F8483C0122595CA0F500500DF034BB4C
:105F6000704700BF904B00202DE9F34100F500532E
:105F700000F54F5593F8183C03F0010603F00208B2
:105F800003F004075B07044605F1280535D01F4AD6
:105F90000621284656F076FF26B104F53D501C3008
:105FA0007CF0A8FAB8F1000F04D004F54250343068
:105FB0007CF01CF827B104F548500C307CF0C4FE8E
:105FC00004F5C044012384F82934114A114B1249C5
:105FD000B8F1000F08BF1A46002F08BF1946CDE9D7
:105FE00000210E4A0621002E18BF134628460C4AEF
:105FF00056F048FF02B0BDE8F0810A4A0621284663
:1060000002B0BDE8F04156F03DBF00BFC9480D08E1
:10601000BE480D0864360E08C5480D08B8480D087E
:10602000DA480D08EC480D0810B5044600F53D505F
:106030001C307CF08BFA04F5425034307CF002F8CE
:1060400004F548500C307CF0B9FE04F5C04393F8D9
:1060500029245AB1002283F8292404F54F50044A18
:10606000BDE810400621283056F00CBF10BD00BF1F
:106070000C490D0809B1FFF777BFFFF7D5BF000046
:1060800000F580430949D3F8202F8A420CD093F8B9
:106090002D3F3BB900F599418A4203D100F5A0405C
:1060A00090F81235184670470023FBE7B0780020BF
:1060B00010B504468CF092FA054BD3F8403FC01A55
:1060C000642804D82046BDE810405EF057BF10BDDC
:1060D000906B002010B500F53054D4ED027AF5EE47
:1060E000C07AF1EE10FA8AB04FF0000304F1080410
:1060F00044D907930893099306AB019307AB009328
:1061000003AA05AB04A900F5965013F031FA30B399
:10611000DDED080A9DED070AB1F096FDDDED090AF7
:10612000B1F092FDD4ED007A9DED047A77EEA76A86
:10613000B4EEE70AF1EE10FAF4EEC76AACBF012044
:106140000020F1EE10FA0CD802309DED037AF4EE47
:10615000C77AF1EE10FA0CD8003818BF01200AB047
:1061600010BDF4EEC77AF1EE10FA9CBF0130C0B258
:10617000EBE7012894BF00200120F0E70020EEE7C4
:1061800038B5124B1A7A0446FAB901251D7253F03C
:106190000BFE2A4604F5C1451121583553F0BCFBCE
:1061A000284607F0BBFC80B1284607F073FC0622A6
:1061B00038B104F59B411431BDE8384004480DF076
:1061C0002BB904F59A415831F6E738BDD08F00203D
:1061D000902B002010B5074B1A7A4AB100241C728C
:1061E00053F0E2FD22461121BDE8104053F094BB6C
:1061F00010BD00BFD08F00202DE9FF41054605F5F9
:106200009658684619F0EAF96946404613F004FBCF
:106210000646E8B137487AF00BF950B105F530532E
:10622000D3ED027AF5EEC07AF1EE10FA94BF0126B2
:10623000002605F5C140583007F070FC2E4C2F4F5A
:1062400000B146B1002328462380FB73FFF7C2FF4D
:1062500004B0BDE8F0812846FFF73CFFA0B36378A7
:106260007BBB23780133DBB2082B237002D140467D
:1062700013F0EAF92378092B02D1404613F0DCF938
:106280002378092B1DD94FF48573238053F08CFD9F
:106290000222102153F040FB8CF0A0F96368C01A71
:1062A00047F23053984209D905F54F50144A02215C
:1062B000283056F0E7FD8CF091F960602846FFF732
:1062C0005FFF6378FB73C3E72378002BF9D0013BB2
:1062D0006278DBB22370002AF3D0002BF1D1667014
:1062E00053F062FD3246102153F016FB2846FFF7AB
:1062F00071FFE6E7208C0020D08F00207D900020E9
:1063000020490D0810B500F5A044D4F85C35042BE5
:1063100001D1012010BD00F5C140583008F084F9CA
:106320000028F6D194F88805F4E7000073B500F56D
:1063300080450192A5F8381F04468CF04FF9C5F846
:106340003C0FD5F8200F03685B68984785F8360F37
:10635000D5F8200F03685B689847019A182818D869
:10636000DFE800F00D170D0D0D0D0D0D0D17521777
:106370005917595917414141171717415900334BC4
:1063800093F82A3403B304F59841043120460DF004
:1063900043F8D5F8200F95F8366F03685B68984787
:1063A00004F54F54864204F1280447D0D5F8200F55
:1063B00003689B689847264A03460421204602B09A
:1063C000BDE8704056F05EBD04F5005393F91432F9
:1063D000022BD8D0042B0BBF04F5984104F596414D
:1063E00020317431D2E704F5C043D3F89C33D9028D
:1063F00003D504F599412C31C8E704F59B419B0670
:106400004CBF30311431C1E720460192FFF77AFFCB
:10641000019A0028BDD104F50056019296F9143274
:10642000002BB6D0D5F8200F03685B68984785F835
:10643000360F96F91432019A022BCAE7054A042155
:10644000204602B0BDE8704056F01CBD908B002085
:1064500030490D0852490D08F0B5044604F5804650
:1064600085B00F4615465EF00FFDD6F8200FA6F852
:10647000387F03685B68984718281ED8DFE800F06B
:106480000D0D0D0D0D0D0D0D0D1D64810D0D70709B
:106490001D5252521D1D1D520D003D4BD3F85C255F
:1064A000012A21D104F5005393F81532023B012B48
:1064B0001AD904F5405383F8E423D6F8200F354A5F
:1064C000354B052D18BF1346026803939268904719
:1064D00004F54F5428340090039B304A0421204691
:1064E00056F0D0FC05B0F0BD2D4B93F82A343BB1EB
:1064F00004F598412A46043120460CF08DFFDCE774
:1065000004F5005393F91532032B03D1204605F00F
:1065100097F9D2E7022BEBD0042B2DD12A4604F5B4
:106520009941E9E704F5C043D3F89C33DA0223D458
:106530009B0604D504F59B412A463031DCE704F57F
:106540009B412A461431D7E72046FFF7DBFE00289F
:10655000B3D104F5C140583007F00AFB0028EED152
:1065600004F5005393F91532032BCFD0022BBFD083
:10657000042BD3D0012BA0D104F599412A462C310C
:10658000BAE704F5005393F91532042B95D1C5E70A
:10659000907B002068490D08282D0D0870490D08D2
:1065A000908B002070B500F54F5504462835124AEF
:1065B0000421284604F5804656F064FC0023A6F822
:1065C000383F04F5005393F85C31032B12D196F851
:1065D000361F302220460CF0F7FFD6F8200F036854
:1065E0009B689847054A034606212846BDE8704047
:1065F00056F048BC70BD00BF84490D089B490D088A
:1066000000F5405310B500220529044600F54F500F
:1066100083F8E42300F128000CBF054A054A042151
:1066200004F5804456F02EFC0023A4F8383F10BD3A
:10663000B4490D08C5490D08013A38B50446052A84
:106640003ED8DFE802F04A1B86118F0300F5C043F5
:1066500093F8EC3143B100F59B4104226C3143487F
:10666000BDE838400CF0D8BE04F5C04393F8EC31D7
:1066700023B104F59B4104221431F0E704F5804373
:10668000D3F8202F04F59B4314339A4225D004F508
:106690009B436C339A4220D004F5A043D3F85C3579
:1066A000042B1AD0324D95F8513FB3B1314905F55D
:1066B000AC5030F073F920B12F4B012283F88825BC
:1066C00038BD2C4905F5AC5030F068FC28B10422E7
:1066D00004F59941A5F58040C2E704F58043D3F85D
:1066E000202F04F59B4314339A42E9D004F59B43D1
:1066F0006C339A42E4D004F5A04304F5C14058300D
:10670000D3F85C5507F090FF0028D9D1042DD7D0DD
:1067100004F5005393F9DF31022B0DD004F59941B4
:10672000204604222C310CF077FE04F506501F3071
:10673000BDE8384048F0EABB0D4890F8513F002BC7
:10674000ECD00C4900F5AC5030F028F90028B3D15A
:10675000E4E700F5C140BDE83840012214211030C3
:10676000F7F716BABDE8384005F06AB8902B00205C
:10677000906B0020948B0020907B002070B52DED55
:10678000068B04468BF01EFF414BB4F8BE101A88EE
:10679000404E8A420546404A06D0198000233060A8
:1067A0001370BDEC068B70BD33683C49C31A8B4235
:1067B00065D9012313705EF067FC5EF01FFB356046
:1067C0005EF062FC5EF01AFB5EF040FB0428E8D944
:1067D0005EF05AFB204600210BF042F820460021D3
:1067E000B0EE40AA0BF046F820460121F0EE409AA8
:1067F0000BF00AFA00212046B0EE408A0BF044F874
:1068000004F5C1401030F0EE408A79F01BFE9FED98
:10681000249A0028B0EE4A0A4FF0040008BFB0EEF8
:10682000498A5FF043FFB0EE690A13205FF03EFF34
:10683000B0EE680A15205FF039FFB0EE680A1A2042
:106840005FF034FFB0EE480A46205FF02FFF0121D1
:10685000084660F037FAB0EE490A02205FF026FFE2
:10686000B0EE490A03205FF021FF20460BF00AFC3E
:10687000BDEC068B2046BDE870400CF059BB127889
:10688000002A8ED044F6206293428AD993E700BF53
:10689000DC8F0020E08F0020DE8F0020400D030001
:1068A0000000000000F5804200F59943D2F8202F47
:1068B0009A4204D100F5A04090F88805E8B10F4B4A
:1068C00093F85C0103F58043A0F12702012A93F8B5
:1068D00038340FD92C2809D00A2809D0A0F1310268
:1068E000504250410A2B18BF002070470120F9E7A1
:1068F000012070470A3B584258417047904B002096
:1069000008B500F5005393F8A02042B193F8DC30AD
:106910002BB1FFF7C7FF80F00100C0B208BD012016
:10692000FCE700002DE9F04700F50055AF4F95F862
:10693000DC80044600F5C1408AB0103079F078FD63
:10694000D7F85C35042B064642D1012104F50257E5
:10695000DFF8ACA22037384668F0D4FD9AF8383416
:106960000A2B814604D1002E54D100238AF83834F2
:1069700095F8A030002B59D195F9A6309C4D012BEC
:1069800003D0063BDBB2012B11D895F85C310A2B02
:106990000DD104F58046D6F8200F03681B6A98478E
:1069A00028B1D6F8241F2B2220460CF035FD9AF88A
:1069B00038340A2B04BF37238AF8383495F85C3111
:1069C0000A2B02D1372385F85C310AB0BDE8F08785
:1069D0000028BAD004F58043B7F8BE95D3F8200F4D
:1069E00003685B6898471428AFD004F5C14058305D
:1069F00007F068FC0028A8D14946A7F5A040FFF79A
:106A000019FA01460028A1D097F884154B1E594267
:106A100059419BE740EA0803DBB2002BA8D1AAF555
:106A2000C04000F0EFF800289FD0A1E7002ECCD0A6
:106A300004F5BE40343087F0A7FE0028C5D12046BB
:106A4000FFF730FF0028C0D1B9F1000F00F0BD8082
:106A500068494A46384668F02DF995F9A680B8F19C
:106A6000010F06D040F38580A8F10603DBB2012BAD
:106A70007FD85FFA88F8B8F1010F4DD104F5804254
:106A800004F59943D2F8202F9A4209D104F5A04386
:106A900093F8883523B195F8DF31013B012B94D968
:106AA00004F599410A222C31204606AE0CF0B4FCC4
:106AB000304618F093FD95F9B92092BBB8F1010F5B
:106AC0002FD004F5A048B5F9BA30D8F8F01FDFEDA3
:106AD0004A5AD1ED017A002BF8EEE77A52DD07EE43
:106AE000103AF8EEC76AE6EEA57A3046FDEEE77A90
:106AF00017EE901A18F078FD00233846CDE90433DC
:106B000068F09CFD04A969F0DDFA002857D0049BC9
:106B10000893059B099317E004F599410A22643113
:106B2000C2E72046FCF7FCFB07EE900A6F4604F52F
:106B3000C042043221463846B8EEE70AFDF740FD70
:106B400097E80F0086E80F0095F9A630012B10D0CA
:106B500031462046FDF76EF831462046FDF718FC19
:106B600095F9A630072B04D104F54054012384F88D
:106B7000E23353F019F94A4609210AB0BDE8F0475B
:106B800052F0CABED5ED2A6A95ED2D5A95ED2B7AB5
:106B900035EE076A36EEC57AB4EEC67AF1EE10FA33
:106BA00089BF37EE067A95ED907A27EE257AF6EED4
:106BB000006A94BFE7EE257AE7EE267A95E7D8F8E3
:106BC000F03F9A680892DB68A4E7B8F1000F3FF441
:106BD000FCAE95F8DC30002B7FF4F7AE04F54F5097
:106BE000064A0521283056F04DF9C2E7907B002077
:106BF000904B0020E0490D080000C842E9490D080B
:106C0000908B002010B5044600F5C140103079F09B
:106C100019FC98B104F5C140583008F0FBF960B98F
:106C200004F5AA4494ED187ADFED087AB4EEE77A19
:106C3000F1EE10FAACBF0120002010BD04F5AA440B
:106C400094ED187ADFED027AF0E700BFCDCCCC3DB1
:106C50006666663F70B500F5804600F59C43D6F841
:106C6000202F08339A42044600F5A04502D195F83A
:106C70005805D0B904F5C140B5F8BE15583006F036
:106C80008DF998B9D6F8203F04F59944A3420CD168
:106C900095F858354BB1D5F85C35032B05D1B5F8CF
:106CA000BE05A0F116035842584170BD0020FCE714
:106CB0002DE9F74F00F5804200F59943D2F8202FD7
:106CC0009A42044600F5A04504D100F5005B9BF90B
:106CD000B8313BB90023C5F84C3585F8493503B0C8
:106CE000BDE8F08F8BF07AFCD5F80465804636B1AC
:106CF000861B40F6C3139E4294BF00260126204601
:106D0000FFF780FF019028B1002785F848754FF004
:106D1000000A46E004F5C140103079F089FB814655
:106D20000028F1D004F5BE4A0AF1340A504687F033
:106D30002BFD0746002845D095F848A5BAF1000F6D
:106D40003BD156B304F5805041F27071D0F8B824AD
:106D5000002AB8BF52428A4206DCD0F8BC24002A7E
:106D6000B8BF52428A422BDD04F5AB4104F5C04066
:106D70004431043018F094FFDFED487AC5F84C85B3
:106D8000B4EEE70AF1EE10FA4FF000024CBF4FF0FC
:106D9000010A4FF0000AC5F85025012285F8482560
:106DA000374604F59070F7F745F8022832D9002FDE
:106DB00044D10023C5F84C3591E7019EB246ECE77B
:106DC0005646EAE7504687F0C7FC824648B1002E97
:106DD0009DD04FF4FA73C5F850354FF0000A4F4676
:106DE000DFE7D5F85C25012A07D0032AD9D1204650
:106DF000FFF730FF00288AD1E9E7DBED967AF5EE60
:106E0000C07AF1EE10FA82DD95F85835002B7FF448
:106E10007EAFDEE704F5F75604F50059083699F819
:106E20003610304610F0BAFB0028C2D099F8361060
:106E3000304610F0ABFC0028B9D1BAE7D5F84C05C4
:106E400010B9C5F84C854AE7D5F85025A8EB0008DD
:106E50009045FFF444AF95F84925002A7FF43FAFF1
:106E6000012285F849259BF8B811CB0705D504F513
:106E7000C1400C211030F6F78BFE04F54F5028303E
:106E8000BAF1000F06D0064A022103B0BDE8F04F68
:106E900055F0F8BF034A5146F7E700BF000096429D
:106EA000004A0D08164A0D082DE9F04F2DED028B12
:106EB000044685B0002304F5005903938BF08EFB44
:106EC000D9ED6D7AF5EEC07AF1EE10FAC4BF9FED00
:106ED000C67A67EE877A04F5907BC8BFFCEEE77A46
:106EE00080465846CCBF17EE907A9627F6F7A2FF59
:106EF000022840F2098194F8E4339FEDBC7AB02275
:106F000002FB0343D3ED777A67EE877AFCEEE77AEC
:106F100017EE903A9F428CBF00270127B9F9A8319C
:106F2000022BB8BF022307EE903AB8EEE78A03A916
:106F3000F6EE087A04F5965028EE278A12F04AFCFD
:106F4000054640B1DDED037AF4EEC87AF1EE10FAB1
:106F5000ACBF012500255846F6F76CFF012804F563
:106F6000A0461AD804F5C140103079F061FAA0B1FA
:106F70009DB906F5AC6393ED007ADFED9D7AB4EE32
:106F8000E77AF1EE10FA08DDDDED037AF4EEC87A67
:106F9000F1EE10FAACBF0125002504F5C1405830D0
:106FA00005F056FA8246002840F0FF8004F5C14003
:106FB000103079F03DFA002800F0058194F8E433B0
:106FC00004EB0313D3F890317BB158460193F6F7E5
:106FD00031FF012800F29A80019BA8EB030041F2E7
:106FE000873398428CBF00230123D6F8002502B1D5
:106FF0001BB9002D40F08C803D4604F5804204F51D
:107000009943D2F8202F9A421AD199F9E031002BF6
:1070100040F08680002386F84A35D6F85C35042B8C
:1070200000F0AF80072B00F0C280032B08D1204670
:10703000FFF710FE20B1002586F84955C6F8045523
:1070400096F84A3503B18DB907EE905A9FED697AEB
:10705000F8EE677A06F5AC6367EE877AD3ED006ADF
:107060009FED657AE6EE877AC3ED007A2046FFF75A
:10707000C9FD0546A0B196F86415C6F8008509B9A2
:10708000C6F8688504F5804204F59943D2F8202FAC
:107090009A4205D1D6F8043503B109B9C6F804857A
:1070A00096F88C3686F8645565F3C30386F88C36FB
:1070B00072F04EF9294672F027F9504B20465D7167
:1070C000FFF7F6FD2046FAF7CDFA35B199F85E31B3
:1070D0001BB98BF083FAC9F8600189F85E5120462C
:1070E000FFF790FD002840F08D8004F5C14010307E
:1070F00079F0A8F980F00100C0B286F86C0505B0FF
:10710000BDEC028BBDE8F08F002707E753466CE724
:1071100028F0DEFC27F02CFE00287FF46DAF6CE732
:107120005B4207EE903A04F69803F8EEE77A93EDA7
:10713000DB7AF4EEC77AF1EE10FA13DD012386F85C
:107140004A35C6F8548506F5AC63DFED2D7A93ED2C
:10715000007AB4EEE77AF1EE10FA7FF75EAFC3ED96
:10716000007A5AE796F84A35002B3FF456AFD6F826
:10717000543540F6B832A8EB030393423FF64AAFCA
:107180004BE704F5BE40343087F0E6FA00283FF4C0
:1071900057AF06F59E6393ED007ADFED197AB4EEF2
:1071A000E77AF1EE10FA7FF74BAF012548E706F5D5
:1071B0009E6393ED007AFEEE007AB4EEE77AF1EE8C
:1071C00010FAF2D43CE7D6F85C35002D18BF3D46E6
:1071D000012B01D1002533E704F5BE40343087F0A0
:1071E000B1FA0028F6D12BE70000B4420000C842F3
:1071F0009A99993E9A99193E9A99593F7D90002003
:10720000CDCC4C3E002078E700207047002070472E
:1072100001207047034BD3F85C05431E5842584188
:10722000704700BF907B002030B587B002A818F0EF
:10723000D5F93A4887F086FA20B139493948FCF740
:107240000BFD1FE0354887F087FAE8B1364C04F1B2
:107250002405234604F11002A4F11001A4F1D0008A
:10726000009587F09FFACDE90045A4F60C3292ED27
:10727000000A2E4904F11003A4F11002A4F1D00079
:1072800087F052FA07B030BD244802A987F0A2FA6D
:1072900008B102A9D2E7264CD4F8D03B002B0CDD74
:1072A00094F8703B4BB1A4F500501F49FCF7D4FC97
:1072B000A4F50050FCF71CF9E4E71A4804F058F96B
:1072C0000028BAD11B4C237D5B071FD4A36A002B77
:1072D000B3D0134AA2F12001A2F1100018F04CFC27
:1072E0000028AAD1144C0F48D4ED007AB7EE000A5A
:1072F00004F6183130EE670AFCF7DEFC094804F6A4
:10730000F82204F61831FCF737F8BBE7A4F5C040C3
:10731000FCF748FD0028B5D1D8E700BFC48A00209B
:10732000A48B0020902B0020948B0020E05700209D
:10733000904B0020908B00208C80002008B50A48DC
:1073400090F85132013B012B03D8A0F50050F8F71B
:1073500029F80648F7F7ECFE0448F7F7E3FFBDE825
:1073600008400248F8F744BB904B0020902B0020C7
:1073700010B5044607480CF045FF50B1064B93F892
:10738000190230B1236820469B6B984780F00100BA
:10739000C0B210BDA08E0020908B0020124B9842EE
:1073A00010B5044601D1002010BD03F11C0290422B
:1073B000F9D003F138029042F5D003F17402904203
:1073C000F1D0D4339842EED003681B6A984720B1BD
:1073D000064B93F8E233002BE5D1206907F03EF924
:1073E00080F00100C0B2DFE720770020905B002032
:1073F000174B984210B504460ED003F11C02904280
:107400000AD003F13802904206D003F17402904290
:1074100002D0D433984206D10E4B93F90902B0FA48
:1074200080F0400910BD03681B6A984718B10A4BE9
:1074300093F8E23343B9206907F010F930B12069BD
:10744000BDE8104009F0B0BC0020EBE70120E9E7FF
:1074500020770020904B0020905B002073B50F4EEA
:107460000D46114696F9A4211AB90124204602B00E
:1074700070BD036801915B69984704460028F4D108
:10748000D6F89C33019913F4802FEED00448054BB5
:1074900000682A46C06A25F011FDE7E7908B0020BE
:1074A0008C2B0020284A0D08084A0260084A4260D6
:1074B000111F816002F10801C160A2F1380102F5DB
:1074C0009C724261034A016182617047744A0D08EF
:1074D000A08C0020503E002008B503681B6E984722
:1074E0000648D0F8202F00F664439A4205D0BDE844
:1074F0000840A0F58040FEF797BD08BD906B0020C6
:107500002DE9F7435C4C04F59B6300221A60A4F557
:107510006073C11A4B42A4F500584B4188F8783685
:1075200004F59D63002584F8BC54A4F8125584F832
:10753000165584F8D45484F8495584F84A55C4F84B
:107540003C55C4F83855C4F83455C4F844551A604D
:10755000836904F58059D3F8FC31A4F80C3509F19E
:10756000040306460FCB04F6F47787E80F0084F88F
:10757000155584F82455C4F8D05F8BF02FF844F8E3
:10758000D80C336830465B6998474FF0FF3384F876
:10759000195588F8E45344F8A83C84F81805306974
:1075A00006F0F0F989F82D5084F817553368304605
:1075B000DB6D9847A4F580570546002858D03368FE
:1075C00030469B6B984784F85805D8F80406036842
:1075D000DB6B9847A4F5E4507BF0F4F8A4F5A040E9
:1075E0000AF090F8A7F5FB5067F0F2FF94F88835A1
:1075F000CBB1A4F5A040FFF705FBA0B909F19000BD
:1076000078F020FF78B9D7F8200F03685B6B9847B4
:1076100048B95CF097FA194A062155F033FC04F595
:10762000B0602FF067FA1648F6F7E0FE336993F979
:10763000CC206AB1586801A912F0CCF834699DEDEC
:10764000010A014604F18800FBF716FC84F84101A9
:10765000336830465B69984750B1336993F93C22EF
:10766000002A02DD93F8A03213B9002387F82D3FDA
:10767000284603B0BDE8F083907B0020344A0D0813
:10768000902B002070B503685B6E0E461546984738
:10769000044650B995F900303BB90548054B0068E0
:1076A0003246C06A294625F009FC204670BD00BF5D
:1076B0008C2B0020584A0D0810B50E4C20467AF04D
:1076C0007DFE04F5AC707AF0F5FB04F52C707BF0D0
:1076D00023FB094B03F5A042002182F8D41402F5E4
:1076E0009B62002103F500531160012283F8A82E4C
:1076F00010BD00BFEC5A0020902B002008B52DEDE6
:10770000028B1520B0EE408A5EF0D0FFB0EE480A42
:10771000BDEC028B1A20BDE808405EF0C7BF000038
:1077200008B5084890F909320121A0F5005033B19D
:107730000AF06AFABDE8084046205EF0B7BF0AF0DA
:107740008BFAF7E7904B002001207047012070472B
:1077500001207047012070470120704719207047B1
:1077600000487047DC4A0D0800487047EC4A0D0895
:1077700084B038B505AC84E80E00054614210C48E9
:10778000FCF700FA2A696423B2F9C01068B1032239
:107790005943204617F028FF05482146FCF7F8FD1D
:1077A000BDE83840012004B070470122F0E700BF77
:1077B000902B002013B50F4901AAA1F1100017F07A
:1077C000FBFF40B1DFED0C7A9DED017AB4EEE77A74
:1077D000F1EE10FA0CD8094CD4F8040603689B6B40
:1077E000984728B106492E22A4F540500BF014FE0C
:1077F00002B010BDA48B0020000000B4905B0020FC
:107800002479002030B51D4C0546D4F8240F0368B8
:1078100087B05B69984738B119491A482F220BF095
:10782000FBFD012007B030BD174806F017FF002808
:10783000F2D1A4F58054D4F8040603689B6B9847F2
:1078400028B1D4F8040603681B6C984798B10F4B15
:107850000FCB02AC84E80F00284601F06BF82868D3
:10786000059B009394E80E00446C2846A0472846E8
:10787000FFF7A0FFD5E7064BEAE700BF906B0020BB
:1078800024790020902B0020688C0020948B00200D
:10789000A48B002010B50446FFF78CFF2046BDE8FE
:1078A000104001F083B80000042070470048704782
:1078B000E1500D0800487047E1500D08037F73B197
:1078C000D0ED087AFDEEE77A17EE903A084AC2F852
:1078D0007035437F3BB1436AC2F8743570478369A2
:1078E000D3F8F831F2E78369D3F8FC31F4E700BF4D
:1078F000907B002008B50023838300F12801806974
:1079000011F07EFF012008BD70B56E4E2DED048B89
:1079100006F59E4304460121304693ED1C9ADFEDA7
:107920006A9A09F09DFF0121B0EE408A304609F0C5
:10793000A1FFC8EE297A06F50055A069B5F92C32E9
:1079400004F1280108EE903AF8EEE88AB5F92E32F3
:1079500068EEA78AC0EE297A08EE103AB8EEC88A17
:1079600028EE278A11F04CFF95F9323263B39FED70
:10797000577AF0EEE87AF4EEC77AF1EE10FA23D5F2
:10798000227FA369002A55D1012222770022226298
:1079900094ED087ADFED4E7AD3F8F8314D4A4E482F
:1079A00067EEC77A9FED4D7A67EE877AB0EE490AA7
:1079B000FDEEE77A17EE901A0B44C2F870350023FB
:1079C00001227AF08BFC08E0002343482377F0EE95
:1079D000490AB0EE680A7AF07DFC04205EF066FE8B
:1079E00095F9323243B19FED397AF0EEC87AF4EE70
:1079F000C77AF1EE10FA28D4002339486377F0EE05
:107A0000490AB0EE480A7AF0BFF813205EF04EFE45
:107A1000B5F93032002B03DD324E96F9223263BBCA
:107A200028482021F7F71CF8002843D1254809F001
:107A300039FD42E0D3EDC56A96ED467AD4ED087A79
:107A4000E6EE877AC4ED087AA2E7637F2BB90123BB
:107A50006377A369D3F8FC3163621E4B616AC3F894
:107A60007415A369D3F8FC010023091A1A461C48AF
:107A7000B0EE490A7AF06EF9C7E70121A6F5405049
:107A800009F002FF80EE297AB5F93032002106F5BF
:107A9000037007EE903AF8EEE77AF0EE490A27EE27
:107AA000870A7BF039F8BDEC048B2046BDE87040B6
:107AB000FFF724BE0348F7F707FE07EE900AB8EE7B
:107AC000E70AF0E7902B002000A08C45000000346E
:107AD000E02E6542907B0020EC5A00200000C84256
:107AE000445C0020905B00202DE9F04F2DED0C8BC5
:107AF000DFF8A8A39FEDDEDA9FEDDE9A97B00AF5D6
:107B00009E4300F1280504460121504693ED1CBA1E
:107B100009F0A6FE01215046F0EE408A09F0AAFEC7
:107B200001215046B0EE408A09F0AEFEDFEDD27A78
:107B300088EEA77A0AF5005601A8B6F92C320AF5A4
:107B4000A04B0AEE903AF8EEEAAAB6F92E32DFED33
:107B5000CB8A6AEE87AA88EE277A0AEE103AB8EE48
:107B6000CAAAB6F930329FEDC68A2AEE07AA80EE7D
:107B7000277A09EE903AF8EEE99A6AEE8D7A69EE84
:107B8000879AF0EEEACAF4EEC8CACDED017AB0EEFB
:107B9000CACA6AEE0D7AF1EE10FAF0EEE9BAB4EE66
:107BA000C8CACDED027A58BF4FF0010969EE8D7A4F
:107BB00048BF4FF00009F1EE10FAF4EEC8BA9AEDA2
:107BC000460ACDED037A54BF4FF001084FF000088C
:107BD000F1EE10FA54BF012700272BF017FE01A980
:107BE00028462BF0BDF828462BF0B4F928462BF098
:107BF00023F920EE090A284620EE280ABDEEC00A25
:107C000010EE103ACBF870352BF030F920EE090A5F
:107C100020EE280ADFED9B8ABDEEC00ACDED0D8A6D
:107C200010EE103ACBF874350DF1280B4FF07E535F
:107C30005946A0690A93CDED0C8ACDED0B8A11F05F
:107C4000DFFD0021504609F0DFFFB0EEC00AB4EEC0
:107C5000C80AF1EE10FA16D55046FEF7D3FF90B9D8
:107C6000F4EEC8CAF1EE10FA0DD5B4EEC8CAF1EEC2
:107C700010FA08D5F4EEC8BAF1EE10FA44BF9BE84A
:107C80000F0085E80F000AA82BF0C8F9294612A8B2
:107C90008DED141A8DED120ACDED130ACDED151AE6
:107CA0002BF0CEF90DF1100A51460EA88DED101AE9
:107CB000CDED048ACDED058ACDED068A8DED0E0A57
:107CC000CDED0F0ACDED111A2AF084FFB6F92C3252
:107CD000DFED6D7A01EE103AB6F92E3209EE103A68
:107CE000B6F9303208EE903AB8EEC11AB8EEC99A39
:107CF000F8EEE88A21EE271A29EE279A68EEA78A7D
:107D0000F4EEC8CAF1EE10FA21EE0D1A29EE0D9A22
:107D100068EE8D8A07D594F83830DFED5A7A002B5B
:107D200018BFB0EE671AB4EEC8CAF1EE10FA07D564
:107D300094F83930DFED537A002B18BFB0EE679A14
:107D4000F4EEC8BAF1EE10FA07D594F83A30DFED48
:107D50004D7A002B18BFF0EE678A9AE807000DF104
:107D60001C0B8BE80700F1EE410AC2209DED070ACB
:107D700028F0EAFBC3208DED070AB0EE491AF1EEB8
:107D8000490A9DED080A28F0DFFBB0EE681AF1EE13
:107D9000680A8DED080AC4209DED090A28F0D4FB7D
:107DA000514658468DED090A2BF0C6FC12A928460B
:107DB0008DED120ACDED130A8DED141A06F57666D7
:107DC0002AF0CEFF28462BF0C5F8DDED076A96EDC8
:107DD000007A2E4B9FED270AC6EE877A5846DDEDD6
:107DE000086ACDED077AD3ED2E7A86EEA77ADDED1F
:107DF000096A8DED087A86EEA77A8DED097A2BF067
:107E000005FDB9F1000F01D0CDED07AAB8F1000FC3
:107E100001D08DED08AA0FB1CDED099AF0EE4B0A15
:107E20009DED070A1A487AF055FA04205EF03EFCF0
:107E3000F0EE4B0A9DED080A164879F0A5FE1320D6
:107E40005EF034FC0021F0EE4B0A9DED090A124869
:107E50007AF062FE2046FFF751FC84F8389084F8EF
:107E6000398084F83A7017B0BDEC0C8BBDE8F08F08
:107E700035FA8E3CE02E654200A08C450000C842D9
:107E80000000003400000000CDCC4C3E905B002090
:107E9000EC5A0020445C00209C5D0020902B0020C8
:107EA00010B50446FFF73CFC0B4B93F93222022A33
:107EB0000DD1B3F93022002A09DD03F5805393F97F
:107EC000223223B12046BDE81040FFF70DBE204608
:107ED000BDE81040FFF718BD904B00200A20704706
:107EE00000487047EE700D0800487047EE700D08AE
:107EF0000120704701207047012070470120704722
:107F0000034BD3F85C05031F58425841704700BF2C
:107F1000907B002070B505462C48D0F8242F00F641
:107F2000E4439A4215D12B6993F844318BB100F5A3
:107F3000AC502EF0A9F9044658B95BF003FE244A70
:107F4000032154F09FFF2B69012283F8432120462F
:107F500070BD204C94F8EC3123B194F9A4319A1EF1
:107F6000534253411C4E86F81835231D0FCB06F69D
:107F7000F475143485E80F0084E80F0006F5B0604E
:107F80002EF0F8FF154B1C68E56A2B6828465B68E5
:107F90009847B0B195F84D309BB1E36A9B8F83B1A0
:107FA0005BF0D0FDE36A0E4A9B8F062154F06AFF16
:107FB000E36A06F5B060998F2EF0C8FDE36A0022EF
:107FC0009A87084887F040FB0124C0E7906B0020A7
:107FD000D44B0D08908B0020907B00208C2B002030
:107FE000EE4B0D087855002038B50D4C94F88435CB
:107FF000012B10D104F5B0602CF0A2F8B4F8BE55F6
:108000000848294605F022FD28B9152D03D104F6AC
:10801000347086F077FC0023C4F8043538BD00BF07
:10802000907B0020688C002008B511F003FE90F8CA
:108030007C32DB0704D5BDE8084002482EF036BE8E
:1080400008BD00BF1081002038B5344C94F8843549
:10805000012B0ED0A4F555710822A4F5A0400BF019
:10806000DBF95BF06FFDBDE838402D4A062154F086
:1080700009BF2C48B4F8BE5505F00CFD20B1BDE891
:108080003840284808F03ABE162D05D0152D36D1B7
:10809000D4F85C35072B0AD123480CF0D5FF2248D1
:1080A0000DF01EF9BDE838401F480DF02FB8A4F5BB
:1080B000A040F7F72DFEA4F5A040F7F709FDA4F5C1
:1080C0004053D4F8701593F9702264235A4304F690
:1080D000347086F073FBC4F8700504F6347086F0D3
:1080E000AFFC30B1BDE838409FED100A46205EF08D
:1080F000DDBAA4F5A040BDE83840F7F7CDBA1E2D93
:1081000018BF4FF0FF33084818BFC4F8D034F7F752
:10811000FFFD0548F7F7DCFC0348ECE7907B002007
:10812000084C0D08688C0020902B002000000000F7
:1081300070B5134890F9A4310E46154613B90124C1
:10814000204670BDD0F89C335B0311D5A0F5805359
:10815000D830B3F8BE1504F021FF044640B9094BEE
:108160000948006832462946C06A24F0A7FEE7E7BE
:1081700006482EF089F804460028E0D1044BEFE7CA
:10818000908B0020344C0D088C2B00201081002097
:10819000484C0D0810B5144BB3F8BE35532B0446AC
:1081A0001ED10AF045F99FED110A46205EF07EFAD5
:1081B0009FED0E0A49205EF079FA9FED0C0A4A20E5
:1081C0005EF074FA46205EF051FB49205EF04EFBF3
:1081D0004A205EF04BFB2046BDE81040FFF76CBA2A
:1081E000BDE81040FFF7AAB8907B00200000000017
:1081F0000820704700487047D44C0D08004870476D
:10820000E04C0D080120704708B50248FDF7ACFEB0
:10821000012008BD902B0020014800F061B900BF8B
:108220009477002010B50446FFF788F82046BDE893
:108230001040FFF775BA00000120704700487047F2
:10824000584D0D0800487047604D0D0801207047DB
:108250000120704710B5044B03F1140404330FCB15
:1082600084E80F00012010BD908B002008B50B485A
:1082700000F5A04200F500530321D3F8403C93FBE6
:10828000F1F3C2F87035F7F787FC0448F7F720FCE4
:10829000BDE808400148F7F7FFB900BF902B002068
:1082A0000720704700487047E52E0D0800487047CA
:1082B000D84D0D08012070470120704701207047FC
:1082C0007047000008B5002303774362034887F036
:1082D000BBF90348FBF782FC012008BD785500205C
:1082E000902B002010B5194CD4F8283CB3F9083075
:1082F00023B9D4F8343CB3F90830F3B10023037741
:108300004362D4F8280C5CF0AFFF04F54463D3ED6E
:10831000007A0F48F8EEE77A27EE800ABDEEC00A31
:1083200010EE103AC0F87035A0F5A040F7F734FC15
:10833000BDE81040074803F01BB8037F002BE0D0D6
:10834000A4F50050F7F7E4FCF2E700BF904B0020E3
:10835000907B0020902B00202DE9F0412DED048B27
:108360004F4DDFED507A95F8E4339FED4F9A9FED36
:108370004F7AB02606FB035393ED788A28EE278ABE
:1083800005F5A653BDEEC88A93ED030AF8EEC87A48
:10839000044667EE897A97EE870A28F0C1F8237FB2
:1083A000F0EE408A002B64D105F50053D3F8283C49
:1083B000B3F90830002B5CD1284609F073F8002887
:1083C00057D195F8E43395F8281406FB035393F836
:1083D000C12100294DD1012A4BD993ED777AF0EED6
:1083E000087AB4EEE77AF1EE10FA42DBDFED307A8C
:1083F000B0EEE80AB4EEE70AF1EE10FA39D5636A96
:10840000A3B38AF0EBF8636AC01AB0F5FA7F34D8E8
:10841000237F002B3FD0274FA7F10C0595E80F00D5
:1084200007F1140686E80F0094ED088A391D2846E6
:10843000B8EEC88A17F034FC28EE098ADFED1E0A70
:10844000304670EE200AA7F54057B0EE480A17F004
:10845000CDFCBDEC048BD7F804069FED180A036829
:10846000324629469B6ABDE8F04118478AF0B6F8C3
:108470006062636A002BCBD0C3E70123237700231C
:1084800063620C4B84ED088AA3F10C0504330FCB17
:1084900085E80F00BCE7BDEC048BBDE8F08100BFB0
:1084A000902B00200000C8420AD7233C35FA8E3CAE
:1084B000DB0FC93F908B002000007A4400000000D1
:1084C000036A0B60007F70470520704700487047C3
:1084D000504E0D0800487047604E0D08012070474F
:1084E00038B54B4D2DED028BD5F8280C9FED498A00
:1084F0005CF0BAFED5F8403C07EE903AF8EEE77A29
:1085000005F5405427EE800AA5F50050BDEEC00ADF
:1085100010EE103AC4F87035F7F73EFBD5F82C0C86
:108520005CF0A2FEB5EEC00AF1EE10FADABF05F675
:108530004443D3ED007AD5ED707A3748CBBF20EEB7
:10854000270A20EE270A20EE080A28EE400ABDEE90
:10855000C00A10EE103AC4F87435F7F7E9FA95ED51
:10856000707AD4F8740505F6444327EE087AD3ED03
:10857000007A27EE888AFDEEC77A17EE902AFDEE84
:10858000C87A17EE901A28F07FF8C4F874052248CC
:10859000FDF776FD20B1D4F874355B42C4F874352C
:1085A0001E4B93F8343F63B195F91432022B08D176
:1085B000002301214620C4F87035C4F874355EF0FC
:1085C000D9FB5CF061FD5F215DF022FDE8B15DF05B
:1085D000EFFC022819D194F81535B3B904F59D6361
:1085E00093ED007AD5ED987AB4EEE77AF1EE10FAD1
:1085F0000BD5012384F81535BDEC028B084A0948D8
:10860000BDE83840042154F03DBCBDEC028B38BDC0
:10861000904B00200000C842902B0020906B00205F
:10862000684E0D08785F002010B50446FEF786FE00
:108630002046BDE81040FFF773B8000006207047E1
:1086400000487047E84E0D0800487047F84E0D0886
:1086500001207047012070470120704701207047BA
:108660007047000008B5044886F0EEFF0348FBF7AA
:10867000B5FA012008BD00BF78550020902B0020DE
:1086800038B50F4C04F50055D5F8280C5CF0ECFD1E
:1086900004F53152D2ED007AF8EEE77A04F5A04302
:1086A00027EE800A2046BDEEC00A10EE102AC3F85D
:1086B0007025F7F771FA2046BDE8384002F058BE41
:1086C000902B00200F20704700487047704F0D0816
:1086D00000487047784F0D0801207047012070470F
:1086E000012070470120704701207047012070472A
:1086F00030B5184B2DED028B002283F8E22303F5F1
:108700004053043305460FCB85B06C4684E80F0018
:10871000114804F001FC90B1A86900F57F702AF0BF
:10872000A5FE0D48B0EE408A04F05EFCF0EE400A73
:108730009FED0A0A204628EE000A17F057FB002397
:108740000748EB612146FBF723FE012005B0BDEC95
:10875000028B30BD905B0020688C0020E02E6542CB
:10876000902B002038B5424C94F819354BB104F5E4
:10877000805393F8EC3123B1BDE838403D4808F010
:108780008FBAD4F83435002B18DC3B48F7F7C0FA21
:10879000D4F83835002B29DC3748F7F799F93748F2
:1087A00090F8E233002B46D00121A0F5405009F0AB
:1087B0002BFABDE8384046205DF078BF89F00EFF07
:1087C000D4F83435C01A40F6B7339842DDD82C4D72
:1087D000D4F82805D5F8402C514227F055FFC4F8AD
:1087E0007005A5F50050F7F7D7F9D1E789F0F6FE47
:1087F000D4F83835C01A40F6B7339842CCD8204B5D
:10880000DFED206A93ED707AD4F82C0503F644432B
:10881000D3ED007A27EE267A67EEA67ABDEEC77A08
:10882000FDEEE77A17EE102A17EE901A27F02CFFCC
:10883000C4F87405B3E7A0F5805090F99F31012B7F
:1088400004DCBDE838400C48F6F726BFD4F84435C0
:10885000002BF6D089F0C2FED4F84435C01A40F699
:10886000B7339842EDD804F5A86494ED000AA0E768
:10887000907B0020688C0020902B0020905B0020D3
:10888000904B00200000C842D0ED077A0348FCEE70
:10889000E77A17EE903A99B202F06ABF902B002067
:1088A00084B010B503AC84E80E000B4821466F225B
:1088B000FBF7BEFC9DF80C1011F0040102D120461C
:1088C00016F056FF04482146FBF762FDBDE8104054
:1088D000012004B0704700BF902B0020B0EEC00A0A
:1088E000FDEEC07A38B54FF6FF7205460C4617EE1E
:1088F000900A002127F0C8FE07EE900A002CF8EE3F
:10890000E77A054BC5ED077A14BF4FF0FF3201221D
:1089100083F8CC2F38BD00BF907B0020FEF784BCCD
:108920000C2070470048704751520D0800487047AE
:108930005A930E0808B50C48FCF76EFA0A480B4922
:10894000FBF778F90848F6F713FB40B106484FF4F7
:108950008051F6F785F810B10348FBF73FF902485C
:1089600002F0DEF9012008BD902B0020A48B00202E
:1089700008B50D48F7F7CCF90B48F6F7F9FA50B1FE
:1089800009484FF48051F6F76BF820B1BDE8084074
:10899000054802F0EDBC0448F7F79AF8BDE8084036
:1089A0000148F6F779BE00BF902B002008B50948B2
:1089B0004FF48051F6F754F828B107480022416A75
:1089C000143016F011FEBDE808400248002102F004
:1089D000CFBE00BF902B0020908B0020881A10B5CE
:1089E00027F07AFD104BD3F8C82F0028B8BF4042BB
:1089F000002AB8BF524248F6A041B2FBF1F24FF450
:108A00007A7102FB011188420CDC03F580531A7D58
:108A1000D20605D503F1140404330FCB84E80F000C
:108A2000012000E0002010BD907B002013B504461B
:108A30008069019100F57F702AF018FDDFED0A7A58
:108A400020EE270A27F0EAFCDFED087A019920EEF4
:108A5000270A2046FDEEC07A17EE902A02B0BDE844
:108A60001040FFF7BBBF00BFE02E65420000C842C8
:108A700084B070B52DED048B86B00FAD85E80E0087
:108A80004E4CDFED4F8A0646D4F8040604F5005438
:108A900004F57E6393ED000A0368B0EEC00A5B6ADA
:108AA0009847B4EEE80AF1EE10FAB0EE408A07DA21
:108AB000012006B0BDEC048BBDE8704004B07047E7
:108AC0004049284616F0F8FF02A8CDED030A8DEDC7
:108AD000020A2AF09BFD04A88DED040AB0EE480AB4
:108AE000CDED050A2AF04EFC13A928468DED000AAB
:108AF000CDED010A16F0E0FF02A88DED020ACDEDE2
:108B0000030A2AF0FDFCB4EEE80AF1EE10FACFDB1E
:108B1000B4EEC08AF1EE10FA9FED2B9ADFED2B8AAE
:108B2000DFED2B9A2BD802A869462AF01BFC04A87B
:108B30008DED040ACDED050A2AF098FC684620EE7A
:108B4000098A2AF093FC94F9CC3F07EE903AF8EEAC
:108B5000E77A28EE288AA7EEA90A27F0E1FC20EEA2
:108B6000090ABDEEC88A20EE280A18EE101AFDEE9A
:108B7000C07A304617EE902AFFF730FF99E738EEBB
:108B8000400A38EE088A80EE080AAFF0C5F902A85C
:108B9000B0EE408A2AF06AFC94F9CC3FF0EE007AFD
:108BA000B0EE697AA8EE677A07EE903AF8EEE77AC7
:108BB000A7EE270A27F0B4FCC0E700BF905B0020B7
:108BC00000000034948B0020E02E65420000C84273
:108BD000DB0FC93F10B504460848F6F7C9F920B9BC
:108BE0002046BDE81040FEF71FBB04484FF48051FB
:108BF000F5F736FF0028F3D010BD00BF902B002002
:108C0000002070470048704760500D0800487047CA
:108C100068500D0800207047036993F8140118B1DB
:108C2000D3F8C402C0F380107047000038B5154C6B
:108C300005460021204608F013FE04205DF036FDB5
:108C40000021204608F016FE13205DF02FFD0021C4
:108C5000204608F019FE2846FEF750FD2046012167
:108C600008F0D2FF46205DF021FDAB6904F5A04479
:108C7000D3F8F831C4F87035AB69D3F8FC31C4F8D7
:108C8000743538BD902B0020FEF716BD17207047B5
:108C900000487047E0500D0800487047E8500D0844
:108CA00001207047012070470120704710B503690B
:108CB000002283F8402103690446D3F83C0103688D
:108CC0009B689847A368186880F082F8206904F0D0
:108CD0009BFE0349A06910F093FD012010BD00BF69
:108CE000807700201FB50D4C9FED0D0A04F5C043A1
:108CF00004F5A044D3F80C016C302AF033FDFDEEEE
:108D0000E00ABDEEC00A10EE903AC4F8743510EED9
:108D1000103AC4F8703504B010BD00BF902B00208D
:108D20009F0CB34530B52DED028B83B0044689F01E
:108D300055FC0146206900F50E700BF0ADF938B115
:108D4000204603B0BDEC028BBDE83040FEF7F6BA1A
:108D5000206990F84031BBB1012104F0DBFDA3682C
:108D6000DFED400A1868036801215B6EB0EE600A0F
:108D70009847206903F030FA3B4803B0BDEC028B02
:108D8000BDE83040FFF78CB8384DDFED398A02215D
:108D900004F0C0FDD5F82C0C5CF066FA2369D3ED25
:108DA000390A93F93C2220EE200A002A60EE280AB4
:108DB0003FDD93F8A032002B3BD0D5F8340CCDED3D
:108DC000000A5CF051FA2369D5F8280C93ED3A8A31
:108DD00020EE080A20EE288A5CF046FA236993ED1B
:108DE000381A20EE410A20EE281ADDED000A20692B
:108DF000CDED010A8DED001A03F02AFAA36895F96A
:108E0000322218689DED001ADDED010A0368F0EECC
:108E1000408A2AB31B6CB0EE480A9847A3681868CA
:108E20000368F2EE040A5B6E0021B0EE680A984710
:108E3000A2E7D5F8280CCDED000A5CF015FA2369FD
:108E4000D5F8340C93ED388A20EE080A20EE288AF3
:108E50005CF00AFA236993ED3A1A20EE010AC2E7A0
:108E6000DB6BD8E70000000058770020904B002013
:108E70000000C842122070470048704760510D083A
:108E80000048704768510D08012070470120704765
:108E90000120704738B52DED028B43689FED1C8A89
:108EA0001D680446006904F0D5F9236993ED131A8F
:108EB000D3ED110A434200EE103A21EE081A60EE9B
:108EC000880AB8EEC00A284681F03CF96368206938
:108ED0001D6804F0BFF9236993ED131AD3ED110A4D
:108EE000434200EE103A21EE081A60EE880AB8EE0E
:108EF000C00A284681F0A0F99FED060A206903F018
:108F000097F9206905F03AFFBDEC028B012038BDCE
:108F10000000C84200000000014800F073BE00BF1E
:108F2000CC78002013B5044600698830FAF704F9BC
:108F300089F054FB0146206900F50E700BF0ACF887
:108F400028B1204602B0BDE81040FEF7F7B920690D
:108F500090F840313BB3012104F0DCFCA368DFED65
:108F6000170A18680368B0EE600A5B6E0121984723
:108F7000206903F031F963689FED100A186882F0E8
:108F80000BFB0F48F6F7D4F80D48F6F7CBF920465F
:108F90009FED0A0AFEF7B2FB2069883002B0BDE8F7
:108FA0001040FAF787B9074804F018FE20690190CD
:108FB00004F0B6F9019806F0EDFAE2E700000000CF
:108FC000902B0020688C00201420704700487047C8
:108FD000E64A0D08004870476D930E08012070475F
:108FE0000020704770B504460E4800F03BF8236936
:108FF000002583F84051206904F0CEFF6069052107
:1090000003F08CFD084826690221FAF791FC86EDF1
:10901000B70A2369C3F848512369C3F84C510120AA
:1090200070BD00BF04790020902B0020014800F0A3
:10903000E9BD00BFCC780020014800F069B800BF4E
:1090400004790020132070470048704750520D08E3
:109050000048704758520D080120704701207047A2
:109060000120704738B52DED028BDFED240AC3686F
:109070009FED238A0446B0EE600A18687DF02AFA54
:10908000E36818687DF004FB636820691D6804F0DC
:10909000E1F8236993ED131AD3ED110A434200EE70
:1090A000103A21EE081A60EE880AB8EEC00A284687
:1090B00081F048F8636820691D6804F0CBF82369E3
:1090C00093ED131AD3ED110A434200EE103A21EE4C
:1090D000081A60EE880AB8EEC00A284681F0ACF89B
:1090E000206905F04BFE256989F078FAC5F86C0116
:1090F000BDEC028B00230120E36138BD00000000BD
:109100000000C842014800F07DBD00BFCC780020BF
:1091100030B52DED048B0446006985B08830FAF730
:109120000BF838B1B64805B0BDEC048BBDE8304053
:10913000FFF7F8BE89F052FA05462069294600F586
:109140000E700AF0A9FF38B1204605B0BDEC048BC3
:10915000BDE83040FEF7F2B8206990F8403163B3C3
:10916000012104F0D7FBA368DFEDA60A18680368A5
:109170000121B0EE600A5B6E9847206903F02CF87D
:1091800063689FEDA00A186882F006FADFED9D0A79
:10919000E368B0EE600A18687DF09CF9E36818682F
:1091A0007DF076FA9848F5F7C3FF974805B0BDEC17
:1091B000048BBDE83040F6F7B5B8C36A93F8CB30FE
:1091C00013B99248FFF74EFF206903F06BF918B10D
:1091D000E36818687DF07AF92369D3F86C31EB1AEB
:1091E000B3F5FA7F0BD9E368DFED860A1868B0EEB5
:1091F000600A7DF06FF9E36818687DF049FA236929
:109200009FED838AC3F86C510221206904F082FB30
:10921000636820691D6804F01DF8236993ED131A33
:10922000D3ED110A434200EE103A21EE081A60EE27
:10923000880A2846B8EEC00A80F084FFD4E90335D6
:1092400018687DF0B1F9A368186803689B6EF0EEAA
:10925000408A984703AAF0EE400A02A9B0EE680AD5
:10926000284603F039F8E368DDED030A18689DED40
:10927000020A7DF02FF96368186880F055FF18B96D
:109280006368186881F046FEE368624D1868012142
:109290007DF06AFBE36860481B689B68D3EDCF7A7A
:1092A000FDEEE77A17EE903AC5F87035E3681B6873
:1092B0009B68D3EDD07AFDEEE77A17EE903AC5F8C9
:1092C000743504F08BFC2369D3F83C01036805F284
:1092D00074525B6B05F5AE61984748B163681B68D3
:1092E000D3F88823C3F89423D3F88C23C3F89823A6
:1092F0002069DFED4A9A04F081FBD5F870352069CA
:1093000007EE903A012105F27453F8EEE78A93EDE7
:10931000009A06F0D9F8A368B8EEC99A186820EE4A
:10932000290A036868EEA98A29EE299ADB6A20EEE9
:10933000081A69EE080A28EE880A9847384BD3F8CD
:10934000202F03F694518A4248D1636993F8643020
:10935000062B0AD8206903F0F1FC30B160690721BF
:1093600003F0DCFB206904F017FE27480221FAF71E
:10937000DFFA206903F0C2F8636993F86430072BC1
:10938000B0EE408A08D12369D3F8C4329B0403D4D9
:10939000A069012110F0FAFE6368B5EEC08AF1EE13
:1093A00010FA1868CCBF01210021B1EE480A80F004
:1093B0004FFF206907F002FE206903F069FF1248A1
:1093C000F5F7B6FE1048F5F7ADFF9FED0E0A204603
:1093D000FEF794F905B0BDEC048B30BD03F6E44311
:1093E0009A42206907D190F8423123B19FED050AD6
:1093F00002F01EFFE0E7019003F092FF0198F7E70B
:10940000E878002000000000902B00200479002064
:109410000000C842907B0020688C00200AD7233CC3
:10942000906B00201520704700487047D0520D08FF
:1094300000487047D0520D08012070470120704746
:1094400000207047C369012B06D1044B93F8AC028E
:10945000431E58425841704700207047908B0020AF
:109460000E4BB3F9D221B3F9043207EE102A07EEFE
:10947000903AB8EEC77AF8EEE77AB0EEC77AF0EE37
:10948000E77AB4EE677AF1EE10FAC8BFF0EE477AE9
:10949000B7EE080A27EE800A704700BF904B002005
:1094A0002DE9F043844D2DED048B95F81C928BB083
:1094B0000446B9F1000F0BD080493122A5F5C04018
:1094C00009F0AAFF01200BB0BDEC048BBDE8F083CE
:1094D0000123C3612E1D96E80F00A5F10C0787E854
:1094E0000F00236955F8102CB3F8C070DB6A52687E
:1094F00093F8A0306421022B17FB012740F0B680BF
:1095000007EE907A3246B8EEE70AA5F5C04106A804
:10951000FBF756F806A9304616F0C2FB2046F0EEDF
:10952000408AFFF79DFF2369B3F9C020D3ED310ACC
:1095300001EE102AB3F9C220B0EE409A00EE102AD4
:10954000B8EEC11A1A20B8EEC00A26F0FDFF236952
:10955000B3F9C030F4EEC98A07EE903AF1EE10FA92
:1095600054BFF0EE686AF0EE496AB8EEE77AC8EEEA
:10957000A67A236820465B68B0EE408A67EE877A59
:10958000B4EE670AF1EE10FA48BFB0EE678A98476A
:109590000146A5F5C040FAF7F5FA082102468046D3
:1095A000A5F5C040FAF776F9DFED457A38EE408A46
:1095B000B4EEE78AF1EE10FA31DBC4F81C9096E8BD
:1095C0000F0005F1140484E80F009FED3E9AB8F1F6
:1095D000000F14D005AA0321304616F03BF870B1F5
:1095E000DDED057AF8EEE77A0322E8EE097A204607
:1095F000FDEEE77A17EE901A15F0F6FF62E7D5ED6B
:10960000028A3148F8EEE88A16F018F8E8EE098A7E
:1096100002462E48FDEEE87A17EE901AECE7F4EEDB
:10962000C98AF1EE10FA21D505AA4946304616F04E
:1096300011F818B1059B9F42A8BF1F465AF082FA45
:10964000064619EE100AF2F75FFFCDE9020118EEA7
:10965000900AF2F759FF1E4ACDE900010621304673
:1096600053F010FC6069032103F058FA3946194899
:10967000FAF75EFF206903F0D7FC134805AA002122
:1096800015F0E8FF68B96269AB68A9698B4292F886
:109690002010D4BF0023012363F3000182F82010BF
:1096A00010E70A4806AA002115F0D4FF0028EAD0E6
:1096B000DDE905316269E9E7908B0020247900201B
:1096C000000000340000C842948B0020A48B0020CE
:1096D000D8520D08902B0020014800F093BA00BF2B
:1096E000CC780020F0B52DED028B99B0044688F0BF
:1096F00075FF0146206900F50E700AF0CDFC0546A5
:1097000038B1204619B0BDEC028BBDE8F040FDF742
:1097100015BEE36983B1012B00F01E81A048F5F767
:1097200007FD9F48F5F7FEFD9D4819B0BDEC028B83
:10973000BDE8F040F6F75CB99FED9A8A60688DED60
:10974000098A8DED0A8A8DED0B8A8DED0C8A0BAAA4
:1097500009A901230068944E80F00AFC2069B0EE4C
:10976000480A03F025F9636890481B68D3EDCF7A67
:10977000FDEEE77A17EE903AC6F8703563681B681D
:10978000D3EDD07AFDEEE77A17EE903AC6F874354D
:1097900004F024FA2369D3F83C01036806F27452FA
:1097A0005B6B06F5AE61984748B163681B68D3F8F8
:1097B0008823C3F89423D3F88C23C3F89823206913
:1097C00004F022F9A36820691D682B68DF6AD6F8C7
:1097D000703507EE903AD6F87435F8EEE78A07EE62
:1097E000903AF8EEE70ACDED050A05F0E1F8DDED77
:1097F000050AB0EE401A2846B0EE680AB84720695C
:10980000C36B93ED070A02F013FD206903F040FDDE
:1098100063688DED0D8A8DED0E8A8DED0F8A1868C7
:109820000FA980F0F7FE0D9B14930E9B1593022257
:109830000F9B169314A910A816F0A8FA5C4907AA62
:1098400010A815F0B9FF48B1DFED5A7A9DED077AFF
:10985000B4EEE77AF1EE10FAFFF660AF564D012351
:10986000E36195E80F0006F6F47787E80F00D6F875
:10987000F03F22695B68B2F8C0604949642216FB78
:10988000023607EE906A2A46B8EEE70A14A8FAF7FD
:1098900097FE284614A916F003FA2046B0EE408A37
:1098A000FFF7DEFDB4EEC08AF1EE10FAF0EE408A6A
:1098B000A5F1040722D508AA002105F1100015F032
:1098C000C9FE18B1089B9E42A8BF1E465AF03AF93D
:1098D000054618EE900AF2F717FECDE9020118EEE0
:1098E000100AF2F711FE354ACDE90001062128469B
:1098F00053F0C8FA6069032103F010F93146284893
:10990000FAF716FE206903F08FFB294907AAA1F197
:10991000100015F051FF636988B19DED077ADFED06
:10992000257A93F82020B4EEE77AF1EE10FAACBF76
:109930000121002161F3000283F82020EEE6BA68DD
:10994000B9698A4293F82010D4BF0022012262F341
:10995000000183F82010E1E6206906F085F86369CC
:1099600093F86430042B07D90F4B1148D3F8F03F1C
:109970002A46596815F038FE636993F86430032B62
:1099800002D9206907F05AFB236993F8D431013BCF
:10999000012B3FF6C3AE0248F5F704FDBEE600BF5B
:1099A000902B002000000000907B0020688C00209D
:1099B000A48B002000000034948B0020D8520D08A6
:1099C00030B5C369012B85B004D1404C94F8AC325A
:1099D000012B04D005B0BDE83040FDF725BCA4F54F
:1099E0008043DFED3B6AB3F9D2219FED3A0A07EEDF
:1099F000102AB3F9042207EE902AB8EEC77AF8EEDF
:109A0000E77AB4F99821B0EEC77AF0EEE77AB4EECF
:109A1000677A00EE902AF1EE10FAC8BFF0EE477AAE
:109A2000B8EEE07AD3ED900A03F6085270EEC70A5A
:109A300092ED007A27EE267AF5EEC00AF7EE006A7C
:109A4000F1EE10FAB4EEE67A48BFDFED220AF1EE4D
:109A500010FAD8BFB0EE667AF3EE046A77EEA71A72
:109A600067EEA67AC0EE876A14346D4693ED6B7A82
:109A7000194BB0EE612AA6EE872A93ED001AF4EE98
:109A8000427AF1EE10FA48BFB0EE672AF4EE421ABD
:109A9000F1EE10FAC8BFB0EE612A26F087FC94E818
:109AA0000F0007EE901A9FED0D7AF8EEE77A85E841
:109AB0000F00E0EE077A0A482946FDEEE77ACDED81
:109AC000017AFAF7C9F805B030BD00BF908B0020CD
:109AD0009A99193F00000000888000200000C842C9
:109AE000902B0020112070470048704768530D08E4
:109AF0000048704774530D080120704701207047DB
:109B000001207047012070470369002283F840213B
:109B100001207047174B184993EDD07AB3F9E02034
:109B2000D3F81402B5EEC07AF1EE10FA07EE902ADF
:109B3000C8BFDFED126AF8EEE77ACABF27EE267AD1
:109B400020EE270A27EE000A67EEA07ABDEEC00AD3
:109B5000FDEEE77A10EE102AC1F8702517EE902A74
:109B6000C1F87425036801F274525B6B01F5AE61B4
:109B7000184700BF908B0020907B00200000C84257
:109B80001E4BDFED1F6AB3F9E010A3F58050A3F57B
:109B90008043F5EEC00AD3F8402C8A42A8BF0A469B
:109BA00007EE902AF1EE10FAF8EEE77AD6BF03F648
:109BB000444393ED707A93ED007A27EE800A07EE26
:109BC000901ACCBF27EE267A27EE667AF8EEE77A6F
:109BD000BDEEC00AB4EEE77AF1EE10FA58BFB0EE6F
:109BE000677A60EE870A10EE102AFDEEE00AC0F8F0
:109BF000702510EE903AC0F874357047908B0020B5
:109C00000000C84237B52C4CD4F8283CB3F90820E2
:109C10001B8B07EE102A07EE903AD4F82C3CB8EED6
:109C2000C77AB3F908201B8BF8EEE77A054687EE72
:109C3000270A224807EE102A07EE903AB8EEC77AB4
:109C4000F8EEE77A8DED010AC7EE270ACDED000A9E
:109C500009F0D2FFDDED000A9DED010A28B128468A
:109C600003B0BDE83040FFF755BF04F58043D3F89B
:109C70009C23520405D4284603B0BDE83040FFF7CA
:109C80007FBFB3F9E03007EE903AF8EEE77A04F5DB
:109C9000405427EE800A67EEA00ABDEEC00AFDEE32
:109CA000E00A10EE103AC4F8703510EE903AC4F89D
:109CB000743503B030BD00BF904B0020A08E002053
:109CC00010B5044688F08AFC0146206900F50E7044
:109CD0000AF0E2F920B12046BDE81040FDF72EBBA6
:109CE000114803F07BFF206990F9D0304BB102F0AE
:109CF00039FA0E48F5F71CFABDE810400B48F5F7A5
:109D000011BB02F0A5FA206905F0FEFB0748F5F744
:109D10000FFA0648F5F706FB20469FED050ABDE859
:109D20001040FDF7EBBC00BF688C0020902B00209A
:109D3000000000000B207047004870478E560D0849
:109D400000487047EC530D08012070470120704710
:109D5000012070470020704738B53048F5F7D8FF2C
:109D60002E48F5F7B5FE2D48F5F796FC2B48102147
:109D7000F4F776FED8B12A4A936892699342D4BF29
:109D800000230123264C94F888207AB9A4F5805545
:109D900073B3231D0FCBA4F10C0585E80F00A4F5C8
:109DA000C040F9F7CBFC012384F8883038BD1D4A48
:109DB000B2F90C1C0029F9DD02F5804002F5405291
:109DC0008368D2F8F82F9FED187A9B1A07EE903A25
:109DD000F8EEE77A67EE877A07EE101AB8EEC77AE0
:109DE000F4EEC77AF1EE10FACCBF01230023C9E7E5
:109DF000A4F58044642394F97022D5F8700512FB11
:109E000003F2D4F8403C9A42A8BF1A465142C4F823
:109E1000402C26F039FCC5F87005C7E7902B0020D0
:109E2000908B0020904B00200AD7233CF0B52E4C9D
:109E30002DED028B251D074695E80F00A4F10C06B9
:109E400086E80F0083B0A4F5C040F9F769FA01462F
:109E5000A4F5C040FAF76CFBA4F50052002384F887
:109E60008830C2F8483F94F8EC31C3B394F81C3200
:109E70003BB13122A6F59351A4F5C04009F0CCFACC
:109E80002DE094F9A631032B02D118492C22F3E7D7
:109E9000013BDBB2012B22D83B69DB6A93F8A0308F
:109EA000022B1CD104F11401284615F0F9FE0F48CD
:109EB000B0EE408AFFF7D4FAB4EEC08AF1EE10FAA1
:109EC0000DD501AA0121284615F0C4FB38B1B4F81C
:109ED0009831642213FB02F3019A9342D5DC0120EE
:109EE00003B0BDEC028BF0BD908B002040790020C8
:109EF00010B52DED028B244B93F9A621012A03D036
:109F00000020BDEC028B10BDA3F58043B3F90442E1
:109F1000002CB8BF6442A4B22CB9B3F9D241002CD2
:109F2000B8BF6442A4B2194BD3F8040603689B6B14
:109F3000984730B116491748272209F06DFA0120D9
:109F4000DFE7154AA2F1200101F1100015F014FE1F
:109F50000028EFD1114B03F53E6093ED008A03F02A
:109F600043F807EE904AF8EEE77AB4EEE70AF1EE2E
:109F700010FA44BF07EE904AB8EE670AB4EEC08A02
:109F8000F1EE10FABCD5D5E7908B0020905B002055
:109F900040790020902B0020A48B00208880002096
:109FA00070B5474C94F8EC3188B0054693BB454DED
:109FB000B5F9043283EAE371A1EBE37189B205F5E7
:109FC0004054002955D1404801F0D2FB94F8163591
:109FD000002B3ED195F9DF31022B52D13B4D95F844
:109FE000513F9BB13A4905F5AC502CF0D7FF68B111
:109FF000012384F8B935282205F54861A5F580408C
:10A0000009F00AFA28BB002384F8B935012384F843
:10A0100016351EE094F9A631022BA4F500561AD18C
:10A0200003AD284615F0DAFA04F114030FCB85E8E6
:10A030000F0001A9A4F5C040FBF740F9D6F8483F4E
:10A04000052B06D1272206F55B61A4F5C04009F077
:10A05000E3F908B070BD88F0C1FAD6F8283FC01AFD
:10A06000B0F57A7FA3D92846FFF742FF00289ED09B
:10A07000EFE7002BB4BF4FF0FF33012384F8CC3F50
:10A08000A1E7012B0CD1104801F072FA40B10E4843
:10A09000F9F712FB0028B8BF4042B0F57A7F9DDB8C
:10A0A00095F9DF31042BD4D1084D95F8513F002BA1
:10A0B000ACD0074905F5AC502CF0ECFF97E700BF9A
:10A0C000908B0020904B0020902B0020906B002064
:10A0D000948B0020022070470048704769530D0898
:10A0E0000048704754930E08034B0022C3F87025B4
:10A0F000C3F87425704700BF907B002038B5094D28
:10A1000004462846F5F714F82846F5F70BF92046DB
:10A11000F5F720F92846F5F76BFC2046BDE83840F6
:10A12000FDF7FEBA902B00200D20704700487047C5
:10A13000D4540D0800487047DC540D0801207047C6
:10A140000120704701207047002380F8273080F8F5
:10A1500038300120704700000148002101F008BBA1
:10A16000902B00202DE9F041B44CD4E903322DEDC1
:10A17000088B1343A268134388B005460FD1B0483B
:10A18000F5F7C6FDAE48F5F7A3FC9FEDAE0A4620F5
:10A1900008B0BDEC088BBDE8F0415CF087BA0FF069
:10A1A00049FD90F87C32DB07E9D5B5F91C3095F80C
:10A1B000271009EE103AB5F9243008EE903AB8EEBF
:10A1C000C99AF8EEE88AA4F58056002940F0D780B5
:10A1D0009FED9DAA29EE0ABA0122FDEECB7AA4F5E5
:10A1E000C04017EE903AC6F8E034F9F753FBA8697F
:10A1F00000F57F700790B0EE408A29F037F9DFED67
:10A20000937A20EE270A26F009F90798F0EE409A93
:10A2100029F076F9A4F5C040F0EE40AAFCF7F2FC74
:10A22000002878D1271D97E80F0005F1280C8CE84D
:10A230000F0097E80F0006F6F47C8CE80F0004F19D
:10A24000140C8CE80F00D4ED067A8148F8EEE77A1A
:10A25000F0EE680A77EE8B7AB0EE690AFDEEE77AE7
:10A26000C4ED067A15F0C2FD002386F8493595F94C
:10A270002630734803EB830303EB83039B00012128
:10A28000A6F80E35F4F780F896F85885B8F1000F67
:10A2900075D1704B9FED707AB3F9A83107EE903A03
:10A2A000F8EEE77A67EE877AF4EEE7AAF1EE10FAB5
:10A2B00065DD59F047FC074619EE900AF2F724F9DC
:10A2C000CDE9040118EE900AF2F71EF9CDE902017A
:10A2D00019EE100AF2F718F9604ACDE900010621DB
:10A2E000384652F0CFFD88F079F9C6F8CC84C6F82C
:10A2F000B80488F073F90123C6F8C80429EE8A0A65
:10A3000085F8273026F0B4F8BDEEC00A10EE103AFA
:10A31000C6F8D03433E088F061F9D6F86835C01A51
:10A3200042F2107398427FF67DAFF0EE087AF4EEB9
:10A33000E7AAF1EE10FA7FF775AFBCEEC88A04F118
:10A34000140718EE103A9BB208EE103AB8EEC88A1D
:10A35000B4EEC89AF1EE10FA47D859F0F3FB404A30
:10A36000062152F08FFD231D0FCB87E80F0001233C
:10A3700085F827300321A4F5C040F4F705F83048EC
:10A380000BF0EEF830B12E480321F3F7FDFF002368
:10A3900085F82730D6F85C35012B40F0B080A368F3
:10A3A000EA6A9FED29AA9B1A07EE903AD6F8D034B4
:10A3B0000133F8EEE79A5BD0DFED2A7AE9EE0A7A0C
:10A3C000F4EEE79AF1EE10FA0ADA274905F12800CF
:10A3D00015F066FCF4EEC08AF1EE10FA00F28F8000
:10A3E00017480321F3F7D0FF89E059F0ABFB1F4A70
:10A3F000062152F047FD04F1040C9CE80F0005F122
